:100000000C9424090C9443090C9443090C94D509CD
:100010000C940B0A0C9443090C9443090C94430967
:100020000C9443090C9443090C9443090C94430920
:100030000C9443090C9443090C9443090C94360D19
:100040000C9443090C9443090C9443090C94430900
:100050000C94B76C0C9468640C9443090C94430999
:100060000C9443090C943D650C9443090C94316540
:100070000C9443090C9443090C9443090C944309D0
:100080000C94EA770C9443090C9443090C944309AB
:100090000C947B650C9443090C946F650C94430994
:1000A0000C9443090C9443090C9443090C944309A0
:1000B0000C9443090C9443090C9443090C94430990
:1000C0000C9443090C9443090C9443090C94430980
:1000D0000C9443090C9443090C9443090C94430970
:1000E0000C9443090C94706C0C947A6C0C94666CB0
:1000F0000C94266C0C94AB6C0C949C6C0C94906CD3
:100100000C94846C0C9443090C9443090C9443099B
:100110000C9443090C9443090C9443090C9443092F
:1001200023814281C181B082D082F082F882A5828F
:10013000084AD73B3BCE016E84BCBFFDC12F3D6C4E
:1001400074319ABD56833DDA3D00C77F11BED9E4B4
:10015000BB4C3E916BAAAABE000000803F076342E1
:1001600036B79BD8A71A39685618AEBAAB558C1D4E
:100170003CB7CC5763BD6DEDFD753EF6177231BFD0
:10018000000000803F08000000BE922449123EABF0
:10019000AAAA2ABECDCCCC4C3E00000080BEABAAA1
:1001A000AAAA3E00000000BF000000803F0000003F
:1001B0000000084178D3BB4387D1133D190E3CC3DF
:1001C000BD4282AD2B3E68EC8276BED98FE1A93E5E
:1001D0004C80EFFFBE01C4FF7F3F00000000002500
:1001E000730A005854414C5F5452494D3D256400F8
:1001F00025730A0025730A00546573742036202580
:10020000730A005465737420352025730A00546501
:10021000737420342025730A0054657374203320CE
:1002200025730A005465737420322025730A005424
:1002300065737420312025730A006368616E3D2563
:10024000640A0074787077723D25640A0035303096
:100250006B0A003235306B0A003131356B0A0035DC
:10026000366B0A0033386B0A0025730A00765F6C20
:100270006F773D252D332E32660A0025730A0073F1
:10028000656E743D252D75206475703D252D752096
:1002900069676E6F7265643D252D752074746C5F9F
:1002A0007A65726F3D252D750A0025372E3366203D
:1002B00025372E33660025352E32662000457272B2
:1002C0006F72203020566F6C74004E6F74207375FF
:1002D00070706F727465640A004572726F722030BC
:1002E00020566F6C74004572726F72203020566F0A
:1002F0006C7400256C7500416C6C6F7765642073BD
:100300007065656420312F31302F3130302F34301B
:1003100030206B6269742F730025630074746C3D28
:10032000252D64200074746C3D252D6420004E65DD
:10033000772074746C3D252D6420002563004D5397
:100340003536313120503D252D372E326620252D72
:10035000372E32666D0A00424D5030383520256CFC
:10036000642050612020252D372E32666D002563D4
:1003700000545F484541545F4944583D252D352E72
:1003800032662000545F4445573D252D352E326698
:10039000200041483D252D352E32662000545F5304
:1003A000485432583D252D352E3266200052485F84
:1003B00053485432583D252D352E32662000545F67
:1003C00052483D252D342E3166200052483D252DC2
:1003D000342E316620002563002563002563002547
:1003E00063002563007265706F72745F616C6C3DB1
:1003F000007265706F72743D0025630025630025EF
:100400006300256300204F534343414C3D25642046
:100410000020467573653A2065653D2530327820A9
:1004200068663D25303278206C663D253032782074
:100430006C623D25303278004D43553D2530366C99
:10044000780025630074785F6C656E3D252D6C75B2
:100450002C765F6C6F773D252D6C752C736874322C
:10046000783D252D6C750A002563004F4B0A002549
:100470006300256300256300256300256300256371
:100480000025630025630064656275675F616C6CBD
:100490003D0064656275673D0064656275673D0097
:1004A00025730A00646565700A006E6F6E650A0048
:1004B000707772733D00696E74725F7365635F700D
:1004C000313D252D372E33660A00696E74725F70D8
:1004D000313D252D6C640A00696E74725F7365632B
:1004E0005F70303D252D372E33660A00696E7472B9
:1004F0005F70303D252D6C640A00765F6D63753D3D
:10050000252D352E32660A00745F6D63753D252DED
:10051000352E32660A00707077723D25730A0064CA
:10052000656275673D0072636D643D25730A002541
:10053000730A006175746F0A006C6F675F6D6F649A
:10054000653D007573625F7077723D25730A0072B6
:10055000656C61793D25730A0074746C3D252D64CA
:100560000A0052494D455F616464723D252D642E39
:10057000252D640A006E65696768626F725F746139
:10058000626C655F73697A653D25640A00765F6C0D
:100590006F773D252D332E32660A00747870773DD3
:1005A00025640A006368616E3D25640A0069643D44
:1005B000006932635F6275733D006932635F737017
:1005C0006565643D252D6C750A007478743D25734E
:1005D0000A0053797374656D2053756D6D6172797E
:1005E0000A006D61736B3D002C00696E7465727654
:1005F000616C3D252D750023252D642C00745F68EA
:100600006561745F69647800745F64657700616830
:1006100000705F6D73353631310072685F736874D6
:10062000327800745F736874327800706100700013
:1006300061643400616433006164320061643100DC
:10064000613300613200613100765F696E0072686B
:100650000065727200757074696D650070315F6C51
:1006600073740070315F740070310070305F6C73B0
:10067000740070305F7400703000765F6D637500D9
:10068000745F6D63750074310074006964006536D1
:100690003400747874002D002B006175746F006E47
:1006A0006F6E6500706F7765725F736176655F6C02
:1006B000656472790072656C61795F6C656479005C
:1006C000636F6D7061737300616363656C0070725A
:1006D000657300705F707772006165730070315FE1
:1006E0006C6564790070305F6C6564720065766576
:1006F0006E74006C6564006F7700706B74007478C2
:100700005F6C6564790072785F6C656472006F700D
:100710006572006E6F6E65002530327800765F611D
:1007200064343D252D382E3666002000765F6164E6
:10073000333D252D382E3666002000765F61643209
:100740003D252D382E3666002000765F6164313DF0
:10075000252D382E3666002000765F6C6967687438
:100760003D252D382E3666002000765F61323D250E
:100770002D372E3366002000765F61313D252D3701
:100780002E3366002000765F696E3D252D352E32B2
:100790006600204E657665722D75736564207374EE
:1007A00061636B203E2025642062797465730A00C2
:1007B000757074696D653D252D642D646179732DA7
:1007C000253032643A253032643A253032642D685F
:1007D0006F7572730A0074657374205B6F66667C54
:1007E000317C327C337C347C355D202020202020FD
:1007F00020202D2074657374206D6F6465730A0D5D
:10080000007478205B706B74207061796C6F616428
:100810005D2020202020202020202020202D20733B
:10082000656E6420726164696F20706B74206B6503
:1008300079626F6172640A0D00776474205B6F6E79
:100840007C6F66667C746573745D20202020202098
:1008500020202020202D207761746368646F670A50
:100860000D00765F6C6F77205B765F6C6F775D2035
:1008700020202020202020202020202020202D206B
:100880006C6F77657374207265706F727420766F09
:100890006C746167650A0D007570677220202020F6
:1008A0002020202020202020202020202020202048
:1008B000202020202D207265626F6F742076696180
:1008C00020626F6F746C6F616465720A0D007561F0
:1008D0007274205B33386B7C35366B7C3131356B11
:1008E0007C3235306B7C3530306B5D202D2073656C
:1008F00074207465726D2F756172742073706565F4
:10090000640A0D00626F6F742020202020202020B8
:1009100020202020202020202020202020202020D7
:100920002D207265626F6F740A0D007077727320EC
:100930005B646565707C6E6F6E655D202020202095
:10094000202020202020202D206D637520736C65D1
:100950006570206D6F64650A0D00726573742065A3
:100960006570726F6D202020202020202020202004
:100970002020202020202D20726573746F72652046
:10098000656570726F6D0A0D0070707772205B6F15
:100990006E7C6F66665D2020202020202020202095
:1009A00020202020202D2070726F6772616D6D6194
:1009B000626C65207077720A0D00747874205B7326
:1009C0007472696E675D2020202020202020202066
:1009D0002020202020202D20536574207265706F08
:1009E0007274207465787420737472696E670A0D6E
:1009F0000074787077205B31352D305D2020202009
:100A0000202020202020202020202020202D2054A5
:100A100058205077722E20486967686573742030BB
:100A200020283364426D290A0D0074746C205B30F9
:100A30002D31355D20202020202020202020202046
:100A40002020202020202D2074696D652D746F2DAD
:100A50006C69766520666F72207061636B65747374
:100A60000A0D007373202020202020202020202029
:100A70002020202020202020202020202020202D69
:100A80002073797374656D2073756D6D6172790A69
:100A90000D007273202020202020202020202020E4
:100AA00020202020202020202020202020202D2039
:100AB000726164696F2073746174730A0D007269E6
:100AC000205B236E5D205B696E745D2020202020FA
:100AD000202020202020202020202D207265706FD3
:100AE000727420696E74657276616C0A0D007263AF
:100AF0006D64205B6F6E7C6F66665D202020202019
:100B0000202020202020202020202D20616C6C6FB0
:100B10007720636D642066726F6D206E65746F72EE
:100B20006B0A0D007265205B236E5D205B2B7C2DB4
:100B30005D205B6D61736B7C6175746F2C6D61738F
:100B40006B5D202D206D6F7465207265706F7274FF
:100B5000207365742F6D6F646966790A0D006F7775
:100B60002020202020202020202020202020202085
:100B7000202020202020202020202D206F6E652D79
:100B8000776972652073656E736F72730A0D006CFE
:100B90006F67205B6175746F7C6F6E7C6F66665DDE
:100BA00020202020202020202020202D206D6F7448
:100BB00065732064617461206F6E205553420A0D85
:100BC000006E65205B666C7573685D2020202020B8
:100BD000202020202020202020202020202D206EBA
:100BE00065696768626F72207461626C650A0D00E6
:100BF000657272202020202020202020202020200C
:100C00002020202020202020202020202D20657240
:100C1000726F722073746174730A0D006D637520B6
:100C200020202020202020202020202020202020C4
:100C300020202020202020202D206D637520696E2B
:100C4000666F0A0D00693263205B70726F62657CAB
:100C5000737065656420236E5D2020202020202095
:100C6000202D206932632070726F62652062757377
:100C70007C736574206275732073706565640A0DFA
:100C8000006964205B72657365745D2020202020FC
:100C9000202020202020202020202020202D2069FE
:100CA000642068616E646C696E670A0D0068756D1A
:100CB0002020202020202020202020202020202034
:100CC0002020202020202020202D2068756D6964A0
:100CD0006974792073656E736F720A0D0072656CAA
:100CE0006179205B6F6E7C6F66667C737461747370
:100CF0005D20202020202020202D2072656C61792D
:100D0000206E6574776F726B207265706F7274738A
:100D10000A0D006465205B6D61736B5D20202020EF
:100D20002020202020202020202020202020202DB6
:100D30002064656275670A0D006368616E205B312F
:100D4000312D32365D202020202020202020202020
:100D500020202020202D206368616E2031312D322B
:100D6000362028322E3430352D32343830204D683C
:100D70007A290A0D0063616C69205B5B765F696E9E
:100D80007C61317C61325D20766F6C747C7265733E
:100D900065747C6E6F6E655D202D2063616C696289
:100DA000726174650A0D0061646320202020202098
:100DB0002020202020202020202020202020202033
:100DC0002020202D2073686F7720765F696E2C209D
:100DD00061312C20613220766F6C74616765730A13
:100DE0000D007520202020202020202020202020E1
:100DF00020202020202020202020202020202D20E6
:100E0000757074696D650A0D007620202020202001
:100E100020202020202020202020202020202020D2
:100E200020202020202D2076657273696F6E0A0DB8
:100E3000006820202020202020202020202020208A
:100E4000202020202020202020202020202D20684D
:100E5000656C700A0D00256300756E6B6E6F776EA2
:100E600020636D640A00484D4335383833002573DC
:100E700000257300202573002025362E32662000C1
:100E8000253032780074656D705F65787465726EB8
:100E90003D252D362E326600202573002025362E66
:100EA0003266204F6E2D426F6172640025303278B9
:100EB0000074656D705F626F6172643D252D362E22
:100EC0003266000A00503A20256C642050612020D0
:100ED000252D372E3266206D0A002563002563001C
:100EE0004932433A2000452025642E256420636C56
:100EF0006F636B20256C752063707520256C7520E1
:100F00006C706D20256C752069727120256C7520C0
:100F1000676C656420256C7520796C656420256C90
:100F20007520726C656420256C7520747820256CA2
:100F300075206C697374656E20256C752073656E01
:100F4000736F727320256C752073657269616C20F4
:100F5000256C750A00532025642E256420636C6F70
:100F6000636B20256C7520747820256C7520727851
:100F700020256C752072747820256C75207272782B
:100F800020256C75207265786D697420256C75203C
:100F900061636B747820256C75206E6F61636B7470
:100FA0007820256C752061636B727820256C752024
:100FB00074696D65646F757420256C752062616459
:100FC00061636B727820256C7520746F6F6C6F6E27
:100FD0006720256C7520746F6F73686F727420259D
:100FE0006C752062616473796E636820256C75206E
:100FF00062616463726320256C7520636F6E746533
:101000006E74696F6E64726F7020256C75207365E5
:101010006E64696E6764726F7020256C75206C6CED
:10102000747820256C75206C6C727820256C750A9C
:1010300000257325730A004F6E6C696E650A000AFD
:10104000002C20636865636B2072617465202575D0
:1010500020487A0025732025732C206368616E6E0A
:10106000656C20257520706F776572202575000AE4
:101070000025783A004D41432061646472657373C2
:10108000200052616E646F6D2045554936342061F1
:101090006464726573732067656E657261746564FC
:1010A0000A000A2A2A2A2A2A2A2A426F6F74696E9B
:1010B000672025732A2A2A2A2A2A2A0A0045455007
:1010C000524F4D20697320636F72727570742C20BB
:1010D000726577726974696E6720776974682064D5
:1010E000656661756C74732E0A006C6F63616C6861
:1010F0006F73740041544D45474131323872666117
:101100003100020000FFFE0000016E616E00696E9A
:10111000660000407A10F35A00A0724E18090010C1
:10112000A5D4E80000E87648170000E40B5402005C
:1011300000CA9A3B000000E1F50500008096980087
:10114000000040420F000000A086010000001027B0
:1011500000000000E8030000000064000000000040
:101160000A00000000000100000000002C76D88872
:10117000DC674F0823DFC1DFAE59E1B1B796E5E385
:10118000E453C63AE651997696E8E6C28426EB899E
:101190008C9B62ED407C6FFCEFBC9C9F40F2BAA53B
:1011A0006FA5F490055A2AF75C936B6CF9676DC1D3
:1011B0001BFCE0E40D47FEF520E6B500D0ED902ED7
:1011C0000300943577050080841E080000204E0A35
:1011D000000000C80C333333330F986E1283114173
:1011E000EF8D2114893BE65516CFFEE6DB18D1843E
:1011F0004B381BF77C1D901DA4BBE4242032847265
:101200005E228100C9F124ECA1E53D274E414E4903
:101210004E495459494E46CDCCCC3D0AD7233C17B4
:10122000B7D13877CC2B329595E6241FB14F0A0001
:101230000020410000C84200401C4620BCBE4CCAF1
:101240001B0E5AAEC59D740011241FBECFEFD1E412
:10125000DEBFCDBF19E0A0E0B2E0E6EDFBE201E0C9
:101260000BBF02C007900D92AE3BB107D9F711E357
:10127000AEEBB9E001C01D92A33DB107E1F70E94BA
:10128000C7830C94E9950C9400008115910511F029
:101290000197F1F7089580EB94E09F938F930E945C
:1012A000C2928091580290915902A0915A02B09135
:1012B0005B020F900F9093FF03C08AEA94E002C094
:1012C00084EA94E09F938F930E94C2920F900F90B4
:1012D0000895E091771BEF73F0E0E453F44E8083C0
:1012E0008091771B8F5F8093771B80910D29886099
:1012F00080930D294EE352E061E1CA010E944854F7
:1013000080E090E00895CF93DF93EC018091C509D0
:101310009091C60986FF1DC08E811F928F938D818B
:101320001F928F938C811F928F938B811F928F932B
:101330008A811F928F9385E693E09F938F930E94FB
:10134000B0928DB79EB70C960FB6F8949EBF0FBEA5
:101350008DBFBE018CEF99E00E947A55BE0184E0FA
:1013600092E0DF91CF910C94EF548823B9F052981A
:101370005A981DBA80916900806280936900EA9A48
:1013800053985B98EB9A809169008068809369001C
:1013900080916800816080936800089510926900D0
:1013A0005A9AEA985B9AEB9808951F920F920FB69B
:1013B0000F9211248F939F93AF93BF9380916800F6
:1013C00080FF20C08091E8289091E928A091EA2828
:1013D000B091EB280196A11DB11D8093E828909350
:1013E000E928A093EA28B093EB288091C509909151
:1013F000C60987FF07C0749882E090E09093850249
:1014000080938402BF91AF919F918F910F900FBEF7
:101410000F901F9018951F920F920FB60F921124E4
:101420008F939F93AF93BF938091680080FF20C0FC
:101430008091EC289091ED28A091EE28B091EF28B2
:101440000196A11DB11D8093EC289093ED28A093E7
:10145000EE28B093EF288091C5099091C60990FFBE
:1014600007C0739882E090E0909385028093840295
:10147000BF91AF919F918F910F900FBE0F901F90D2
:10148000189580937C0080917B00877F80937B0000
:1014900080917C00806C80937C0085E080937A0052
:1014A00080917A00806880937A0080917B0087FF2A
:1014B000FCCF80917B0085FFFCCF80917A00806417
:1014C00080937A0080917A0086FDFCCF109279009B
:1014D0001092780084E090E060E070E020917A0063
:1014E000206420937A0020917A0026FDFCCF209181
:1014F000780030917900620F731F0197009771F7A0
:1015000010927C0080917A008F7780937A00769594
:1015100067957695679580E090E00E941D89089513
:1015200080E00E94410A20917C0230917D0240912E
:101530007E0250917F020E94018B21EE3AE744E93E
:101540005EE30E94B68708950F931F93CF93DF93B6
:10155000CFE1D0E00BE51EE0C093510187EC90E0B5
:101560000E9445098091510185FD0DC0C031D10512
:1015700021F02CF00B54110904C004EC19E00253C3
:1015800011092197E9CFB80180E090E00E941D8900
:1015900020E030E04AE754E40E948088DF91CF9158
:1015A0001F910F910895CF93DF93EC01888199816A
:1015B000009799F08636904121F01982188283E0D5
:1015C00011C0623171F40E94A40A60933F247093A9
:1015D0004024809341249093422486E690E19983AD
:1015E000888381E0DF91CF91089580917B008860AE
:1015F00080937B0089EC80937C0085E080937A0067
:1016000080917A00806880937A0080917B0087FFC8
:10161000FCCF80917B0085FFFCCF80917A008064B5
:1016200080937A0080917A0086FDFCCF80917A00C9
:10163000806480937A0080917A0086FDFCCF60916F
:1016400078007091790080917A008F7780937A008A
:1016500080E090E00E941D8927ED33EA40E95FE3D6
:101660000E94018B26E636E648E853E40E94B587DF
:101670000895BF92CF92DF92EF92FF920F931F9344
:10168000CF93DF93CDB7DEB729970FB6F894DEBFBF
:101690000FBECDBF6C011092BE098FEF898708E89D
:1016A0001BE1B12C7E0189E0E80EF11C89858823BD
:1016B000E9F1E8E0BE16E1F1BE016F5F7F4FC701BF
:1016C0000E94E35D89858F3F11F08E3F19F480936E
:1016D000BE092CC0CE010196C114D10471F40E9440
:1016E000FC5D80930A29FE013196A2E0B9E2819166
:1016F0008D93EE15FF05D9F71DC00E94FC5DF80122
:101700008083FE01319620E030E0A8014850510965
:101710008191DA01A20FB31F8C932F5F3F4F2830C6
:101720003105B1F7B394075F1F4FC0CF8B2D03C0B6
:1017300088E001C081E029960FB6F894DEBF0FBEA5
:10174000CDBFDF91CF911F910F91FF90EF90DF9070
:10175000CF90BF90089583EC9EE09F938F930E945B
:10176000C2920F900F9008952F923F924F925F92E6
:101770006F927F928F929F92AF92BF92CF92DF92A1
:10178000EF92FF920F931F93CF93DF93EC014B01E6
:10179000009711F427E004C08130910549F426E058
:1017A0004AE250E06BE270E089E290E00E94C35CA4
:1017B000CE010E94390B9E012154364F5901D901A7
:1017C0008C93CD2B69F098E8C92E9BE1D92EC0E807
:1017D000DBE1E12CF12C24E7222E2EE0322EA6C0F4
:1017E00082E099E20E94315FBC01882777FD8095F5
:1017F000982F0E941F896B017C01892869F020E0E5
:1018000030E048EC52E40E9480889F938F937F934E
:101810006F9381EB9EE0ACC0C2E0D9E20CEA1EE01F
:1018200089911F928F931F930F930E94C2920F90E2
:101830000F900F900F90B9E2CA30DB0789F720E0D4
:1018400030E048EC52E4C701B6010E9480889F93C3
:101850008F937F936F938CE99EE09F938F930E9469
:10186000C2920F900F900F900F900F900F90809159
:101870000A29882319F084E993E002C088E094E003
:101880009F938F9388E99EE09F938F930E94C292CB
:101890000F900F900F900F9075C000E010E0FE01C8
:1018A000E00FF11F80811F928F93A0E8BEE0BF93ED
:1018B000AF930E94C2920F5F1F4F0F900F900F9037
:1018C0000F900830110559F720E030E048EC52E461
:1018D000C301B2010E9480889F938F937F936F937F
:1018E000A8E7BEE0BF93AF930E94C2920F900F9003
:1018F0000F900F900F900F90D6018C91882309F4D0
:1019000055C084E993E09F938F933F922F920E945A
:10191000C2920E94AB0BBFEFEB1AFB0AE9E0CE0EBE
:10192000D11C29960F900F900F900F90D5018C919C
:1019300090E0E816F906ECF5CE010E94315FBC019B
:10194000882777FD8095982F0E941F892B013C01E5
:101950008114910409F4A1CF20E030E048EC52E476
:101960000E9480889F938F937F936F9385E89EE07A
:101970009F938F930E94C2920F900F900F900F90A1
:101980000F900F90DF91CF911F910F91FF90EF90EB
:10199000DF90CF90BF90AF909F908F907F906F908F
:1019A0005F904F903F902F900C94AB0B88E094E0A9
:1019B000AACFDF91CF911F910F91FF90EF90DF9011
:1019C000CF90BF90AF909F908F907F906F905F90DF
:1019D0004F903F902F900895CF93DF9300D0CDB7D5
:1019E000DEB7809103298983809109298A83CE01FA
:1019F00001960E943C520F900F90DF91CF91089575
:101A0000CF93DF93EC01209102293091032940917B
:101A10000429509105296091062970910729809128
:101A2000082990910929AFEF0E94318EE1F427E057
:101A30004AE250E06BE270E089E290E00E94C35C11
:101A400080E090E00E94390BC154D64F888349E072
:101A500050E06AE070E082E099E20E943494DF9105
:101A6000CF910C94EC0CDF91CF9108951F920F92BF
:101A70000FB60F9211240BB60F92DF92EF92FF92E6
:101A80000F931F932F933F934F935F936F937F9386
:101A90008F939F93AF93BF93CF93DF93EF93FF9376
:101AA00080910D29826080930D298091580286FDD6
:101AB0002B9A8091580287FD2B9A809184029091F5
:101AC00085021816190614F4749A739A8091C50940
:101AD0009091C60985FF02C07498739880910202A4
:101AE0009091030201979093030280930202892B45
:101AF00009F03DC18091D3099091D409019690934A
:101B0000D4098093D3098091432490914424A091D7
:101B10004524B09146240196A11DB11D8093432414
:101B200090934424A0934524B093462480E190E010
:101B300090930302809302028091580280FD02C0BC
:101B40001D9B07C01092C3091092C20983B7817F01
:101B500009C081E090E09093C3098093C20983B7E4
:101B6000817F866083BF8091C5099091C60997FFE8
:101B700008C08091C2099091C309892B61F0749AC1
:101B8000739807E21BE1C4E5D4E234E0E32EF12CC4
:101B9000DD24D3941FC0739A7498F3CF8091D30936
:101BA0009091D40901960E94028C892BD1F0F80102
:101BB000608571856115710509F5F801608571858C
:101BC0006115710569F5065F1F4F2596FBE10F341E
:101BD0001F07D1F1F801608571856115710539F331
:101BE000DDCF77988091C5099091C60992FFDFCF2C
:101BF0007498F0928502E0928402D9CF8091D30943
:101C00009091D40901960E94028C892BB1F61C8216
:101C10001B82AE0162E186E192E00E944854CDCF82
:101C20008091D3099091D4090E94028C892B59F696
:101C3000D8821A8309831C821B82AE0162E184E38D
:101C400092E00E944854BFCF60915E0270915F02A3
:101C500061157105A1F18091D3099091D4090E9479
:101C6000028C892B61F58091E8289091E928A09158
:101C7000EA28B091EB284091351C5091361C6091B8
:101C8000371C7091381C841B950BA60BB70B8093E7
:101C90004F1B9093501BA093511BB093521B8091EC
:101CA000E8289091E928A091EA28B091EB28809348
:101CB000351C9093361CA093371CB093381C609150
:101CC0005C0270915D0261157105A1F18091D309EB
:101CD0009091D4090E94028C892B61F58091EC28A7
:101CE0009091ED28A091EE28B091EF284091391CF9
:101CF00050913A1C60913B1C70913C1C841B950BCD
:101D0000A60BB70B8093531B9093541BA093551BAA
:101D1000B093561B8091EC289091ED28A091EE286D
:101D2000B091EF288093391C90933A1CA0933B1CF0
:101D3000B0933C1C8091580286FD2B9880915802EC
:101D400090915902A0915A02B0915B0291FF0FC08D
:101D50000E94E2688A3119F0C1E0C80F01C0CBE0EF
:101D60000E949C678C2F0E94FA680E94E46740E002
:101D700050E060E086E892E00E944854FF91EF91C5
:101D8000DF91CF91BF91AF919F918F917F916F9193
:101D90005F914F913F912F911F910F91FF90EF9085
:101DA000DF900F900BBE0F900FBE0F901F901895F5
:101DB0008091771B90915324891B08950E94D80E1F
:101DC000882371F0E0915324EF73F0E0E453F44E74
:101DD000808190E0209153242F5F20935324089515
:101DE0008FEF9FEF0895CF93DF93EC011092F009EE
:101DF0001092EF09888199810097C1F08A3793404A
:101E000021F01982188283E0B8C0613109F0B4C0B2
:101E1000F89478940E94DE0E99279093EB098093B2
:101E2000EA098D3009F443C08F3F49F40E94D80E6F
:101E30008111EECF8AE793E0998388839DC0823138
:101E4000910509F45AC08F37910509F052C080916D
:101E5000E8099091E909181619060CF56091CD3141
:101E60007091CE3188E090E00E947E926091CD31F9
:101E70007091CE3180E290E00E947E926091CD31EF
:101E80007091CE3188E090E00E947E928091E809C6
:101E90009091E90901979093E9098093E80980916D
:101EA000E8099091E9098F37910509F0BFCF1092A9
:101EB00053241092771B8091E8099091E909FC0165
:101EC000E859FB4D10829093F0098093EF0910922E
:101ED000E9091092E80980910B2990910C2900974B
:101EE00009F4A4CF40E050E06091FE110E944854F4
:101EF0009DCF8830910571F5AACF6091CD31709159
:101F0000CE318DE090E00E947E921092E70910920F
:101F1000E6098091E6099091E7092091E80930915E
:101F2000E909821793070CF0BACFFC01E859FB4D81
:101F300080816091CD317091CE3190E00E947E928F
:101F40008091E6099091E70901969093E7098093C3
:101F5000E609DFCF6091CD317091CE310E947E9243
:101F60008091E8099091E9092091EA09FC01E8597A
:101F7000FB4D208301968FCF81E0DF91CF910895B3
:101F80008091C2099091C309892BD1F080915802A8
:101F900090915902A0915A02B0915B0293FD10C03A
:101FA0000E949C6783B7817F866083BFF89483B764
:101FB000816083BF7894889583B78E7F83BF789440
:101FC0000895CF93DF93EC0188819981009719F0F0
:101FD0008939904199F40E9459660E94C00F40E0EF
:101FE00050E065E880910212909103120E944854DB
:101FF00089E990E19983888381E003C0198218827E
:1020000083E0DF91CF910895CF93DF9300D0CDB7D8
:10201000DEB7892B81F05F934F9381E79EE09F931A
:102020008F9369837A830E94C2920F900F900F90D2
:102030000F907A8169817F936F938EE69EE09F93E4
:102040008F930E94C2920F900F900F900F900F905D
:102050000F90DF91CF910895FF920F931F93CF932D
:10206000DF930E94596680EB0E94BE5F81111CC005
:102070000E94226080913D2090913E20816090934B
:102080003E2080933D208DE993E09F938F938EE6D1
:102090009EE09F938F930E94C2920F900F900F909B
:1020A0000F90C1E0D0E002C0C0E0D0E0FEB08F2DC4
:1020B0008470F82E729A0E9459668EE40E94BE5F68
:1020C000811116C00E94226080913D2090913E2097
:1020D000826090933E2080933D208E010F5F1F4FC2
:1020E00043E259E065EA73E0CE010E940410E80182
:1020F000F11001C072980E9459668EEE0E94BE5F78
:10210000811116C00E94226080913D2090913E2056
:10211000846090933E2080933D208E010F5F1F4F7F
:1021200043E259E06DEA73E0CE010E940410E80139
:102130000E94596686EA0E94BE5F811116C00E9405
:10214000226080913D2090913E20886090933E20B7
:1021500080933D208E010F5F1F4F43E259E064EBF7
:1021600073E0CE010E940410E8010E9459668CE3DE
:102170000E94BE5F81111EC00E94226080913D209E
:1021800090913E20806190933E2080933D208E016F
:102190000F5F1F4F43E259E06CEB73E0CE010E94EA
:1021A000041086E69EE09F938F930E94C2920F9048
:1021B0000F90E8010E94596682ED0E94BE5F811176
:1021C00016C00E94226080913D2090913E20806246
:1021D00090933E2080933D208E010F5F1F4F43E27E
:1021E00059E064EC73E0CE010E940410E8010E9403
:1021F000596680E80E94BE5F811116C00E9422606D
:1022000080913D2090913E20916090933E2080935C
:102210003D208E010F5F1F4F43E259E06DEC73E0EC
:10222000CE010E940410E8010E94596680ED0E94D0
:10223000BE5F811116C00E94226080913D20909166
:102240003E20806890933E2080933D208E010F5F5A
:102250001F4F43E259E063ED73E0CE010E9404108A
:10226000E8010E9459668CEE0E94BE5F811116C083
:102270000E94226080913D2090913E209260909338
:102280003E2080933D208E010F5F1F4F43E259E0B7
:102290006BED73E0CE010E940410E80107E010E04E
:1022A0000E9459668CE70E94BE5F811113C00E9494
:1022B000226080913D2090913E20806490933E204A
:1022C00080933D2043E259E062EE73E0CE010E942C
:1022D000041005C0015011090115110509F70E94EC
:1022E0002260DF91CF911F910F91FF900C94AB0B67
:1022F000CF93DF9300D0CDB7DEB74A8369830E94C6
:10230000F95F6981862F0E942A604A81842F0E948A
:102310002A600F900F90DF91CF910C942260AF92C2
:10232000BF92DF92EF92FF920F931F93CF93DF93B1
:1023300000D01F92CDB7DEB7182FD22E4A835B8311
:1023400069830E94F95F6981862F0E942A60812F2C
:1023500081600E9420604A81A42E5B81B52E00E03E
:1023600010E0ED2CF12C81E0E81AF1080D1580F455
:102370000E151F0519F40E94456002C00E943B60C3
:10238000F50180830F5F1F4FFFEFAF1ABF0AEECF3B
:102390000F900F900F90DF91CF911F910F91FF90B1
:1023A000EF90DF90BF90AF900C942260AF92BF92FD
:1023B000CF92DF92EF92FF920F931F93CF93DF9311
:1023C000CDB7DEB760970FB6F894DEBF0FBECDBFB6
:1023D000B82EA42E6623E9F18E010F5F1F4F80E116
:1023E000F80111928A95E9F728E0A80168E980EBE5
:1023F0000E948F11BB2041F02BEE33E03F932F93CF
:102400000E94B0920F900F906E01F8E0CF0ED11C99
:1024100052EFE52E53E0F52EF80181918F011F92C6
:102420008F93FF92EF920E94B0920F900F900F90B7
:102430000F900C151D0581F788851F928F9327E457
:1024400034E03F932F930E94B0920F900F900F9023
:102450000F90AA20E9F18E010F5F1F4F80E1F80174
:1024600011928A95E9F728E0A80160E880EB0E94C4
:102470008F11BB2041F087EF93E09F938F930E94D1
:10248000B0920F900F906E01F0E1CF0ED11C42EF91
:10249000E42E43E0F42EF80181918F011F928F9377
:1024A000FF92EF920E94B0920F900F900F900F90BA
:1024B0000C151D0581F788851F928F9387E494E0A2
:1024C0009F938F930E94B0920F900F900F900F9058
:1024D00060960FB6F894DEBF0FBECDBFDF91CF91EF
:1024E0001F910F91FF90EF90DF90CF90BF90AF9032
:1024F0000895CF93DF9300D0CDB7DEB71A8219824B
:1025000022E0AE014F5F5F4F6AEA8EEE0E948F11AC
:10251000898190E0982F88272A81822B90930D1C27
:1025200080930C1C22E0AE014F5F5F4F6CEA8EEE91
:102530000E948F11898190E0982F88272A81822B11
:1025400090930F1C80930E1C22E0AE014F5F5F4FF3
:102550006EEA8EEE0E948F11898190E0982F882775
:102560002A81822B9093111C8093101C22E0AE01D3
:102570004F5F5F4F60EB8EEE0E948F11898190E07C
:10258000982F88272A81822B90931F1C80931E1CD2
:1025900022E0AE014F5F5F4F62EB8EEE0E948F1123
:1025A000898190E0982F88272A81822B9093211C83
:1025B0008093201C22E0AE014F5F5F4F64EB8EEEF4
:1025C0000E948F11898190E0982F88272A81822B81
:1025D0009093231C8093221C22E0AE014F5F5F4F3B
:1025E00066EB8EEE0E948F11898190E0982F8827EC
:1025F0002A81822B9093131C8093121C22E0AE013F
:102600004F5F5F4F68EB8EEE0E948F11898190E0E3
:10261000982F88272A81822B9093151C8093141C55
:1026200022E0AE014F5F5F4F6AEB8EEE0E948F118A
:10263000898190E0982F88272A81822B9093191CFA
:102640008093181C22E0AE014F5F5F4F6CEB8EEE63
:102650000E948F11898190E0982F88272A81822BF0
:1026600090931B1C80931A1C22E0AE014F5F5F4FBA
:102670006EEB8EEE0E948F11898190E0982F882753
:102680002A81822B90931D1C80931C1C0F900F900D
:10269000DF91CF9108952F923F924F925F926F9268
:1026A0007F928F929F92AF92BF92CF92DF92EF92E2
:1026B000FF920F931F93CF93DF93CDB7DEB76A9747
:1026C0000FB6F894DEBF0FBECDBF182F488F298FED
:1026D00019821A821B828091301C811107C06A8F77
:1026E0000E94791281E08093301C6A8D662309F480
:1026F0006CC04EE264EF8EEE0E94781169E07AE1E0
:1027000080E090E00E949C5F22E0AE014F5F5F4F4F
:1027100066EF8EEE0E948F112981822F90E0A0E05B
:10272000B0E02227382F492F5A2F8A81282B8091F9
:10273000221C9091231C281B390B41095109A0919F
:10274000201CB091211C0E94DF8B6B017C018FE06B
:10275000F594E794D794C7948A95D1F760911A1CA1
:1027600070911B1C882777FD8095982F2BE0660FB2
:10277000771F881F991F2A95D1F720911C1C309133
:102780001D1C442737FD4095542F2C0D3D1D4E1D1B
:102790005F1D0E944C8CC20ED31ED092171CC0929B
:1027A000161C88E0C80ED11C34E0D594C7943A9525
:1027B000E1F7EE24D7FCE094FE2CC092241CD092CA
:1027C000251CE092261CF092271C012F0295000F79
:1027D000000F007C0C5CA12FB0E0BD8BAC8BA3E0A4
:1027E000B0E0012E02C0AA0FBB1F0A94E2F725E356
:1027F00035E00E94D88BDC01CB010296A11DB11DF2
:102800008C879D87AE87BF8780E593ECA0E0B0E022
:1028100004C0B595A795979587951A95D2F7888B9B
:10282000998BAA8BBB8B10E0188619861A861B869B
:10283000A8E02A2E312CAC89BD892A1A3B0A988D32
:10284000191709F436C1402F64EF8EEE0E947811FB
:102850006C857D858E859F850E949C5F23E0AE01FF
:102860004F5F5F4F66EF8EEE0E948F11E091161C56
:10287000F091171CE05AFF409F01DF010E94C18BBD
:102880006B017C0180910E1C90910F1C9F8B8E8B95
:10289000A0900C1CB0900D1C2091101C3091111CAC
:1028A0000E94C18B2B013C013DE0759467945794C5
:1028B00047943A95D1F7A091121CB091131CA7012F
:1028C00096016CE055954795379527956A95D1F710
:1028D0000E94EA8BBB2797FDB095AB2F480E591E7F
:1028E0006A1E7B1E92E0490E511C611C711CB2E0F5
:1028F0007594679457944794BA95D1F7A0E85A0E07
:10290000611C711CA0911E1CB0911F1CA30192019F
:102910000E94DF8BDC01CB012FE0B695A795979540
:1029200087952A95D1F78C839D83AE83BF832981B8
:102930008A8190E0A0E0B0E04424582E692E7A2EDF
:10294000622A8B81482A022C04C07594679457949C
:1029500047940A94D2F74501AA2497FCA094BA2C74
:1029600042E0880C991CAA1CBB1C4A95D1F7A09187
:10297000141CB091151CA70196010E94EA8B6B01F3
:102980007C0157E1F594E794D794C7945A95D1F711
:102990002E893F89DF010E94C18BEBE095958795D9
:1029A00077956795EA95D1F7C60ED71EE81EF91EF2
:1029B0008C0C9D1CAE1CBF1C0C8804C0880C991C80
:1029C000AA1CBB1C0A94D2F792E0890E911CA11C90
:1029D000B11CF2E0B594A79497948794FA95D1F737
:1029E000481859086A087B08A30192016889798907
:1029F0008A899B890E94F28B97FD0DC0660F771F15
:102A0000881F991F2C813D814E815F810E942A8CF5
:102A100049015A010CC02C813D814E815F810E9489
:102A20002A8C49015A01880C991CAA1CBB1C9927A5
:102A3000B7FC9A958B2D7A2D692D9B01AC010E94D4
:102A4000F28B9B01AC01AEEDBBE00E94DF8B6C0111
:102A5000FF24D7FCF094EF2CA3E4B3EEA50194017E
:102A60000E94ED8BBB2797FDB095AB2FC80ED91EEA
:102A7000EA1EFB1EAFECCA0EAEE0DA1EE11CF11C32
:102A8000A4E0F594E794D794C794AA95D1F7C80C1D
:102A9000D91CEA1CFB1C88859985AA85BB858C0DF1
:102AA0009D1DAE1DBF1D88879987AA87BB871F5FA5
:102AB000C6CE112391F0212F30E040E050E0688530
:102AC00079858A859B850E942A8C2093281C3093C7
:102AD000291C40932A1C50932B1CA98DAA2389F1F1
:102AE0006091281C7091291C80912A1C90912B1CAC
:102AF000611571058105910521F10E941F8920E86A
:102B000036EE45EC57E40E94808821E03EED42E439
:102B10005EE30E94648B9B01AC0160E070E080E8A2
:102B20009FE30E94B5872BE43AE34DEB57E30E9405
:102B3000808860932C1C70932D1C80932E1C909386
:102B40002F1C6A960FB6F894DEBF0FBECDBFDF9183
:102B5000CF911F910F91FF90EF90DF90CF90BF909A
:102B6000AF909F908F907F906F905F904F903F902D
:102B70002F9008950F931F93CF93DF9300D000D031
:102B800000D0CDB7DEB78E010F5F1F4F86E0F80192
:102B900011928A95E9F780911E1B811113C040E0C4
:102BA00061E386EA0E9478114AE06CE286EA0E94BC
:102BB000781181E080931E1B6CE77EE380E090E05B
:102BC0000E949C5F48E06DE286EA0E9478116CE703
:102BD0007EE380E090E00E949C5F26E0A80162E333
:102BE00086EA0E948F1147E06DE286EA0E94781122
:102BF0008A8190E0982F88272981822B9093191B36
:102C00008093181B2C8130E0322F22274B81242BFC
:102C100030931B1B20931A1B4E8150E0542F4427E6
:102C20006D81462B50931D1B40931C1B5F934F934C
:102C30003F932F939F938F938BEF93E09F938F936B
:102C40000E94B0920FB6F894DEBF0FBECDBF26969D
:102C50000FB6F894DEBF0FBECDBFDF91CF911F91AD
:102C60000F910895CF92DF92EF92FF920F931F93EF
:102C7000CF93DF93CDB7DEB72A970FB6F894DEBFB8
:102C80000FBECDBF8E010F5F1F4F86E0F80111927E
:102C90008A95E9F741E062E08CE30E94781148E50B
:102CA00060E08CE30E94781162E174E380E090E0E0
:102CB0000E949C5F26E0A80163E08CE30E948F11D4
:102CC00043E062E08CE30E947811098110E0102F4C
:102CD00000278A81082B1093F91A0093F81AEB80C9
:102CE000F12CFE2CEE248C81E82AF092FB1AE09263
:102CF000FA1ACD80D12CDC2CCC248E81C82AD0921B
:102D0000FD1AC092FC1AB801882777FD8095982F8C
:102D10000E941F899B01AC01B701882777FD809530
:102D2000982F2F83388749875A870E941F892F81C0
:102D3000388549855A850E94298820EE3EE245E67D
:102D400052E40E94018B20E030E044E353E40E940F
:102D5000B6879F938F937F936F93DF92CF92FF926B
:102D6000EF921F930F9389E094E09F938F930E94BB
:102D7000B0920FB6F894DEBF0FBECDBF2A960FB645
:102D8000F894DEBF0FBECDBFDF91CF911F910F91A1
:102D9000FF90EF90DF90CF900895CF93DF93EC01F9
:102DA000888199810097F9F08238904121F0198249
:102DB000188283E063C085ED99E00E94EE56892B6E
:102DC000E1F08091C5099091C60993FD18C08091EA
:102DD000C5099091C60994FD43C08091C5099091A1
:102DE000C60995FD44C060E870E085ED99E00E9459
:102DF000C75682E890E19983888381E03FC0809143
:102E00003D2082FFE4CF21E048E061E083E00E94C2
:102E10004B1380912F1C8F9380912E1C8F93809148
:102E20002D1C8F9380912C1C8F9380912B1C8F9342
:102E300080912A1C8F938091291C8F938091281C4C
:102E40008F9385EC9EE09F938F930E94C2928DB7E3
:102E50009EB70A960FB6F8949EBF0FBE8DBFB7CF30
:102E600080913D2083FFB9CF0E94BA15B6CF8091E3
:102E70003D2084FFB8CF0E943216B5CFDF91CF91AD
:102E80000895CF93C82F8CEE0E9420608C2F0E9453
:102E90002A6065E375E080E090E00E949C5F8DEE23
:102EA0000E9420600E943B60C82F0E9445602C2F2A
:102EB00030E0322F2227A901482BCA01CF91089573
:102EC000CF93DF93C82F8CEE0E9420608C2F0E943E
:102ED0002A6062E174E380E090E00E949C5F8CEEE7
:102EE0000E94206080E00E942A6065E375E080E037
:102EF00090E00E949C5F8DEE0E9420600E943B60EB
:102F0000C82F0E943B60D82F0E9445604D2F50E093
:102F100060E070E0762F652F542F44276C2B482BF0
:102F2000CB01BA01DF91CF9108952F923F924F923A
:102F30005F926F927F928F929F92AF92BF92CF9249
:102F4000DF92EF92FF920F931F93CF93DF93CDB752
:102F5000DEB7CD54D1090FB6F894DEBF0FBECDBF9A
:102F60008091000290910102892BD1F1109201020F
:102F7000109200028CEE0E9420608EE10E942A6076
:102F80006BE17EE480E090E00E949C5F82EA0E9418
:102F900041179093D2098093D10984EA0E94411786
:102FA0009093D0098093CF0986EA0E9441179093AD
:102FB000CE098093CD0988EA0E9441179093CC09ED
:102FC0008093CB098AEA0E9441179093CA098093A3
:102FD000C9098CEA0E9441179093C8098093C709D8
:102FE00088E40E9460176FAB78AF89AF9AAF88E52D
:102FF0000E9460174B015C018091C9099091CA0938
:1030000020E030E040E050E0BA0126962FAF26974E
:1030100027963FAF279728964FAF289729965FAFFF
:1030200029972A966FAF2A972B967FAF2B979C01F3
:1030300040E050E060E070E080E090E008E00E9456
:10304000D38D0E947F8D3901B42FA52FF62FE72F46
:103050008C019401A50160E070E080E090E05301F4
:10306000CB2EDA2EEF2EFE2E0E940A8E29833A8373
:103070002A011B014C01B101C401315041095F4FCC
:103080006F4F7F4F8F4F9F4FA1E0B0E02596BFAFAE
:10309000AEAF259721153F4F4F4F51406105710548
:1030A0008105910509F020F425961FAE1EAE2597E7
:1030B00025966EAC7FAC25978091C7099091C80981
:1030C0005C01C12CD12CE12CF12C00E010E0298115
:1030D0003A81A201B101C4010E94A28CD22EE32E3A
:1030E000F42E052F162FB72FF82FE92FA0E00E94FE
:1030F000318E84F42150310940485F4F6F4F7F4F2C
:103100008F4F9F4FD22EE32EF42E052F162FB72F61
:10311000F82FE92F2D2D3E2D4F2D502F612F7B2F76
:103120008F2F9E2F07E10E94EC8D2B8F3C8F4D8FB0
:103130005E8F6F8F78A389A39AA32053384F4F4F88
:103140005F4F6F4F7F4F8F4F9F4F2B8B3C8B4D8B24
:103150005E8B6F8B788F898F9A8F2056304F4F4FB1
:103160005F4F6F4F7F4F8F4F9F4F243D304341053F
:103170005105610571058105910541F038F02596ED
:103180006EAC7FAC2597FFEF6F1A7F0A8091CF0955
:103190009091D0099C0140E050E060E070E080E058
:1031A00090E000E10E94D38D2B833C834D835E83AE
:1031B0006A8779878F8398874091CB095091CC0992
:1031C000A980BA806201710184019A0140E050E057
:1031D00060E070E080E090E00E94A28CD22EE32EAE
:1031E000F42E052F162FB72FF82FE92FA0E00E94FD
:1031F000318E5CF4AFE70E94138ED22EE32EF42EB4
:10320000052F162FB72FF82FE92F2D2D3E2D4F2DDF
:10321000502F612F7B2F8F2F9E2F07E00E94EC8D68
:1032200059016A017B018C012B813C814D815E81BA
:103230006A8579858F8198850E940A8E2B833C83CD
:103240004D835E836F8378878F87988B2E5F3F4F88
:10325000434051096E4F7F4F8F4F9F4F22303105B2
:10326000494F5F4F644071058105910521F018F0C9
:103270001FEF611A710A8091D1099091D209BC01A6
:1032800080E090E020E030E840E050E00E94FB8CDD
:1032900029873A874B875C876A8B798B8D879E87D6
:1032A0004091CD095091CE09A980BA806201710187
:1032B00084019A0140E050E060E070E080E090E03E
:1032C0000E94A28CD22EE32EF42E052F162FB72F9C
:1032D000F82FE92FA0E00E94318E84F421503F4F57
:1032E0004F4F5F4F6F4F7F4F8F4F9F4FD22EE32E29
:1032F000F42E052F162FB72FF82FE92F2D2D3E2D49
:103300004F2D502F612F7B2F8F2F9E2F08E00E9473
:10331000EC8D59016A017B018C0129853A854B8529
:103320005C856A8979898D859E850E940A8E2987A8
:103330003A874B875C876D877E87898B9A8B2F5F57
:103340003F4F4140510961097109810991092130BB
:1033500030484C4F5F47614071058105910521F070
:1033600018F0BFEF6B1A7B0A2B893C894D895E8967
:103370006F89788D898D9A8D2F3C37404105510595
:10338000610571058105910511F00CF0A5C1A980B9
:10339000BA806201710184019501A201B101C401E9
:1033A0000E94A28CA12CB12CC12C10E8D12EE12CB2
:1033B000F12C00E010E00E94658C2BAF3CAF4DAFCC
:1033C0005EAF6FAF21967FAF219722968FAF229786
:1033D00023969FAF2397AB8CBC8CCD8CDE8CEF8C6F
:1033E000F8A009A11AA19501A601B701C8010E9480
:1033F000A28C59016A017B01E82F192F02E00E947B
:10340000D38D0E2F0E940A8E69017A01162F272E66
:10341000F82FE92F322E8D2C942EAF2CB62E072F9D
:10342000582EB92FA0E00E94318E5CF4A1E00E94DA
:10343000138E322E832E942EA52EB62E072F582EA5
:10344000B92F232D382D492D5A2D6B2D702F852DF9
:103450009B2F01E00E94EC8D2E962FAF2E972D967C
:103460003FAF2D9749A75AA76BA77CA78DA79EA70B
:10347000522E432E4BA35CA36DA37EA38FA398A7CC
:10348000B22D9601A701612F722D8F2F9E2FA0E0E4
:103490000E94318E4CF4A3E00E94138E69017A01E0
:1034A000162FB72FF82FE92F9601A701612F7B2F39
:1034B0008F2F9E2F02E00E94EC8D2FA738AB49ABD7
:1034C0005AAB6BAB7CAB8DAB9EAB19014A01B62FEF
:1034D000A72F24968FAF2497F92F2B893C894D89EC
:1034E0005E896F89788D898D9A8D24323A4F4F4F3E
:1034F0005F4F6F4F7F4F8F4F9F4F0CF08CC02B8DC6
:103500003C8D4D8D5E8D6F8D78A189A19AA124553A
:10351000324F4F4F5F4F6F4F7F4F8F4F9F4F59012C
:103520006A017B018C010E94A28C19014A01B62F0D
:10353000A72FFC0103E00E94D38D51016401EB2E03
:10354000FA2E8F010E941F8E59016A017B018C01A6
:103550002E962FAD2E972D963FAD2D9749A55AA5A6
:103560006BA57CA58DA59EA50E940A8E522E432E8A
:103570004BA35CA36DA37EA38FA398A79101A40185
:103580006B2F7A2FCF0102E00E94D38D510164018D
:10359000EB2EFA2E8F010E941F8E02E00E94D38D27
:1035A0000E2F0E941F8EF22E032F142FD52EE62EE3
:1035B000B72FF82FE92FA0E00E94318E5CF4A1E034
:1035C0000E94138EF22E032F142FD52EE62EB72F26
:1035D000F82FE92F2F2D302F412F5D2D6E2D7B2FB2
:1035E0008F2F9E2F01E00E94EC8D59016A017B0113
:1035F0008C012FA538A949A95AA96BA97CA98DA925
:103600009EA90E940A8E19014A01B62FA72F24965F
:103610008FAF2497F92F2B813C814D815E816F8183
:1036200078858F859889A52CB42CCBA0DCA0EDA043
:10363000FEA00FA118A50E941F8E2B833C834D83F3
:103640005E836F8378878F87988B29853A854B8532
:103650005C856D857E8589899A8951016401EB2E8F
:10366000FA2E24960FAD24971F2F0E941F8E2987B4
:103670003A874B875C876D877E87898B9A8B2B89EE
:103680003C894D895E896F89788D898D9A8DABAC27
:10369000BCACCDACDEACEFAC2196FFAC2197229652
:1036A0000FAD229723961FAD23970E941F8E2056A1
:1036B000304F4F4F5F4F6F4F7F4F8F4F9F4F243D86
:1036C000304341055105610571058105910521F0E2
:1036D00018F02FEF621A720A6FA978AD89AD9AAD12
:1036E000AB01BC0180E090E0DC0124964FAF249751
:1036F00025965FAF259726966FAF269727967FAFC3
:10370000279728968FAF289729969FAF29972A96B3
:10371000AFAF2A972B96BFAF2B97A984BA84CB84DF
:10372000DC84ED84FE8409891A899A01AB0160E08A
:1037300070E080E090E00E94A28CF22E032F142F04
:10374000D52EE62EB72FF82FE92FA0E00E94318E5C
:1037500084F421503109404E5F4F6F4F7F4F8F4FA0
:103760009F4FF22E032F142FD52EE62EB72FF82FB2
:10377000E92F2F2D302F412F5D2D6E2D7B2F8F2F79
:103780009E2F05E10E94EC8DAB80BC80CD80DE8059
:10379000EF80F8840F8518890E941F8EF22E032F68
:1037A000142FD52EE62EB72FF82FE92FA0E00E9478
:1037B000318E84F4215030484F4F5F4F6F4F7F4F11
:1037C0008F4F9F4FF22E032F142FD52EE62EB72F9B
:1037D000F82FE92F2F2D302F412F5D2D6E2D7B2FB0
:1037E0008F2F9E2F0FE00E94EC8D69017A018B01D3
:1037F0008A83998329011A014B015C01285E3340B9
:10380000410951096109710981099109283D304D2A
:1038100041405105610571058105910521F018F0C0
:10382000BFEF6B1A7B0A0E942260672859F096014D
:10383000A701B8018A8199810E947F8D29011A010F
:103840004B015C019201A101B401C5010E941989DB
:1038500020E030E048EC52E40E948088C35BDF4FF8
:103860000FB6F894DEBF0FBECDBFDF91CF911F9191
:103870000F91FF90EF90DF90CF90BF90AF909F900F
:103880008F907F906F905F904F903F902F90089512
:103890004F925F926F927F928F929F92AF92BF9260
:1038A000CF92DF92EF92FF922B013C0169017A01E6
:1038B00023EC35EF4CE851E4C701B6010E94018BBF
:1038C0004B015C0128EB3EE143E753E4C701B6013D
:1038D0000E94B6879B01AC01C501B4010E9480889B
:1038E0000E94ED884B015C0120E030E048EC52E49E
:1038F000C301B2010E94808821E835E943EC50E41D
:103900000E94018BA50194010E94018B4B015C0177
:1039100023E333E948E853E4C701B6010E94B687C0
:103920009B01AC01C501B4010E94808823E333EB05
:1039300048E553E40E94018BFF90EF90DF90CF9019
:10394000BF90AF909F908F907F906F905F904F90BF
:1039500008954F925F926F927F928F929F92AF9253
:10396000BF92CF92DF92EF92FF9269017A010E949B
:10397000838A20E030E040E050E40E94B58722E9ED
:103980003CE54EED5EE30E9480884B015C0123EC38
:1039900035EF4CE851E4C701B6010E94018B2B01C1
:1039A0003C0128EB3EE143E753E4C701B6010E9426
:1039B000B6879B01AC01C301B2010E9480889B01C4
:1039C000AC01C501B4010E94B6876B017C0128EBF4
:1039D0003EE143E753E40E94018B4B015C01A701E8
:1039E000960163EC75EF8CE891E40E94B5879B012A
:1039F000AC01C501B4010E948088FF90EF90DF9078
:103A0000CF90BF90AF909F908F907F906F905F907E
:103A10004F9008954F925F926F927F928F929F92F4
:103A2000AF92BF92CF92DF92EF92FF922B013C01B7
:103A300069017A0123EC35EF4CE851E4C701B60186
:103A40000E94018B4B015C0128EB3EE143E753E40C
:103A5000C701B6010E94B6879B01AC01C501B40144
:103A60000E9480880E94ED884B015C0120E030E0DC
:103A700048EC52E4C301B2010E948088A501940180
:103A80000E94018B20E030E040E251E40E94B587C3
:103A900024EE38E34EE05FE30E94018B9B01AC0112
:103AA000C701B6010E94B687FF90EF90DF90CF90DC
:103AB000BF90AF909F908F907F906F905F904F904E
:103AC000089580E80E94206081110DC08EEF0E9451
:103AD0002A60811108C06BE17EE480E090E00E94E2
:103AE0009C5F0C9422600E94226080914F249091F0
:103AF0005024A0915124B09152240196A11DB11DD2
:103B000080934F2490935024A0935124B093522437
:103B10000895FC01DC0182E020E041E39D9129272A
:103B200098E0322F330F27FF03C0232F242701C033
:103B3000232F9150B1F7815089F781E090E03281D5
:103B4000231711F080E090E00895DF92EF92FF924A
:103B50000F931F93CF93DF930E94611D80E80E9413
:103B6000206081116DC08AEF0E942A60811168C0B7
:103B70008FE00E942A60811163C065E375E080E0F8
:103B800090E00E949C5F81E80E942060811158C0F3
:103B90000E943B60C82F0E943B600E943B60D82F70
:103BA0000E943B600E943B60182F0E943B600E9475
:103BB0004560082F80E80E942060811141C08CEF91
:103BC0000E942A6081113CC089EC0E942A60811108
:103BD00037C065E375E080E090E00E949C5F81E87B
:103BE0000E9420600E943B60E82E0E943B60D82E1D
:103BF0000E943B600E943B60F82E0E9445601F922D
:103C0000DF921F92EF921F920F931F921F931F92AA
:103C1000DF931F92CF931F928F931F92FF928EE19B
:103C200094E09F938F930E94B0920E9422608DB780
:103C30009EB742960FB6F8949EBF0FBE8DBF17C0B9
:103C40000E94226080914F2490915024A091512491
:103C5000B09152240196A11DB11D80934F249093E1
:103C60005024A0935124B09352240E94611D20E05F
:103C700030E040E050E060E070E080E090E0DF9114
:103C8000CF911F910F91FF90EF90DF900895EF92E9
:103C9000FF920F931F93CF93DF9300D01F92CDB766
:103CA000DEB78C0180E80E942060811154C00115AC
:103CB000110551F085EE0E942A6081114CC061E02F
:103CC00077E980E090E009C083EE0E942A608111CC
:103CD00042C069E97AEB81E090E00E949C5F81E854
:103CE0000E942060811137C00E943B60F82E8983BA
:103CF0000E943B60E82E8A830E9445608B830E946D
:103D00002260CE0101960E94891D892B21F16E2D22
:103D100070E07F296C7F80E090E0012B69F00E94C9
:103D20001D8920E030E04AEF5AE30E94018B20E039
:103D300030E040EC50E40CC00E941D8922E538EBD5
:103D40004FE25BE30E94018B26E636E64BE352E44A
:103D50000E94B5871BC00E94226080914F249091E1
:103D60005024A0915124B09152240196A11DB11D5F
:103D700080934F2490935024A0935124B0935224C5
:103D80000E94611D60EF7FEF89E794E40F900F9030
:103D90000F90DF91CF911F910F91FF90EF900895B9
:103DA0000F931F93CF93DF93729A8091580283FFF2
:103DB00008C08EE40E94BE5F811167C0C0E5D0E0FC
:103DC0000AC0C0E5D0E087EE93E00E944509219744
:103DD0002097C9F7EECF87EE93E00E94450921971F
:103DE0002097C9F78FE40E94BE5F0E943B60082FB6
:103DF0000F730E943B60182F0E943B60D82F0E94D7
:103E00004560C82F0E9422608091580283FF7298FB
:103E1000602F70E0762F6627610F711D80E090E0C3
:103E20000E941D8920E134E048EC5BE30E94018B95
:103E30006093311C7093321C8093331C9093341C1C
:103E40006D2F70E0762F66276C0F711D7695679544
:103E50007695679580E090E00E941D8924EA3CEF0A
:103E600044E25CE30E94018B20E030E040E252E457
:103E70000E94B58760930E2970930F2980931029B3
:103E80009093112980E090E002C081E090E0DF9102
:103E9000CF911F910F9108957298729A8EE40E94AB
:103EA000BE5F80EA0E942A6080E00E942A6080E073
:103EB0000E942A608FE40E94BE5F0E943B608EE4F5
:103EC0000E94BE5F80E80E942A6080E00E942A6013
:103ED00080E00E942A600E94226080E090E00895C5
:103EE00089E59EE09F938F930E94C2928091730216
:103EF0000F900F90882361F01F928F9386E59EE0CC
:103F00009F938F930E94C2920F900F900F900F90EB
:103F1000089581E39EE09F938F930E94C29289E06F
:103F20009EE09F938F930E94C29282EE9DE09F93AA
:103F30008F930E94C29287EA9DE09F938F930E9485
:103F4000C29285E79DE09F938F930E94C29289E37E
:103F50009DE09F938F930E94C29283E19DE09F9387
:103F60008F930E94C2928DED9CE09F938F930E944D
:103F7000C29280913D2090913E20827091702DB729
:103F80003EB7205F3F4F0FB6F8943EBF0FBE2DBF28
:103F9000892B41F08DEA9CE09F938F930E94C292FF
:103FA0000F900F9081E89CE09F938F930E94C292A4
:103FB00085E49CE09F938F930E94C2928CE19CE0E9
:103FC0009F938F930E94C29280EF9BE09F938F9369
:103FD0000E94C29281EC9BE09F938F930E94C292B9
:103FE0008FE89BE09F938F930E94C2928EE59BE0A7
:103FF0009F938F930E94C29284E29BE09F938F9342
:104000000E94C2928EEE9AE09F938F930E94C2927A
:104010008EEB9AE09F938F930E94C29282E99AE07E
:104020009F938F930E94C29283E69AE09F938F930F
:104030000E94C2928AE29AE09F938F930E94C2925A
:1040400081EF99E09F938F930E94C2928AEB99E04F
:104050009F938F930E94C29289E899E09F938F93D8
:104060000E94C2928DB79EB780960FB6F8949EBFFD
:104070000FBE8DBF8AE599E09F938F930E94C292F5
:104080008BE299E09F938F930E94C29284E099E023
:104090009F938F930E94C2928EEC98E09F938F9390
:1040A0000E94C29288E998E09F938F930E94C292E7
:1040B00082E698E09F938F930E94C29289E398E0F2
:1040C0009F938F930E94C29281E098E09F938F9379
:1040D0000E94C29286ED97E09F938F930E94C292B6
:1040E0002DB73EB72E5E3F4F0FB6F8943EBF0FBEC2
:1040F0002DBF08958DE494E00C94E6924F925F9268
:104100006F927F928F929F92AF92BF92CF92DF92E7
:10411000EF92FF92CF93DF93CDB7DEB728970FB61C
:10412000F894DEBF0FBECDBF80914324909144240C
:10413000A0914524B091462489839A83AB83BC83A4
:10414000409043245090442460904524709046242D
:104150008091432490914424A0914524B091462419
:104160008D839E83AF83B8876091432470914424EC
:1041700080914524909146242CE3822E912CA12CF1
:10418000B12CA50194010E942A8C7F936F9330E19A
:10419000C32E3EE0D32EE12CF12C6D817E818F81E8
:1041A0009885A70196010E942A8CA50194010E947E
:1041B0002A8C3F932F9340E8842E41E5942EAA2425
:1041C000A394B12CC301B201A50194010E942A8CD1
:1041D000A70196010E942A8C3F932F9369817A81CF
:1041E0008B819C81A50194010E942A8C3F932F937F
:1041F00080EB97E09F938F930E94C2920FB6F89442
:10420000DEBF0FBECDBF28960FB6F894DEBF0FBE3F
:10421000CDBFDF91CF91FF90EF90DF90CF90BF9017
:10422000AF909F908F907F906F905F904F90089588
:10423000E3EDF1E3808191818234924479F0E35D92
:10424000F143FF93EF9382E997E09F938F930E944E
:10425000C2920F900F900F900F9008953A96E53FFD
:1042600081E4F80738F30895CF93DF93EC018C9A3B
:104270000E94900A9F938F937F936F9386E897E0B5
:104280009F938F930E94C2920F900F900F900F9068
:104290000F900F90209719F00E94AB0B08C084E894
:1042A00097E09F938F930E94C2920F900F9081E0AE
:1042B0000E94410A209178023091790240917A025D
:1042C00050917B020E94018B9F938F937F936F93FA
:1042D00088E797E09F938F930E94C2920F900F9070
:1042E0000F900F900F900F90209719F00E94AB0B3A
:1042F00008C086E797E09F938F930E94C2920F9029
:104300000F9082E00E94410A209174023091750260
:1043100040917602509177020E94018B9F938F9378
:104320007F936F938AE697E09F938F930E94C29248
:104330000F900F900F900F900F900F90209719F003
:104340000E94AB0B08C088E697E09F938F930E9472
:10435000C2920F900F9083E00E94410A9F938F9327
:104360007F936F9389E597E09F938F930E94C2920A
:104370008C980F900F900F900F900F900F902097A8
:1043800019F00E94AB0B08C087E597E09F938F93CD
:104390000E94C2920F900F9080913D2087FF83C0B2
:1043A00021E042E161E080ED0E9482619F938F9362
:1043B0007F936F938AE497E09F938F930E94C292BA
:1043C0000F900F900F900F900F900F90209719F073
:1043D0000E94AB0B08C088E497E09F938F930E94E4
:1043E000C2920F900F9021E042E162E080ED0E94C6
:1043F00082619F938F937F936F938BE397E09F935B
:104400008F930E94C2920F900F900F900F900F9079
:104410000F90209719F00E94AB0B08C089E397E03A
:104420009F938F930E94C2920F900F9021E042E1E0
:1044300063E080ED0E9482619F938F937F936F93DF
:104440008CE297E09F938F930E94C2920F900F90FF
:104450000F900F900F900F90CD2B19F00E94AB0B87
:1044600008C08AE297E09F938F930E94C2920F90B8
:104470000F9021E042E164E080ED0E9482619F9311
:104480008F937F936F938DE197E09F938F930E941B
:10449000C2920F900F900F900F900F900F90DF919E
:1044A000CF910C94AB0BCD2BD1F3DF91CF9108952D
:1044B0000F931F93CF93DF93882389F049E050E057
:1044C0006FEF70E082E099E20E94049249E050E0D0
:1044D0006AE070E082E099E20E94349413C0C2E086
:1044E000D9E208E117E089911F928F931F930F93F0
:1044F0000E94C2920F900F900F900F9089E2CA30E5
:10450000D80789F7DF91CF911F910F910C94AB0BD6
:10451000CF92DF92EF92FF92CF93DF936B017C01FA
:1045200060FF11C08AE894E09F938F938EE69EE02F
:104530009F938F930E94C2920F900F900F900F90B5
:1045400081E090E002C080E090E0C1FE09C0EC0193
:10455000219643E259E06FE874E00E940410CE0116
:10456000C2FE09C0EC01219643E259E067E974E01C
:104570000E940410CE01C3FE09C0EC01219643E263
:1045800059E06FE974E00E940410CE01C4FE09C036
:10459000EC01219643E259E063EA74E00E940410C2
:1045A000CE01C5FE09C0EC01219643E259E066EA5E
:1045B00074E00E940410CE01C6FE09C0EC012196F1
:1045C00043E259E06AEA74E00E940410CE01C7FE9B
:1045D00009C0EC01219643E259E060EB74E00E94CF
:1045E0000410CE01D0FE09C0EC01219643E259E04F
:1045F00068EB74E00E940410CE01D1FE09C0EC010A
:10460000219643E259E060EC74E00E940410CE0170
:10461000D2FE09C0EC01219643E259E064EC74E05B
:104620000E940410CE0120913D2030913E20247044
:104630003270232B59F0D3FE09C0EC01219643E2DE
:1046400059E06AEC74E00E940410CE0120913D20F4
:1046500023FF0BC0D4FE09C0EC01219643E259E0D0
:104660006FEC74E00E940410CE0120913D2024FFE5
:104670000BC0D5FE09C0EC01219643E259E065ED7F
:1046800074E00E940410CE01D6FE09C0EC01219610
:1046900043E259E06DED74E00E940410CE01B701D1
:1046A000A60144275078452B462B472B61F043E267
:1046B00059E068EE74E0DF91CF91FF90EF90DF90CA
:1046C000CF900C940410CD28CE28CF2841F483E15C
:1046D00097E09F938F930E94C2920F900F90DF916B
:1046E000CF91FF90EF90DF90CF9008950F931F939D
:1046F000CF93DF938C01C0E0D0E00115110509F4E0
:104700008AC06EE077E0C8010E94E391892B09F42A
:10471000C16066E077E0C8010E94E391892B09F44B
:10472000C2606EEF76E0C8010E94E391892B09F424
:10473000C4606AEF76E0C8010E94E391892B09F416
:10474000C86067EF76E0C8010E94E391892B09F405
:10475000C06163EF76E0C8010E94E391892B09F400
:10476000C0626DEE76E0C8010E94E391892B09F4E6
:10477000C06465EE76E0C8010E94E391892B09F4DC
:10478000C0686DED76E0C8010E94E391892B09F4C1
:10479000D16069ED76E0C8010E94E391892B09F4AC
:1047A000D26063ED76E0C8010E94E391892B09F4A1
:1047B000D4606EEC76E0C8010E94E391892B09F485
:1047C000D86068EC76E0C8010E94E391892B09F477
:1047D000D06160EC76E0C8010E94E391892B09F476
:1047E000D06265EB76E0C8010E94E391892B09F461
:1047F000D06464EA76E0C8010E94E391892B09F451
:10480000D068609171027091720280E090E00E9425
:10481000F7918C0172CFCE01DF91CF911F910F9153
:104820000895AF92BF92CF92DF92EF92FF920F93D3
:104830001F93CF93DF93F22E032F142FE52ED62E46
:10484000A72EB82EC92E217030E040E050E060E085
:1048500070E080E090E0A0E00E94318E89F0E9EF06
:10486000F4E0FF93EF93EEE6FEE0FF93EF930E94F8
:10487000C2920F900F900F900F90E1E0F0E002C015
:10488000E0E0F0E080913D2080FF17C02F2D2470E4
:1048900030E040E050E060E070E080E090E0A0E0D8
:1048A0000E94318E51F0EF01219643E259E06DEF05
:1048B00074E0CF010E940410FE012F2D227030E021
:1048C00040E050E060E070E080E090E0A0E00E9416
:1048D000318E51F0EF01219643E259E061E075E03D
:1048E000CF010E940410FE012F2D287030E040E01F
:1048F00050E060E070E080E090E0A0E00E94318E47
:1049000051F0EF01219643E259E069E175E0CF01F2
:104910000E940410FE012F2D207130E040E050E095
:1049200060E070E080E090E0A0E00E94318E51F005
:10493000EF01219643E259E064E075E0CF010E9467
:104940000410FE012F2D207230E040E050E060E0C6
:1049500070E080E090E0A0E00E94318E51F0EF0125
:10496000219643E259E067E075E0CF010E94041010
:10497000FE012F2D207430E040E050E060E070E058
:1049800080E090E0A0E00E94318E51F0EF0121968E
:1049900043E259E06DE075E0CF010E940410FE0192
:1049A0002F2D207830E040E050E060E070E080E0C3
:1049B00090E0A0E00E94318E51F0EF01219643E299
:1049C00059E063E175E0CF010E940410FE0120E090
:1049D000302F317040E050E060E070E080E090E027
:1049E000A0E00E94318E51F0EF01219643E259E0A0
:1049F00066E175E0CF010E940410FE0120E0302F37
:104A0000327040E050E060E070E080E090E0A0E0D4
:104A10000E94318E51F0EF01219643E259E06BE1A3
:104A200075E0CF010E940410FE0120E0302F3470A9
:104A300040E050E060E070E080E090E0A0E00E94A4
:104A4000318E51F0EF01219643E259E062E275E0C8
:104A5000CF010E940410FE0120E0302F387040E0AA
:104A600050E060E070E080E090E0A0E00E94318ED5
:104A700051F0EF01219643E259E065E275E0CF0184
:104A80000E940410FE0120E0302F307140E050E021
:104A900060E070E080E090E0A0E00E94318E51F094
:104AA000EF01219643E259E06AE275E0CF010E94EE
:104AB0000410FE0120E0302F307240E050E060E052
:104AC00070E080E090E0A0E00E94318E51F0EF01B4
:104AD000219643E259E061E375E0CF010E940410A2
:104AE000FE0120E030E040E050E06D2D647070E0A9
:104AF00080E090E0A0E00E94318E51F0EF0121961D
:104B000043E259E068E375E0CF010E940410FE0122
:104B100080913D2081FF17C020E0302F307440E0AD
:104B200050E060E070E080E090E0A0E00E94318E14
:104B300051F0EF01219643E259E06CE375E0CF01BB
:104B40000E940410FE0180913D2090913E2090FF34
:104B500017C020E030E040E05E2D507160E070E072
:104B600080E090E0A0E00E94318E51F0EF012196AC
:104B700043E259E06FE375E0CF010E940410FE01AB
:104B800080913D2090913E2090FF17C020E030E0C2
:104B900040E05E2D507260E070E080E090E0A0E0C8
:104BA0000E94318E51F0EF01219643E259E062E418
:104BB00075E0CF010E940410FE0180913D2090918C
:104BC0003E2090FF17C020E030E040E05E2D5074A2
:104BD00060E070E080E090E0A0E00E94318E51F053
:104BE000EF01219643E259E068E475E0CF010E94AD
:104BF0000410FE0120E0302F307840E050E060E00B
:104C000070E080E090E0A0E00E94318E51F0EF0172
:104C1000219643E259E063E575E0CF010E9404105C
:104C2000FE0120E030E0412F417050E060E070E094
:104C300080E090E0A0E00E94318E51F0EF012196DB
:104C400043E259E068E575E0CF010E940410FE01DF
:104C500020E030E0412F427050E060E070E080E002
:104C600090E0A0E00E94318E51F0EF01219643E2E6
:104C700059E06BE575E0CF010E940410FE0120E0D1
:104C800030E0412F447050E060E070E080E090E060
:104C9000A0E00E94318E51F0EF01219643E259E0ED
:104CA0006EE575E0CF010E940410FE0180913D2069
:104CB00087FF17C020E030E0412F487050E060E0EF
:104CC00070E080E090E0A0E00E94318E51F0EF01B2
:104CD000219643E259E061E675E0CF010E9404109D
:104CE000FE0180913D2087FF17C020E030E0412F7A
:104CF000407150E060E070E080E090E0A0E00E9451
:104D0000318E51F0EF01219643E259E065E675E0FE
:104D1000CF010E940410FE0180913D2087FF17C043
:104D200020E030E0412F407250E060E070E080E031
:104D300090E0A0E00E94318E51F0EF01219643E215
:104D400059E069E675E0CF010E940410FE018091F0
:104D50003D2087FF17C020E030E0412F407450E035
:104D600060E070E080E090E0A0E00E94318E51F0C1
:104D7000EF01219643E259E06DE675E0CF010E9414
:104D80000410FE0180913D2082FF17C020E030E03A
:104D9000412F407850E060E070E080E090E0A0E0DB
:104DA0000E94318E51F0EF01219643E259E06DE30C
:104DB00076E0CF010E940410FE0180913D2082FF29
:104DC00017C020E030E040E05E2D517060E070E000
:104DD00080E090E0A0E00E94318E51F0EF0121963A
:104DE00043E259E061E775E0CF010E940410FE0143
:104DF00080913D2090913E2090FF17C020E030E050
:104E000040E05E2D527060E070E080E090E0A0E055
:104E10000E94318E51F0EF01219643E259E064E7A0
:104E200075E0CF010E940410FE0180913D20909119
:104E30003E2090FF17C020E030E040E05E2D54702F
:104E400060E070E080E090E0A0E00E94318E51F0E0
:104E5000EF01219643E259E06CE775E0CF010E9433
:104E60000410FE0180913D2090913E2091FF1EC0D4
:104E700020E030E040E05E2D587060E070E080E0BF
:104E800090E0A0E00E94318E89F043E259E065E8AD
:104E900075E0CF01DF91CF911F910F91FF90EF90BF
:104EA000DF90CF90BF90AF900C9404102F2D302F37
:104EB000412F5E2D6D2D7A2D8B2D9C2DA0E00E9413
:104EC000318E41F48FE996E09F938F930E94C292B6
:104ED0000F900F90DF91CF911F910F91FF90EF9066
:104EE000DF90CF90BF90AF9008958F929F92BF9226
:104EF000DF92EF920F931F93CF93DF93EC014B015F
:104F0000FB0110826AE976E00E94E391892B61F54A
:104F100080913D207DE4D72EE0E8EE2E82FD02C098
:104F200004E001C004E810E0B12C81FF02C060EC95
:104F3000E62E26E04AE250E06BE270E089E290E083
:104F40000E94C35C81E090E00E94390B882311F03D
:104F50005DE5D52E80913D2090913E2090FD16E09C
:104F600091FF07C0186005C0D12CE12C00E010E0D3
:104F7000B12C68E976E0CE010E94E391892B61F4BF
:104F800081E0F4018083609171027091720280E08F
:104F900090E00E94F791EC0166E976E0CE010E9474
:104FA000E391892B61F48FEFF401808360917102AA
:104FB0007091720280E090E00E94F791EC012097DE
:104FC00009F424C162E976E0CE010E94E391892BC5
:104FD00019F4FD2DF160DF2E6EE876E0CE010E941F
:104FE000E391892B19F48D2D8460D82E6BE876E03F
:104FF000CE010E94E391892B19F4ED2DE260DE2EA3
:1050000069E876E0CE010E94E391892B19F4FD2D29
:10501000F860DF2E66E876E0CE010E94E391892BEE
:1050200019F48D2D8061D82E60E876E0CE010E94C3
:10503000E391892B19F4ED2DE062DE2E6AE776E02C
:10504000CE010E94E391892B19F4FD2DF064DF2E2F
:1050500067E776E0CE010E94E391892B19F48D2D4C
:105060008068D82E62E776E0CE010E94E391892B1A
:1050700019F4EE2DE160EE2E6BE676E0CE010E9493
:10508000E391892B19F4FE2DF260EF2E68E676E0AD
:10509000CE010E94E391892B19F48E2D8460E82EB5
:1050A00063E676E0CE010E94E391892B19F4EE2DA0
:1050B000E860EE2E6CE576E0CE010E94E391892B4C
:1050C00019F4FE2DF061EF2E65E576E0CE010E9429
:1050D000E391892B19F48E2D8062E82E61E576E04C
:1050E000CE010E94E391892B19F4EB2DE460BE2ED2
:1050F0006EE476E0CE010E94E391892B19F4FE2D37
:10510000F064EF2E69E476E0CE010E94E391892BF2
:1051100019F48E2D8068E82E66E476E0CE010E94B8
:10512000E391892B09F4016063E476E0CE010E94EB
:10513000E391892B09F4026060E476E0CE010E94DD
:10514000E391892B09F404606CE376E0CE010E94C0
:10515000E391892B09F4086068E376E0CE010E94B0
:10516000E391892B09F4006164E376E0CE010E94AB
:10517000E391892B09F4006260E376E0CE010E949E
:10518000E391892B09F400646EE276E0CE010E947F
:10519000E391892B09F400686BE276E0CE010E946E
:1051A000E391892B09F4116063E276E0CE010E945D
:1051B000E391892B09F412606AE176E0CE010E9446
:1051C000E391892B09F4146061E176E0CE010E943D
:1051D000E391892B09F418606EE076E0CE010E941D
:1051E000E391892B09F4106168E076E0CE010E941A
:1051F000E391892B09F410626DEF75E0CE010E94F6
:10520000E391892B09F0D2CE1064D0CE2D2D3E2D06
:10521000A8016B2D70E080E090E0DF91CF911F91AD
:105220000F91EF90DF90BF909F908F9008955F92C5
:105230006F927F928F929F92AF92BF92CF92DF92A6
:10524000EF92FF920F931F93CF93DF93782EC7E2D5
:10525000DBE100E010E0F7EFEF2EF5E0FF2E8170CC
:10526000582E872D8270682EA2EECA2EA5E0DA2E67
:10527000BAEEAB2EB5E0BB2E88EE882E85E0982ED8
:10528000772051F01F930F93FF92EF920E94C292EA
:105290000F900F900F900F905520A1F089858F935C
:1052A00088858F93BF92AF920E94C2920F900F9009
:1052B0000F900F906620C1F09F928F920E94C29231
:1052C0000F900F90662081F0DF92CF920E94C292E1
:1052D000288139814A815B816C817D818E819F81AA
:1052E0000E9411240F900F900E94AB0B0F5F1F4F75
:1052F0002A960430110521F6DF91CF911F910F916D
:10530000FF90EF90DF90CF90BF90AF909F908F90E5
:105310007F906F905F90089582ED95E09F938F93BB
:105320000E94C2920E947A208EE09BE19F938F930D
:105330008AEC95E09F938F930E94C29260915202F3
:1053400070915302809154029091550228EE33E0FF
:1053500040E050E00E942A8C5F934F933F932F933D
:105360008AEB95E09F938F930E94C29281EB95E028
:105370009F938F930E94C2920E942C1080913D2097
:105380002DB73EB7225F3F4F0FB6F8943EBF0FBE1A
:105390002DBF80FF05C041E061E081E00E94D61191
:1053A0008DEA95E09F938F930E94C29280E00E94C5
:1053B00058220E947E20809157021F928F9384EA88
:1053C00095E09F938F930E94C2928091C1091F9292
:1053D0008F938BE995E09F938F930E94C292809167
:1053E00083028F93809182028F93809181028F93A9
:1053F000809180028F938DE895E09F938F930E9418
:10540000C2921F9280E48F9385E795E09F938F93DC
:105410000E94C292809113291F928F93809112292A
:105420001F928F9382E695E09F938F930E94C29282
:10543000809156021F928F9389E595E09F938F93F9
:105440000E94C2928091580290915902A0915A02F2
:10545000B0915B022DB73EB7225E3F4F0FB6F89476
:105460003EBF0FBE2DBF96FF03C08EE895E002C081
:1054700081E995E09F938F938FE495E09F938F93BD
:105480000E94C29283E00E9417290F900F900F9004
:105490000F901D9B03C08EE895E002C081E995E066
:1054A0009F938F9383E495E09F938F930E94C29282
:1054B00089E395E09F938F930E94C2928091580256
:1054C0000F900F900F900F900F900F9081FF09C0D9
:1054D00083E395E09F938F930E94C2920F900F9069
:1054E00013C080FF03C08EE895E002C081E995E01B
:1054F0009F938F938FE295E09F938F930E94C29228
:105500000F900F900F900F90809158029091590238
:10551000A0915A02B0915B0297FF03C08EE895E01C
:1055200002C081E995E09F938F9386E295E09F9377
:105530008F930E94C2928FE195E09F938F930E9478
:10554000C2926091C5097091C60980E090E00E9406
:1055500088220E94AB0B0F900F900F900F900F902E
:105560000F90779903C08EE895E002C081E995E03D
:105570009F938F9386E195E09F938F930E94C292B1
:105580000E944B090E94F50A9F938F937F936F931C
:1055900088E095E09F938F930E94C2920E94A40A94
:1055A0009F938F937F936F938AEF94E09F938F9352
:1055B0000E94C29281E090E00E9434218091E8280C
:1055C0009091E928A091EA28B091EB28BF93AF937E
:1055D0009F938F938CEE94E09F938F930E94C2923F
:1055E0008091FD288F938091FC288F938091FB28D8
:1055F0008F938091FA288F9388ED94E09F938F93F7
:105600000E94C2928091EC289091ED28A091EE2802
:10561000B091EF28BF93AF939F938F938AEC94E060
:105620009F938F930E94C2928DB79EB782960FB6BA
:10563000F8949EBF0FBE8DBF809101298F938091FA
:1056400000298F938091FF288F938091FE288F935C
:1056500086EB94E09F938F930E94C29261E070E08A
:1056600080E090E00E94B40B0F900F900F900F908D
:105670000F900F9061E070E081E090E00C94B40B2B
:10568000F894E0E0F0E081E2809357008491E2E05A
:10569000F0E041E2409357004491E4E0F0E091E211
:1056A00090935700E49190E0A0E0B0E0DC019927EE
:1056B000882750E060E070E0762F652F542F442754
:1056C000840F951FA61FB71F8E0F911DA11DB11D21
:1056D0008093C81B9093C91BA093CA1BB093CB1B8C
:1056E00078940895CF93DF93CDB7DEB761970FB667
:1056F000F894DEBF0FBECDBF48E250E06EE170E02F
:1057000087E29BE10E9416942091271B3091281B71
:105710004091291B50912A1B60912B1B70912C1BCF
:1057200080912D1B90912E1BAFEF0E94318E09F0BE
:105730005DC08DE48093271B80E88093281B84E064
:105740008093291B10922A1B10922B1B10922C1B4A
:1057500010922D1B10922E1B8CE390E09093301B27
:1057600080932F1B1092311B1092321B1092331B0F
:105770001092341B1092351B1092361B1092371B5F
:105780001092381B10923A1B1092391B10923B1B3F
:1057900010923C1B10923D1B10923E1B10923F1B1F
:1057A0001092401B1092411B1092421B1092441BFE
:1057B0001092431B1092451B1092461B1092471BE0
:1057C0001092481B1092491B10924A1B10924B1BBF
:1057D00010924C1B10924E1B10924D1B48E250E051
:1057E0006EE170E087E29BE10E94349444E050E077
:1057F0006AE170E0CE010B960E9416948B859C8521
:10580000AD85BE858F3F2FEF9207A207B207A9F49F
:105810008AE090E4A0E0B0E08093580290935902AF
:10582000A0935A02B0935B0244E050E06AE170E05A
:1058300088E592E00E94349408C0809358029093C7
:105840005902A0935A02B0935B0242E050E066E531
:1058500070E0CE010F960E9416948F8598898F3F35
:105860002FEF920769F41092C6091092C50942E021
:1058700050E066E570E085EC99E00E94349404C045
:105880009093C6098093C50949E050E06AE070E052
:1058900082E099E20E9416940E94EC0C44E050E0F1
:1058A0006AE470E0CE010B960E9416948B859C856D
:1058B000AD85BE8544E050E06AE470E08F3F9F4FC5
:1058C000AF4FBF4F29F488E792E00E94349404C0A0
:1058D00088E792E00E94169444E050E066E470E0AD
:1058E000CE010B960E9416948B859C85AD85BE8556
:1058F00044E050E066E470E08F3F9F4FAF4FBF4FF2
:1059000029F484E792E00E94349404C084E792E092
:105910000E94169444E050E06EE470E0CE010B96D5
:105920000E9416948B859C85AD85BE8544E050E031
:105930006EE470E08F3F9F4FAF4FBF4F29F48CE76D
:1059400092E00E94349404C08CE792E00E94169486
:1059500041E050E069E170E0CE0141960E9416946A
:10596000898941E050E069E170E08F3F29F481ECE2
:1059700099E00E94349404C081EC99E00E9416944E
:1059800041E050E068E170E0CE0141960E9416943B
:10599000898941E050E068E170E08F3F29F487E5B4
:1059A00092E00E94349404C087E592E00E9416942D
:1059B00041E050E067E170E0CE0141960E9416940C
:1059C000898941E050E067E170E08F3F29F486E586
:1059D00092E00E94349404C086E592E00E941694FE
:1059E0004AE050E060E070E0CE0101960E9416941B
:1059F00089814AE050E060E070E08F3F29F48EE05A
:105A00009BE10E94349404C08EE09BE10E941694B6
:105A100044E050E062E570E0CE010B960E941694DF
:105A20008B859C85AD85BE8544E050E062E570E0E5
:105A30008F3F9F4FAF4FBF4F29F480E892E00E9405
:105A4000349404C080E892E00E94169444E050E050
:105A500063E170E0CE010B960E9416948B859C85C5
:105A6000AD85BE8544E050E063E170E08F3F9F4F1D
:105A7000AF4FBF4F29F482E592E00E94349404C0F6
:105A800082E592E00E94169461960FB6F894DEBF0C
:105A90000FBECDBFDF91CF910895CF92DF92EF92ED
:105AA000FF92609171027091720280E090E00E941A
:105AB000F79165E975E00E940B92892B09F01FC1EF
:105AC0008DE48093271B80E88093281B84E08093DB
:105AD000291B10922A1B10922B1B10922C1B109228
:105AE0002D1B10922E1B8CE390E09093301B809323
:105AF0002F1B1092311B1092321B1092331B1092ED
:105B0000341B1092351B1092361B1092371B1092CB
:105B1000381B10923A1B1092391B10923B1B1092AB
:105B20003C1B10923D1B10923E1B10923F1B10928B
:105B3000401B1092411B1092421B1092441B10926A
:105B4000431B1092451B1092461B1092471B10924C
:105B5000481B1092491B10924A1B10924B1B10922B
:105B60004C1B10924E1B10924D1B48E250E06EE110
:105B700070E087E29BE10E9434948AE090E4A0E028
:105B8000B0E08093580290935902A0935A02B093C8
:105B90005B0244E050E06AE170E088E592E00E9438
:105BA00034941092C6091092C50942E050E066E5AF
:105BB00070E085EC99E00E94349442E2C42EDD242A
:105BC000DA944CECE42E4BE3F42EC0927802D0929F
:105BD0007902E0927A02F0927B0244E050E06AE4BB
:105BE00070E088E792E00E943494C0927402D092F0
:105BF0007502E0927602F092770244E050E066E4AB
:105C000070E084E792E00E94349487ED94E3AFEE75
:105C1000BCE380937C0290937D02A0937E02B093BC
:105C20007F0244E050E06EE470E08CE792E00E9476
:105C300034948AE999E9A9E1B0E4809380029093D1
:105C40008102A0938202B093830244E050E062E5B7
:105C500070E080E892E00E9434941092C10980E0E4
:105C60000E943E6A41E050E069E170E081EC99E019
:105C70000E9434948AE1809357020E94E56841E0D3
:105C800050E068E170E087E592E00E9434948FE094
:105C90008093560241E050E067E170E086E592E0D3
:105CA0000E9434948AE0EEE0FBE1DF011D928A95C8
:105CB000E9F74AE050E060E070E0CF010E943494E0
:105CC00080EA96E8A1E0B0E08093520290935302FC
:105CD000A0935402B093550244E050E063E170E0B9
:105CE00082E592E00E94349481E00E94582280E094
:105CF00090E0FF90EF90DF90CF900C94000DFF901C
:105D0000EF90DF90CF9008952F923F924F925F9245
:105D10006F927F928F929F92AF92BF92CF92DF92BB
:105D2000EF92FF920F931F93CF93DF93CDB7DEB720
:105D30002B970FB6F894DEBF0FBECDBF9B878A8727
:105D40004A01FC0180819181892B11F00C94224140
:105D50006091710270917202CA010E94F79160E82D
:105D600070E0C4010E942A92009759F46091CD31ED
:105D70007091CE318AE090E00E947E9281E00C9496
:105D800027418130910561F4F401B0801B2D110F82
:105D9000110B012F412E512E612E712EA12EBCC050
:105DA00082309105B9F4F4018081992787FD90959F
:105DB000982F88272181820F911D27FD9A95B82E53
:105DC000192F092F000F000B402E502E602E702E21
:105DD000A02EA2C083309105B1F5F4012081922F4D
:105DE000990F990B392F492F592F692F792F892F07
:105DF00000E10E94D38D19012A013B01B82FA92F80
:105E00002181922F990F990B392F492F592F692FE3
:105E1000792F892F08E00E94D38D59016A017B01F7
:105E20008C019101A201B3018B2F9A2F0E940A8E3F
:105E3000A2801A2D110F110BB12EC12ED12EE12EE1
:105E4000F12E012F55C004970CF45DC0F4012081A0
:105E5000922F990F990B392F492F592F692F792F8D
:105E6000892F08E10E94D38D19012A013B01B82F27
:105E7000A92F2181922F990F990B392F492F592F33
:105E8000692F792F892F00E10E94D38D59016A0172
:105E90007B018C019101A201B3018B2F9A2F0E94EB
:105EA0000A8EA3801A2D110F110BB12EC12ED12EE7
:105EB000E12EF12E012F0E940A8E19012A013B01C9
:105EC000B82FA92F2281922F990F990B392F492F83
:105ED000592F692F792F892F08E00E94D38D5901FE
:105EE0006A017B018C019101A201B3018B2F9A2FD2
:105EF0000E940A8EB22E132F042F452E562E672E87
:105F0000782EA92E09C07AE0B72E10E000E0412CCF
:105F1000512C612C712CA12C0E94AB0B2B2D312FFD
:105F2000402F542D652D762D872D9A2D2736FFE68F
:105F30003F07FCE64F075105610571058105910595
:105F400011F40C942F3B2736EFE63E07ECE64E07A4
:105F50005105610571058105910511F008F096C1A3
:105F60002936F2E73F0741055105610571058105B5
:105F7000910511F40C944C3E2936E2E73E074105A9
:105F80005105610571058105910511F008F0A6C064
:105F90002536F4E63F074105510561057105810588
:105FA000910509F457C62536E4E63E07410551053B
:105FB000610571058105910509F0B8F5A6E70E9414
:105FC000318E11F40C94A1380E94318E09F068F4DE
:105FD000A8E60E94318E09F483C6A5E70E94318E9F
:105FE00011F40C948B380C9420412B2D312F402F21
:105FF000542D652D762D872D9A2D2A33F6E23F07F5
:1060000041055105610571058105910509F41FC31D
:10601000243631464105510561057105810591051B
:1060200011F40C94C53E0C9420412B2D312F402FA0
:10603000542D652D762D872D9A2D2737FFE63F07A6
:1060400041055105610571058105910511F40C9417
:10605000703C2737EFE63E074105510561057105A4
:106060008105910509F0C8F42436F9E63F0741059A
:106070005105610571058105910511F40C94643891
:1060800025363E464105510561057105810591059D
:1060900011F40C94A43C0C9420412B2D312F402F53
:1060A000542D652D762D872D9A2D2333F1E73F074B
:1060B00041055105610571058105910511F40C94A7
:1060C000C53E2536324741055105610571058105FB
:1060D000910511F40C946E3D0C9420412B2D312F21
:1060E000402F542D652D762D872D9A2D2837F4E6D7
:1060F0003F07F1E64F0751056105710581059105DF
:1061000009F4B5C22837E4E63E07E1E64E0751053B
:10611000610571058105910511F008F050C028371F
:10612000F4E73F07410551056105710581059105BA
:1061300009F48DC22837E4E73E07410551056105A2
:1061400071058105910509F0C8F42337F2E73F078F
:1061500041055105610571058105910511F40C9406
:106160009D3E233733474105510561057105810582
:10617000910511F40C94B13E0C9420412B2D312F3C
:10618000402F542D652D762D872D9A2D2133F4E641
:106190003F07F1E64F07510561057105810591053E
:1061A00009F469C22336344641465105610571053B
:1061B0008105910511F40C94C53E0C9420412B2DC2
:1061C000312F402F542D652D762D872D9A2D233676
:1061D000FDE63F07F8E64F075105610571058105AA
:1061E000910509F440C32336EDE63E07E8E64E0785
:1061F0005105610571058105910509F0C8F4223644
:10620000F5E63F07F4E64F07510561057105810585
:10621000910509F41FC522373247454651056105EE
:1062200071058105910511F40C94C93B0C94204132
:106230002B2D312F402F542D652D762D872D9A2D06
:106240002336F2E33F07F9E64F0751056105710573
:106250008105910509F42FC22436E3E63E07ECE6FA
:106260004E075105610571058105910511F40C94E6
:106270002C3B2D3635474846510561057105810592
:10628000910511F00C9420410C94DB3E2B2D312F05
:10629000402F542D652D762D872D9A2D2136EDE634
:1062A0003E07E5E74E07E8E65E07610571058105F3
:1062B000910511F40C948E3C2136FDE63F07F5E77D
:1062C0004F07F8E65F07610571058105910511F03B
:1062D00008F0DAC02437E8E73E07E4E74E07510547
:1062E000610571058105910509F497C72437F8E721
:1062F0003F07F4E74F0751056105710581059105D9
:1063000011F008F055C02133E1E33E07E1E74E0705
:106310005105610571058105910511F40C940A3C44
:106320002133F1E33F07F1E74F075105610571059F
:106330008105910509F0D0F42537E3E63E07EDE647
:106340004E075105610571058105910511F40C9405
:106350000A3C2033314341475105610571058105F0
:10636000910511F40C94C93B0C9420412B2D312F35
:10637000402F542D652D762D872D9A2D2037E5E65B
:106380003E07E2E74E07510561057105810591055C
:1063900011F40C946E3D2C36344744475105610589
:1063A00071058105910511F40C9449400C9420412C
:1063B0002B2D312F402F542D652D762D872D9A2D85
:1063C0002936ECE63E07E1E64E07E3E65E076105A7
:1063D00071058105910509F47BC22936FCE63F076A
:1063E000F1E64F07F3E65F07610571058105910549
:1063F00009F0E0F42437E4E63E07E7E74E075105ED
:10640000610571058105910511F40C9497402437BD
:106410003F464F465246610571058105910511F0D1
:106420000C9420410C9400000C9422412B2D312F10
:10643000402F542D652D762D872D9A2D2633E9E694
:106440003E07E5E74E07E5E65E0761057105810554
:10645000910509F449C42037FCE63F07F5E64F07EC
:10646000F8E65F07610571058105910509F438C4F7
:106470002E36314648465346610571058105910522
:1064800009F49FC60C9420412B2D312F402F542D01
:10649000652D762D872D9A2D2437F3E73F07F5E6F6
:1064A0004F07F2E75F07610571058105910511F45A
:1064B0000C941E3D2437E3E73E07E5E64E07E2E78E
:1064C0005E07610571058105910511F008F055C061
:1064D0002337F2E73F07F7E74F07F0E75F0761056C
:1064E00071058105910511F40C94213D2337E2E7F4
:1064F0003E07E7E74E07E0E75E07610571058105A6
:10650000910509F0C8F42237F7E73F07F0E74F0796
:106510005F07610571058105910509F4A8C123375D
:10652000354642475047610571058105910511F4D3
:106530000C948B3F0C9420412B2D312F402F542D48
:10654000652D762D872D9A2D2436FDE63F07F3E63F
:106550004F07F2E75F07610571058105910509F4B1
:10656000CEC421363C46454652476105710581053A
:10657000910509F4D6C30C9420412B2D312F402FC7
:10658000542D652D762D872D9A2D2437F2E73F0760
:10659000F1E64F07F5E75F07610571058105910594
:1065A00009F408C52437E2E73E07E1E64E07E5E7D0
:1065B0005E07610571058105910509F0C8F424376E
:1065C000F3E73F07F5E64F07F4E75F07610571055D
:1065D0008105910509F44CC6273730474847544791
:1065E000610571058105910509F4C1C50C9420412F
:1065F0002B2D312F402F542D652D762D872D9A2D43
:106600002F36FCE63F07FFE54F07F6E75F0761051A
:1066100071058105910509F41DC42C36E1E63E079C
:10662000E4E74E07E8E75E0761057105810591051E
:1066300011F40C9413402237374640475547610503
:1066400071058105910511F00C942041E0C783E0AC
:106650008093F0281092F2281092F12840EF58E22F
:1066600062E184E392E00E9448540C9422410E942B
:10667000BA150C94224121E042E161E080ED0E94D4
:10668000826121E042E161E080ED0E94826121E0CF
:1066900042E161E080ED0E94826121E042E161E03F
:1066A00080ED0E94826121E042E161E080ED0E9484
:1066B00082610C942241609171027091720280E0BB
:1066C00090E00E94F7916CE975E00E940B92892B93
:1066D00009F0C5C0609171027091720280E090E093
:1066E0000E94F7915C01009709F497C060EE73E097
:1066F0000E940B92892BE1F488EE93E0A0E0B0E0D9
:106700008093520290935302A0935402B093550287
:1067100068EE73E080E090E00E94A95F44E050E002
:1067200063E170E082E592E00E9434940C9422418F
:1067300062EA75E0C5010E940B92892BE1F480E1C9
:1067400097E2A0E0B0E08093520290935302A093AE
:106750005402B093550260E177E280E090E00E943D
:10676000A95F44E050E063E170E082E592E00E94BE
:1067700034940C94224165EA75E0C5010E940B92A5
:10678000892BE1F480EA96E8A1E0B0E08093520220
:1067900090935302A0935402B093550260EA76E8B6
:1067A00081E090E00E94A95F44E050E063E170E086
:1067B00082E592E00E9434940C94224169EA75E0EB
:1067C000C5010E940B92892BE1F480E89AE1A6E0D2
:1067D000B0E08093520290935302A0935402B0937E
:1067E000550260E87AE186E090E00E94A95F44E00B
:1067F00050E063E170E082E592E00E9434940C94F2
:10680000224187EF92E09F938F930E94C2920E9451
:10681000AB0B0F900F900C9422416091520270913B
:106820005302809154029091550228EE33E040E0EB
:1068300050E00E942A8C5F934F933F932F9383EFF6
:1068400092E09F938F930E94C2920E94AB0B0F9095
:106850000F900F900F900F900F900C9422410E9478
:106860002C100C9422410E9432160C94224160910B
:1068700071027091720280E090E00E94F7918C01A9
:106880006EE875E00E940B92892B19F477980C94AE
:10689000224161E975E0C8010E940B92892B19F42D
:1068A000779A0C942241779903C08EE895E002C054
:1068B00081E995E09F938F9380EA94E09F938F9373
:1068C0000E94C2920F900F900F900F900C94224153
:1068D000609171027091720280E090E00E94F791E5
:1068E0008C0168E575E00E940B92892B09F077C056
:1068F000609171027091720280E090E00E94F791C5
:106900008C01009711F40C9422416DEA75E00E940D
:106910000B92892BB1F482E29FEFACECBBE3809346
:10692000780290937902A0937A02B0937B0244E0BC
:1069300050E06AE470E088E792E00E9434940C949E
:10694000224163EB75E0C8010E940B92892BB1F4E0
:1069500082E29FEFACECBAE38093780290937902E5
:10696000A0937A02B0937B0244E050E06AE470E0C6
:1069700088E792E00E9434940C942241C8010E945E
:10698000E1902B013C0120E030E0A9010E947C88CD
:106990008823D9F081E00E94410A9B01AC01C30128
:1069A000B2010E948088609378027093790280938C
:1069B0007A0290937B0244E050E06AE470E088E75A
:1069C00092E00E9434940C94224186EE92E09F93D0
:1069D0008F930E94C2920F900F900C9422416BE50E
:1069E00075E0C8010E940B92892B09F077C0609175
:1069F00071027091720280E090E00E94F7918C0128
:106A0000009711F40C9422416DEA75E00E940B92FC
:106A1000892BB1F482E29FEFACECBBE3809374026C
:106A200090937502A0937602B093770244E050E011
:106A300066E470E084E792E00E9434940C94224172
:106A400063EB75E0C8010E940B92892BB1F482E2DE
:106A50009FEFACECBAE38093740290937502A0931D
:106A60007602B093770244E050E066E470E084E799
:106A700092E00E9434940C942241C8010E94E1905B
:106A80002B013C0120E030E0A9010E947C88882392
:106A9000D9F082E00E94410A9B01AC01C301B2011E
:106AA0000E948088609374027093750280937602CE
:106AB0009093770244E050E066E470E084E792E06F
:106AC0000E9434940C94224189ED92E09F938F931D
:106AD0000E94C2920F900F900C94224163E575E0E2
:106AE000C8010E940B92892B09F073C0609171025A
:106AF0007091720280E090E00E94F7918C01009703
:106B000011F40C9422416DEA75E00E940B92892BDE
:106B1000B1F487ED94E3AFEEBCE380937C029093F5
:106B20007D02A0937E02B0937F0244E050E06EE4C9
:106B300070E08CE792E00E9434940C94224163EB65
:106B400075E0C8010E940B92892B51F48AEC92E007
:106B50009F938F930E94C2920F900F900C942241AA
:106B6000C8010E94E1902B013C0120E030E0A90126
:106B70000E947C88882319F180E00E94410A4B0121
:106B80005C0121EE3AE744E95EE3C301B2010E94F1
:106B9000B587A50194010E94808860937C02709360
:106BA0007D0280937E0290937F0244E050E06EE489
:106BB00070E08CE792E00E9434940C9422418DEBBB
:106BC00092E09F938F930E94C2920F900F900C942B
:106BD00022410E94900A9F938F937F936F9386EB3D
:106BE00092E09F938F930E94C29282E00E94410A9A
:106BF0002091740230917502409176025091770293
:106C00000E94018B162F072FF82EE92E81E00E949B
:106C1000410AEF92FF920F931F93209178023091D7
:106C2000790240917A0250917B020E94018B9F93DE
:106C30008F937F936F938AEA92E09F938F930E9442
:106C4000C2920E94AB0B0FB6F894DEBF0FBECDBF51
:106C50000C942241609171027091720280E090E088
:106C60000E94F7910097C1F00E9476232091C509F8
:106C70003091C6098217930709F19093C609809352
:106C8000C50942E050E066E570E085EC99E00E94BD
:106C9000349489E994E002C082E994E09F938F9351
:106CA0000E94C2926091C5097091C60980E090E08F
:106CB0000E9488220E94AB0B0F900F9087E894E00F
:106CC0009F938F930E94C2926FEF7FEF80E090E0DE
:106CD0000E9488220E94AB0B0F900F900C942241CF
:106CE0000E94891F0C942241F4018481843329F489
:106CF00040E061E080E00E94D61180917302882319
:106D000011F40C9422411F928F9384E894E09F9396
:106D10008F930E94C2920F900F900F900F900C943F
:106D20002241F4018481893709F080C060917102A9
:106D30007091720280E090E00E94F7918C016EE801
:106D400075E00E940B92892B51F48091580290912A
:106D50005902A0915A02B0915B02906410C061E99F
:106D600075E0C8010E940B92892BD1F480915802E2
:106D700090915902A0915A02B0915B029F7B80933F
:106D8000580290935902A0935A02B0935B0244E0D8
:106D900050E06AE170E088E592E00E94349446C0D9
:106DA00068EB75E0C8010E940B92892B21F5809158
:106DB000261B8F938091251B8F938091241B8F938B
:106DC0008091231B8F938091221B8F938091211B95
:106DD0008F938091201B8F9380911F1B8F938FE740
:106DE00092E09F938F930E94C2920FB6F894DEBFF9
:106DF0000FBECDBF1BC08091580290915902A09147
:106E00005A02B0915B0296FF03C08EE895E002C083
:106E100081E995E09F938F938BE792E09F938F9307
:106E20000E94C2920F900F900F900F90809173026A
:106E3000882311F40C9422411F928F9381E894E0EF
:106E40009F938F930E94C2920F900F900F900F907C
:106E50000C942241F40184818737E9F56091710235
:106E60007091720280E090E00E94F7910097D9F053
:106E70000E94E1902B013C0120E030E0A9010E943A
:106E80007C88882381F04092800250928102609237
:106E900082027092830244E050E062E570E080E894
:106EA00092E00E943494809183028F9380918202B9
:106EB0008F93809181028F93809180028F938DE6D2
:106EC00092E09F938F930E94C2920F900F900F9029
:106ED0000F900F900F9080917302882311F40C94FF
:106EE00022411F928F938EE794E09F938F930E948D
:106EF000C2920F900F900F900F900C9422416091CE
:106F000071027091720280E090E00E94F7918C0112
:106F10006EE875E00E940B92409058025090590222
:106F200060905A0270905B02892B19F4689457F8AC
:106F300009C061E975E0C8010E940B92892B99F4A0
:106F4000E89457F8409258025092590260925A02BF
:106F500070925B0244E050E06AE170E088E592E004
:106F60000E94349413C057FE03C08EE895E002C01F
:106F700081E995E09F938F9389E692E09F938F93A9
:106F80000E94C2920F900F900F900F908091730209
:106F9000882311F40C9422411F928F938BE794E085
:106FA0009F938F930E94C2920F900F900F900F901B
:106FB0000C942241609171027091720280E090E025
:106FC0000E94F7915C016EEB75E00E940B92892B99
:106FD00011F489E108C062EC75E0C5010E940B92D2
:106FE000892B49F480E18093C4001092C50082E0AF
:106FF0008093C00055C066EC75E0C5010E940B92FD
:10700000892B11F488E0EFCF6BEC75E0C5010E948D
:107010000B92892B39F060ED75E0C5010E940B924F
:10702000892B11F483E0DFCF8091C400893141F4D2
:1070300084E692E09F938F930E94C2920F900F90EC
:107040008091C400803141F48FE592E09F938F934B
:107050000E94C2920F900F908091C400883041F43A
:1070600089E592E09F938F930E94C2920F900F90B8
:107070008091C400833041F483E592E09F938F9325
:107080000E94C2920F900F908091C400883041F40A
:107090008DE492E09F938F930E94C2920F900F9085
:1070A00080917302882311F40C9422411F928F93D4
:1070B00088E794E09F938F930E94C2920F900F9065
:1070C0000F900F900C9422416091710270917202A6
:1070D00080E090E00E94F7916DEA75E00E940B92CB
:1070E000892B11F481E001C080E00E945822809138
:1070F0007302882311F40C9422411F928F9385E729
:1071000094E09F938F930E94C2920F900F900F90E4
:107110000F900C9422410E947E208091730288235C
:1071200011F40C9422411F928F9382E794E09F9375
:107130008F930E94C2920F900F900F900F900C941B
:1071400022410E947A2080917302882311F40C94CA
:1071500022411F928F938FE694E09F938F930E941A
:10716000C2920F900F900F900F900C94224160915B
:1071700071027091720280E090E00E94F7910E948B
:10718000E590803170F48093C1090E943E6A41E02D
:1071900050E069E170E081EC99E00E9434940C9435
:1071A00022418091C1091F928F9383E492E09F93C3
:1071B0008F930E94C2920F900F900F900F900C949B
:1071C0002241609171027091720280E090E00E9411
:1071D000F7910E94E59095EF980F903170F48093AD
:1071E00057020E94E56841E050E068E170E087E501
:1071F00092E00E9434940C942241809157021F9295
:107200008F938AE392E09F938F930E94C2920F9094
:107210000F900F900F900C94224160917102709129
:10722000720280E090E00E94F791009789F04AE0B6
:1072300050E0BC018EE09BE10E941B924AE050E0CE
:1072400060E070E08EE09BE10E9434940C94224157
:107250008EE09BE19F938F9385ED95E09F938F93B5
:107260000E94B0920F900F900F900F900C942241BB
:10727000609171027091720280E090E00E94F7913B
:107280005C0160EE73E00E940B92892BD9F4219A85
:107290008091580290915902A0915A02B0915B02DC
:1072A00080618093580290935902A0935A02B09340
:1072B0005B0244E050E06AE170E088E592E00E9401
:1072C0003494C0C76CE575E0C5010E940B92892B10
:1072D000D9F4229A8091580290915902A0915A02B1
:1072E000B0915B0280628093580290935902A09300
:1072F0005A02B0935B0244E050E06AE170E088E536
:1073000092E00E9434949EC762EC73E0C5010E9433
:107310000B92892BD9F4239A8091580290915902AB
:10732000A0915A02B0915B028064809358029093BE
:107330005902A0935A02B0935B0244E050E06AE124
:1073400070E088E592E00E9434947CC76FEF74E0AF
:10735000C5010E940B92892BD9F4239A809158027F
:1073600090915902A0915A02B0915B02806880937B
:10737000580290935902A0935A02B0935B0244E0E2
:1073800050E06AE170E088E592E00E9434945AC7C8
:107390006CE679E0C5010E940B92892B71F581E0C2
:1073A0008093542487E29BE1909356248093552444
:1073B00010925824109257248091580290915902AB
:1073C000A0915A02B0915B02916080935802909311
:1073D0005902A0935A02B0935B0244E050E06AE184
:1073E00070E088E592E00E94349444E554E262E162
:1073F00084E392E00E94485425C769EE73E0C5011A
:107400000E940B92892B11F5E7E5FBE11192119295
:107410002BE1E737F207D1F780915802909159029A
:10742000A0915A02B0915B029260809358029093AF
:107430005902A0935A02B0935B0244E050E06AE123
:1074400070E088E592E00E943494FCC661E975E042
:10745000C5010E940B9240915802509159026091CF
:107460005A0270915B02892BC1F44F705C7F40938C
:1074700058025093590260935A0270935B022B9A00
:1074800044E050E06AE170E088E592E00E943494C4
:107490008091F9280E94FA68D5C644FF03C08EE89F
:1074A00095E002C081E995E09F938F938FE292E08F
:1074B0009F938F930E94C292809158020F900F90D9
:1074C0000F900F9085FF03C08EE895E002C081E920
:1074D00095E09F938F9384E292E09F938F930E9415
:1074E000C292809158020F900F900F900F9086FFDC
:1074F00003C08EE895E002C081E995E09F938F93E9
:1075000089E192E09F938F930E94C29280915802EA
:107510000F900F900F900F9087FF03C08EE895E0BB
:1075200002C081E995E09F938F938EE092E09F9354
:107530008F930E94C2928091580290915902A0911B
:107540005A02B0915B020F900F900F900F9090FF36
:1075500003C08EE895E002C081E995E09F938F9388
:1075600083E092E09F938F930E94C2928091580291
:1075700090915902A0915A02B0915B020F900F9026
:107580000F900F9091FF03C08EE895E002C081E953
:1075900095E09F938F9388EF91E09F938F930E9444
:1075A000C2928091580290915902A0915A02B091D2
:1075B0005B020F900F900F900F9091FF43C68DEDDF
:1075C00095E00E94E69257E5A52E5BE1B52E0BE013
:1075D00010E065EE862E65E0962EF50180819181A2
:1075E000F2E0AF0EB11C9F938F931F930F939F9266
:1075F0008F920E94B0920F5F1F4F0F900F900F90CD
:107600000F900F900F900B31110539F71BC68BE6C9
:1076100094E09F938F930E94C292809173020F9087
:107620000F90882361F01F928F9388E694E09F93D8
:107630008F930E94C2920F900F900F900F90F8942A
:1076400028E088E190E00FB6F894A8958093600058
:107650000FBE20936000FFCF0E943361F3C560919D
:1076600071027091720280E090E00E94F7918C01AB
:107670006EE875E00E940B92892BE9F40E94E467A2
:107680008091580290915902A0915A02B0915B02E8
:107690008D7F81608093580290935902A0935A0283
:1076A000B0935B0244E050E06AE170E088E592E06C
:1076B0000E943494C7C561E975E0C8010E940B922D
:1076C000892BE1F40E949C678091580290915902A5
:1076D000A0915A02B0915B028C7F809358029093E4
:1076E0005902A0935A02B0935B0244E050E06AE171
:1076F00070E088E592E00E943494A4C560EF75E0E4
:10770000C8010E940B92892BE9F40E949C6780912A
:10771000580290915902A0915A02B0915B028E7F5B
:1077200082608093580290935902A0935A02B093BA
:107730005B0244E050E06AE170E088E592E00E947C
:10774000349480C58091580281FF0FC080EF95E08E
:107750009F938F9384EF91E09F938F930E94C292A7
:107760000F900F900F900F906DC580FF03C08EE8B3
:1077700095E002C081E995E09F938F9380EF91E0BF
:107780009F938F930E94C2920F900F900F900F9033
:1077900059C5809152248F93809151248F93809169
:1077A00050248F9380914F248F9380914E248F93F8
:1077B00080914D248F9380914C248F9380914B2402
:1077C0008F9380914A248F93809149248F93809145
:1077D00048248F93809147248F9385E494E09F936E
:1077E0008F930E94C292809173020FB6F894DEBF0D
:1077F0000FBECDBF882309F425C51F928F9382E465
:1078000094E09F938F930E94C2920F900F900F90DD
:107810000F9018C5F89481E090E029E0FC012093D6
:107820005700C895E02C80E090E0FC0120935700C1
:10783000C895F02C7894F89483E090E0FC012093B4
:107840005700C895002D82E090E0FC01209357007E
:10785000C895102D78948091CB1B8F938091CA1B73
:107860008F938091C91B8F938091C81B8F9328E3BE
:1078700034E03F932F930E94C2921F92EF921F9287
:10788000FF921F920F931F921F9381E194E09F93A9
:107890008F930E94C2920E941821809166001F92CD
:1078A0008F9385E094E09F938F930E94C2920E94F1
:1078B000AB0B809173020FB6F894DEBF0FBECDBF45
:1078C000882309F4BFC41F928F9382E094E09F93B2
:1078D0008F930E94C2920F900F900F900F90B2C49E
:1078E00060E070E080E090E00E94B40B60E070E047
:1078F00081E090E00E94B40B80917302882309F428
:10790000A1C41F928F938FEF93E09F938F930E9458
:10791000C2920F900F900F900F9094C40E944C1F32
:107920000E94AB0B80917302882309F48BC41F92D1
:107930008F938CEF93E09F938F930E94C2920F904E
:107940000F900F900F907EC460917102709172023F
:1079500080E090E00E94F79165EF75E00E940B9245
:10796000892B31F5F8948CEF99E00E9435555C0134
:10797000009769F0C5010F960E943958B50184E05F
:1079800092E00E94EF54C5010E94DD55F0CF8CEFCC
:1079900099E00E94C255892B29F08CEF99E00E9452
:1079A0006E55F5CF8CEF99E00E943155789434C034
:1079B0008CEF99E00E9435555C010BEF15E0A114A6
:1079C000B10451F1F50186811F928F9380851F923A
:1079D0008F9385811F928F9381851F928F938781CB
:1079E0001F928F9384811F928F9383811F928F9315
:1079F00082811F928F9382851F928F931F930F9383
:107A00000E94B092C5010E94DD555C010FB6F8944A
:107A1000DEBF0FBECDBFD3CF80917302882309F4A0
:107A200011C41F928F9389EF93E09F938F930E94CD
:107A3000C2920F900F900F900F9004C40E944D2D92
:107A400001C4609171027091720280E090E00E9426
:107A5000F7918C016AE376E00E940B92892BD1F4B6
:107A60008091580290915902A0915A02B0915B0204
:107A7000977F8093580290935902A0935A02B09333
:107A80005B0244E050E06AE170E088E592E00E9429
:107A90003494D8C363EB75E0C8010E940B92892B24
:107AA000D1F48091580290915902A0915A02B0915C
:107AB0005B0298608093580290935902A0935A02F7
:107AC000B0935B0244E050E06AE170E088E592E048
:107AD0000E943494B7C30E944B09B4C360917102F1
:107AE0007091720280E090E00E94F791FC01208189
:107AF0002332B1F44AE050E060E070E001960E9469
:107B0000998E1B01609171027091720280E090E089
:107B10000E94F791F4E02F1631040CF094C002C0DB
:107B2000212C312C009709F48EC01982BE016F5FA1
:107B30007F4F0E94752729013A014B01B82FA92FC9
:107B40008AE0829DF001839DF00D1124E95DF44EE1
:107B500020812A8331813B8382818C8393819D8321
:107B600024812E8335813F838681888797819987F9
:107B70009201A301B4018B2F9A2FAA80BB80CC80E5
:107B8000DD80EE80FF80088519850E94288E09F42B
:107B90005DC08981882351F18CF02A81422A3B8182
:107BA000532A8C81682A9D81792A2E81822A3F81DD
:107BB000932A8885B82B9985A92B18C04094509496
:107BC0006094709480949094B095A0952A814222FC
:107BD0003B8153228C8168229D8179222E818222D1
:107BE0003F8193228885B8239985A92340825182B9
:107BF0006282738284829582B683A78348E250E0D2
:107C00006EE170E087E29BE10E94349481EF93E0A3
:107C10009F938F930E94C2928AE0829DF001839D80
:107C2000F00D1124E95DF44E2081318142815381B0
:107C300064817581868197810E9411240E94AB0B1B
:107C40000F900F9003C082E00E94172985EE93E009
:107C50009F938F930E94C2922FEF3FEF4FEF5FEF02
:107C60006FEF7FEF8FEF9FEF0E9411240E94AB0B0D
:107C7000809173020F900F90882309F4E3C21F9242
:107C80008F9382EE93E09F938F930E94C2920F9006
:107C90000F900F900F90D6C2609171027091720296
:107CA00080E090E00E94F791FC0120812332A1F452
:107CB0004AE050E060E070E001960E94998E8B01EE
:107CC000609171027091720280E090E00E94F791E1
:107CD00004301105ECF402C000E010E00097C1F0A0
:107CE0004AE050E060E070E00E94CD8F2AE0209FE3
:107CF000F001219FF00D1124E95DF44E718760873A
:107D000048E250E06EE170E087E29BE10E9434942B
:107D100081E00E94172980917302882309F492C29E
:107D20001F928F938FED93E09F938F930E94C29247
:107D30000F900F900F900F9085C20E947258809103
:107D40007302882309F47EC21F928F938CED93E017
:107D50009F938F930E94C2920F900F900F900F905D
:107D600071C20E948C2980917302882309F46AC22F
:107D70001F928F9389ED93E09F938F930E94C292FD
:107D80000F900F900F900F905DC280E090E00E94E6
:107D9000342180917302882309F454C21F928F9377
:107DA00086ED93E09F938F930E94C2920F900F9065
:107DB0000F900F9047C280913D2081FF2DC00E94FF
:107DC000D01E892B49F58091341C8F938091331CF0
:107DD0008F938091321C8F938091311C8F938BEC09
:107DE00093E09F938F930E94C292809111298F9369
:107DF000809110298F9380910F298F9380910E2964
:107E00008F938EEB93E09F938F930E94C2920FB655
:107E1000F894DEBF0FBECDBF0E94AB0B80913D201A
:107E200090913E2090FF63C081E090E00E94471E49
:107E30003B014C0180E090E00E94471E1B012C0199
:107E40000E94A51D9F928F927F926F928DEA93E080
:107E50009F938F930E94C2925F924F923F922F9274
:107E60008DE993E09F938F930E94C292222D332D30
:107E7000442D552D662D772D882D992D0E94481C57
:107E80009F938F937F936F9382E993E09F938F9358
:107E90000E94C292222D332D442D552D662D772D13
:107EA000882D992D0E94A91C9F938F937F936F9388
:107EB00084E893E09F938F930E94C292222D332DEA
:107EC000442D552D662D772D882D992D0E940A1D44
:107ED0009F938F937F936F9381E793E09F938F930B
:107EE0000E94C2920FB6F894DEBF0FBECDBF0E94B3
:107EF000AB0B80917302882309F4A4C11F928F9366
:107F00008EE693E09F938F930E94C2920F900F9002
:107F10000F900F9097C180913D2082FF2BC021E0F0
:107F200048E061E083E00E944B1380912F1C8F9307
:107F300080912E1C8F9380912D1C8F9380912C1CEF
:107F40008F9380912B1C8F9380912A1C8F9380910B
:107F5000291C8F938091281C8F9387E593E09F9332
:107F60008F930E94C2920E94AB0B0FB6F894DEBFB3
:107F70000FBECDBF80913D2090913E2091FF41C02A
:107F80000E949517B62EA72E982E892E20E030E05D
:107F900048EC52E4D501F4016B2F7A2F8F2F9E2FDE
:107FA0000E94018B20E836EE45EC57E40E94808861
:107FB00021E03EED42E45EE30E94648B9B01AC0154
:107FC00060E070E080E89FE30E94B5872BE43AE32D
:107FD0004DEB57E30E9480889F938F937F936F931D
:107FE0008F929F92AF92BF928EE393E09F938F9375
:107FF0000E94C2920E94AB0B0FB6F894DEBF0FBE78
:10800000CDBF80917302882309F41CC11F928F9306
:108010008BE393E09F938F930E94C2920F900F90F7
:108020000F900F900FC1609171027091720280E009
:1080300090E00E94F7916FE376E00E940B92892B0B
:10804000B1F4609171027091720280E090E00E9440
:10805000F791009709F4F6C00E94E590803108F08E
:10806000F1C090915201982B90935201EBC08091F6
:1080700052018F701F928F9383EE91E09F938F93A5
:108080000E94C2920E94AB0B0F900F900F900F9026
:10809000D9C0609171027091720280E090E00E94FC
:1080A000F791009711F14AE050E060E070E00E9423
:1080B000998E603198F4609356021F926F938EE20E
:1080C00093E09F938F930E94C29241E050E067E15A
:1080D00070E086E592E00E94349411C080915602CF
:1080E0001F928F9385E293E006C0809156021F9203
:1080F0008F938CE193E09F938F930E94C2920F9095
:108100000F900F900F900E94AB0B80917302882309
:1081100009F498C01F928F9389E193E09F938F9306
:108120000E94C2920F900F900F900F908BC06091A1
:1081300071027091720280E090E00E94F7918C01D0
:108140006EE875E00E940B92892BE1F40E944D6667
:108150008091580290915902A0915A02B0915B020D
:1081600090618093580290935902A0935A02B09361
:108170005B0244E050E06AE170E088E592E00E9432
:10818000349460C061E975E0C8010E940B92892BAC
:1081900081F5F8940E945B6688E10FB6F8948093AD
:1081A0006000109260000FBE84B7877F84BF80910B
:1081B00060008861809360001092600078948091E4
:1081C000580290915902A0915A02B0915B029F7E91
:1081D0008093580290935902A0935A02B0935B0285
:1081E00044E050E06AE170E088E592E00E94349457
:1081F00029C064E476E0C8010E940B9240915802C5
:108200005091590260915A0270915B02892B21F4BE
:1082100054FF18C0F894FFCF54FF03C08EE895E0D8
:1082200002C081E995E09F938F938FED91E09F933A
:108230008F930E94C2920F900F900F900F9002C0E8
:108240000E94701FEA85FB851182108283E02B96C5
:108250000FB6F894DEBF0FBECDBFDF91CF911F9157
:108260000F91FF90EF90DF90CF90BF90AF909F90D5
:108270008F907F906F905F904F903F902F900895D8
:108280000F931F93CF93DF93EC018A01888199812B
:10829000009711F18037904121F01982188283E014
:1082A00020C06231E9F4A80162E170E08DEE99E04E
:1082B0000E94842E84E08093F0281092F22810927D
:1082C000F1281093F4280093F32840EF58E262E17C
:1082D00084E392E00E94485480E790E19983888388
:1082E00081E0DF91CF911F910F9108950E94416627
:1082F0006C9A6B9A6A9A6F9A729A749A739A779A2E
:10830000809880B3897F80BB8398849887E080932E
:108310007E00549A0E94402B0E94722B81E00E94A2
:10832000B50980E090E00E94000D609152027091CA
:10833000530280915402909155020E94A95F0E94BD
:10834000A40A60933F247093402480934124909327
:1083500042248091580286FD239A0895CF93DF939B
:10836000EC0188819981009741F08B35904109F4A7
:108370008CC01982188283E093C00E94764180915C
:10838000580280FD05C081FF01C01D9B0E949C67B3
:10839000809170008C7F809370008091B600806225
:1083A0008093B6001092B20082E08093B100809179
:1083B000B6008770E1F78091700081608093700053
:1083C00069E679E080E090E00E942B660E947A20C6
:1083D00080E00E94582280EE9EE09F938F930E943F
:1083E000C2920E942C1080913D200F900F9086FD2C
:1083F0000E94DF6080913D2090913E2090FD0E9480
:10840000611D80913D2087FF06C021E04CE061E0C6
:1084100080ED0E9482618091C1090E943E6A809134
:1084200057020E94E5680E94E2688093EC098091FF
:1084300057020E94E5688091C1091F928F93809135
:10844000EC091F928F9389E496E09F938F930E948B
:10845000B0921092EE091092ED090F900F900F90CC
:108460000F900F900F9088E492E090930C298093E6
:108470000B2983E290E09093FF118093FE118BE52E
:1084800090E19983888381E00BC06332E1F748E68D
:1084900054E260E070E08DEE99E00E94842EE3CF1C
:1084A000DF91CF9108958436910514F19F938F93B6
:1084B0008BE596E09F938F930E94B0928091472422
:1084C00090914824A0914924B0914A240196A11D7D
:1084D000B11D8093472490934824A0934924B093DE
:1084E0004A240F900F900F900F9081E090E0089534
:1084F00080E090E008952F923F924F925F926F92AA
:108500007F928F929F92AF92BF92CF92DF92EF9223
:10851000FF920F931F93CF93DF93CDB7DEB7C85968
:10852000D1090FB6F894DEBF0FBECDBFCF56DF4FD7
:1085300099838883C159D0408A01633871F481EFEF
:1085400099E0C856DF4F6883C859D0400E948B52CB
:10855000C856DF4F6881C859D040CF56DF4FA88139
:10856000B981C159D0402D913C912830B0E13B07F1
:1085700009F4C9C340F42115310581F026343E4089
:1085800009F407C4FBC32A3140E1340709F4D7C317
:108590002132304111F40C94934FF0C34AEE52E073
:1085A00061E870E081EF99E00E94715286E49EE0FC
:1085B000A1C3E3E0F0E0EC0FFD1FE20FF31F108218
:1085C000C9010E945342892B89F720E030E040E046
:1085D00050E0C357DF4F6881CD58D040627070E0E3
:1085E00080E090E0A0E00E94318E09F084C6C5577B
:1085F000DF4F2881CB58D040287030E040E050E079
:1086000060E070E080E090E0A0E00E94318EA1F197
:1086100027E04AE250E06BE270E089E290E00E94DD
:10862000C35C82E099E20E94315FBC01882777FD3C
:108630008095982F0E941F8920E030E048EC52E49A
:108640000E9480889F938F937F936F938FE896E02B
:108650009F938F931F9287E78F93CE018E0D9F1D5F
:1086600003969F938F930E941393E80EF91E0FB603
:10867000F894DEBF0FBECDBFC557DF4F2881CB5862
:10868000D040207130E040E050E060E070E080E0F9
:1086900090E0A0E00E94318EF1F126E04AE250E045
:1086A0006BE270E089E290E00E94C35C81E090E0C0
:1086B0000E94390B8093C00980E89BE10E94315FE2
:1086C000BC01882777FD8095982F0E941F8920E0A4
:1086D00030E048EC52E40E9480889F938F937F9310
:1086E0006F9389E996E09F938F931F9287E78F930B
:1086F000C7010296E1E0F0E0EC0FFD1F8E0F9F1F17
:108700009F938F930E941393E80EF91E0FB6F8946F
:10871000DEBF0FBECDBF272D30E040E050E060E06F
:1087200070E080E090E0A0E00E94318E01F10E94B4
:10873000F50A9F938F937F936F9384EA96E09F93BC
:108740008F931F9287E78F93C701029641E050E015
:108750004C0F5D1F840F951F9F938F930E9413935F
:10876000E80EF91E0FB6F894DEBF0FBECDBFC55799
:10877000DF4F2881CB58D040207430E040E050E0FB
:1087800060E070E080E090E0A0E00E94318E31F186
:10879000809142248F93809141248F938091402433
:1087A0008F9380913F248F9382EB96E09F938F93DA
:1087B0001F9287E78F93C7010296A1E0B0E0AC0F4C
:1087C000BD1F8A0F9B1F9F938F930E941393E80EE8
:1087D000F91E0FB6F894DEBF0FBECDBFC557DF4FF1
:1087E0002881CB58D040207830E040E050E060E075
:1087F00070E080E090E0A0E00E94318E41F1F894BA
:108800008091E8289091E928A091EA28B091EB287E
:108810007894BF93AF939F938F9380EC96E09F9350
:108820008F931F9287E78F93C701029621E030E074
:108830002C0F3D1F820F931F9F938F930E941393C2
:10884000E80EF91E0FB6F894DEBF0FBECDBF20E0D4
:10885000C457DF4F3881CC58D040317040E050E0F1
:1088600060E070E080E090E0A0E00E94318E09F0CE
:1088700054C520E0C457DF4F3881CC58D040327007
:1088800040E050E060E070E080E090E0A0E00E9416
:10889000318E09F0B5C520E0C457DF4F3881CC5880
:1088A000D040347040E050E060E070E080E090E064
:1088B000A0E00E94318E09F0D4C520E0C457DF4FFC
:1088C0003881CC58D040387040E050E060E070E033
:1088D00080E090E0A0E00E94318E09F0F1C520E038
:1088E000C457DF4F3881CC58D040307140E050E061
:1088F00060E070E080E090E0A0E00E94318E09F03E
:1089000052C620E0C457DF4F3881CC58D040307277
:1089100040E050E060E070E080E090E0A0E00E9485
:10892000318E09F070C620E030E040E050E0C357DF
:10893000DF4F6881CD58D040647070E080E090E0F7
:10894000A0E00E94318E09F08CC620E0C057DF4FB6
:108950003881C059D04040E050E060E070E080E0F5
:1089600090E0A0E00E94318E09F0E8C620E0CA56EF
:10897000DF4F3881C659D04040E050E060E070E001
:1089800080E090E0A0E00E94318E09F005C720E071
:1089900030E0402F417050E060E070E080E090E017
:1089A000A0E00E94318E09F025C720E030E0402F82
:1089B000427050E060E070E080E090E0A0E00E9453
:1089C000318E09F04AC720E030E0C657DF4F4881BA
:1089D000CA58D04050E060E070E080E090E0A0E055
:1089E0000E94318E09F06CC720E030E0402F4870C3
:1089F00050E060E070E080E090E0A0E00E94318E06
:108A000009F088C720E030E0402F407150E060E07E
:108A100070E080E090E0A0E00E94318E09F0AAC7EB
:108A200020E030E0402F407250E060E070E080E0F5
:108A300090E0A0E00E94318E09F0CCC720E030E049
:108A4000402F407450E060E070E080E090E0A0E0F3
:108A50000E94318E09F0EFC7F02FF078BF2E20E092
:108A600030E04F2F50E060E070E080E090E0A0E068
:108A70000E94318E11F00C944C4D212F2170C22E8A
:108A800020E030E040E05C2D60E070E080E090E0CD
:108A9000A0E00E94318E11F00C94594D20E030E09E
:108AA0004B2D50E060E070E080E090E0A0E00E949C
:108AB000318E11F00C94674D20E030E040E05C2DE9
:108AC00060E070E080E090E0A0E00E94318E11F064
:108AD0000C949C4D20E030E040E0512F527060E05B
:108AE00070E080E090E0A0E00E94318E11F00C94E4
:108AF000D14D20E030E040E0512F547060E070E054
:108B000080E090E0A0E00E94318E11F00C94044EC1
:108B100020E030E040E0512F507160E070E080E0F4
:108B200090E0A0E00E94318E11F00C94374E20E0CE
:108B300030E040E0512F507260E070E080E090E063
:108B4000A0E00E94318E11F00C94764E20E030E0CF
:108B500040E0512F507460E070E080E090E0A0E0D1
:108B60000E94318E11F00C94B54E20E030E040E0D0
:108B7000512F587060E070E080E090E0A0E00E942B
:108B8000318E11F00C94F44E20E030E040E05D2D89
:108B900060E070E080E090E0A0E00E94318E11F093
:108BA0000C94254F779A8091C5099091C60992FD42
:108BB000749AC557DF4F2881CB58D040C457DF4F38
:108BC0003881CC58D040A801C357DF4F6881CD58B9
:108BD000D040CD56DF4F7881C359D040CC56DF4FBF
:108BE0008881C459D040CB56DF4F9881C559D040B9
:108BF000A0E08E010D5F1F4F0E94318E11F00C948A
:108C0000614F80915602806189838091E5098A8352
:108C1000F801EE0DFF1D10828091C5099091C609E3
:108C200087010D5F1F4F80FF0CC01F930F9387E5D7
:108C300098E09F938F930E94B0920F900F900F90A7
:108C40000F90B801CE0101960E94BA5B8091580244
:108C500082FF0AC028EE34E2A801BE016F5F7F4F99
:108C600081E692E00E944F608091C5099091C6090B
:108C700082FD73980E94E46781EF99E00E948D5213
:108C80008091580290915902A0915A02B0915B02D2
:108C900090FF40C03FEFE31AF30A0E94E268D82E2B
:108CA00089E10E94FA6840915802509159026091FE
:108CB0005A0270915B0250FF29C073988091E509B8
:108CC0008F5F8093E5098A83B7016F5F7F4FCE0185
:108CD00001960E94BA5B81EF99E00E948D5240E0BC
:108CE00050E065E880910212909103120E9448546E
:108CF00088E090E1CF56DF4FA881B981C159D040BB
:108D00008D939C9338C0E12CF12CCDCF8D2D0E94FA
:108D1000FA68739A8091C2099091C309892B11F066
:108D20000E949C678091E5098F5F8093E50980919F
:108D3000C5099091C60982FF39CC739A37CC8DED65
:108D400099E00E94EE56892BB1F00E94E467809171
:108D5000580287FD2B9860E470E08DED99E00E9449
:108D6000C75681E290E1CF56DF4FE881F981C159C2
:108D7000D0409183808381E00C94A64FCF56DF4F83
:108D8000A881B981C159D0401D921C9283E00C94F6
:108D9000A64F623181F7C0905802D0905902E090FE
:108DA0005A02F0905B02D1FC01CCF8018081813045
:108DB00091F50180F281E02D2081C557DF4F288396
:108DC000CB58D0403181C457DF4F3883CC58D04086
:108DD000028113814481C357DF4F4883CD58D0406F
:108DE0005581CD56DF4F5883C359D0408681CC562C
:108DF000DF4F8883C459D0409781CB56DF4F98838B
:108E0000C559D04020843184C257DF4F198218825F
:108E1000CE58D0406AC08230E9F4A381B481C257F1
:108E2000DF4FB983A883CE58D040212C312CB1E03C
:108E3000C557DF4FB883CB58D040C457DF4F188297
:108E4000CC58D04000E010E8C357DF4F1882CD580F
:108E5000D0403CC08330F9F0843009F0A7CB212CFE
:108E6000312CC257DF4F19821882CE58D040E5E02E
:108E7000C557DF4FE883CB58D040C457DF4F188227
:108E8000CC58D04000E010E0F2E0C357DF4FF88349
:108E9000CD58D0401BC0212C312CC257DF4F198236
:108EA0001882CE58D04025E0C557DF4F2883CB58D5
:108EB000D040C457DF4F1882CC58D04000E010E0BB
:108EC00031E0C357DF4F3883CD58D040CD56DF4F08
:108ED0001882C359D040CC56DF4F1882C459D040B5
:108EE000CB56DF4F1882C559D04080903F249090D8
:108EF0004024A0904124B0904224409080025090A1
:108F0000810260908202709083022DEC3CEC4CE474
:108F10005EE3C301B2010E94B6879B01AC01C501AB
:108F2000B4010E94428A87FD0BC0E894E0F8C09229
:108F30005802D0925902E0925A02F0925B024AC063
:108F4000A3019201C501B4010E947C8887FF42C041
:108F500080914B2490914C24A0914D24B0914E24AB
:108F60000196A11DB11D80934B2490934C24A09396
:108F70004D24B0934E24E0FC19CB6894E0F8C092E5
:108F80005802D0925902E0925A02F0925B0245E4F4
:108F9000C557DF4F4883CB58D04050E2C457DF4F0E
:108FA0005883CC58D04000E010E084E0C357DF4F36
:108FB0008883CD58D040CD56DF4F1882C359D0405A
:108FC000CC56DF4F1882C459D040CB56DF4F1882A1
:108FD000C559D040902F9470C657DF4F9883CA5818
:108FE000D04020E030E0492F50E060E070E080E0C9
:108FF00090E0A0E00E94318E09F08C9AC557DF4FB7
:10900000A881CB58D040A0727A2E2A2F30E040E0C1
:1090100050E060E070E080E090E0A0E00E94318EDF
:1090200011F00E94F50AC457DF4FB881CC58D040E8
:10903000B074C057DF4FB883C059D04020E03B2FF9
:1090400040E050E060E070E080E090E0A0E00E944E
:10905000318E11F00E94D01EC457DF4FE881CC58EA
:10906000D040E078CA56DF4FE883C659D04020E0B0
:109070003E2F40E050E060E070E080E090E0A0E053
:109080000E94318E51F00E94900A6093F5287093EF
:10909000F6288093F7289093F828C557DF4F28814A
:1090A000CB58D040217030E040E050E060E070E00C
:1090B00080E090E0A0E00E94318EF1F08EE09BE134
:1090C0009F938F938FE696E09F938F931F9287E7EE
:1090D0008F93CE0103969F938F930E9413936C01FD
:1090E0000E9453420FB6F894DEBF0FBECDBF892B4E
:1090F00009F05CCA760102C0E12CF12CC557DF4FA4
:109100002881CB58D040227030E040E050E060E051
:1091100070E080E090E0A0E00E94318ED1F1C701C4
:10912000029667E776E041E050E04C0F5D1F840F48
:10913000951F0E94149253E0E50EF11C22E0A22E2E
:1091400029E2B22E32EFC32E33E0D32E47E7942E1E
:10915000D5018D915D011F928F93DF92CF921F9267
:109160009F92C7010296E1E0F0E0EC0FFD1F8E0F29
:109170009F1F9F938F930E941393E80EF91E0FB6C3
:10918000F894DEBF0FBECDBF3AE0A31639E2B306B6
:10919000F9F6C557DF4F2881CB58D040247030E016
:1091A00040E050E060E070E080E090E0A0E00E94ED
:1091B000318E09F447C0C70102966BE776E041E0C3
:1091C00050E04C0F5D1F840F951F0E94149254E0D5
:1091D000E50EF11C4E018AE7880E911C80E1D40156
:1091E0001D928A95E9F728E0A40168E980EB0E94C6
:1091F0008F115401B8E0AB0EB11C82EFC82E83E092
:10920000D82E97E7692EF40181914F011F928F9319
:10921000DF92CF921F926F92C701029621E030E059
:109220002C0F3D1F820F931F9F938F930E941393C8
:10923000E80EF91E0FB6F894DEBF0FBECDBF8A143C
:109240009B0409F7512F5078D52E20E030E040E004
:1092500060E070E080E090E0A0E00E94318EE1F4F8
:109260008091C2099091C3099F938F9380E896E003
:109270009F938F931F9287E78F93CE018E0D9F1D33
:1092800003969F938F930E941393E80EF91E0FB6D7
:10929000F894DEBF0FBECDBF20E030E040E050E0EC
:1092A000C357DF4F6881CD58D040617070E080E0D7
:1092B00090E0A0E00E94318E09F487C9E3E0F0E07D
:1092C000EC0FFD1FEE0DFF1D80E28083EBE6F4E264
:1092D000808197012F5F3F4F7901882309F469C985
:1092E0008081A1E0B0E0AC0FBD1FAE0DBF1D129696
:1092F0008C933196EDCFCE018E0D9F1D67E876E001
:1093000003960E94149297E0E90EF11CC7010E9497
:109310005342892B09F04AC96AC92114310409F45E
:10932000A8CAF8944090E8285090E9286090EA286C
:109330007090EB2878948091781B9091791BA09184
:109340007A1BB0917B1BA3019201281B390B4A0B9E
:109350005B0BCA01B9010E941D894B015C01B1017F
:1093600080E090E00E941D899B01AC01C501B40121
:109370000E948088B82EC92E9F938F937F936F93FE
:109380008BEC96E09F938F931F9287E78F939E01BC
:109390002E0D3F1D2D5F3F4F3F932F93C856DF4F3C
:1093A0006883C859D040C956DF4F7883C759D04029
:1093B0000E941393E80EF91EC856DF4F6881C85902
:1093C000D040C956DF4F7881C759D040862F972F9C
:1093D000AB2DBC2D8093FA289093FB28A093FC28FA
:1093E000B093FD284092781B5092791B60927A1BB3
:1093F00070927B1B0FB6F894DEBF0FBECDBF39CA8B
:109400002114310409F447CAF89480914F1B9091BC
:10941000501BA091511BB091521B78949F938F9336
:1094200080915F028F9380915E028F9388ED96E02A
:109430009F938F931F9287E78F93C7010296A1E0B6
:10944000B0E0AC0FBD1F8A0F9B1F9F938F930E94AC
:109450001393E80EF91E0FB6F894DEBF0FBECDBF12
:109460001ACAF8948091EC289091ED28A091EE28EA
:10947000B091EF287894BF93AF939F938F9388EE2A
:1094800096E09F938F931F9287E78F93C701029671
:1094900021E030E02C0F3D1F820F931F9F938F938D
:1094A0000E941393E80EF91EC7010E9453420FB6A3
:1094B000F894DEBF0FBECDBF892B09F077C8FDC978
:1094C0002114310409F40BCAF8944090EC28509010
:1094D000ED286090EE287090EF28789480917C1BA6
:1094E00090917D1BA0917E1BB0917F1BA3019201E7
:1094F000281B390B4A0B5B0BCA01B9010E941D895D
:109500004B015C01B10180E090E00E941D899B014C
:10951000AC01C501B4010E948088B82EC92E9F936A
:109520008F937F936F9383EF96E09F938F931F9218
:1095300087E78F939E012E0D3F1D2D5F3F4F3F9379
:109540002F93C856DF4F6883C859D040C956DF4FA4
:109550007883C759D0400E941393E80EF91EC8566D
:10956000DF4F6881C859D040C956DF4F7881C7594D
:10957000D040862F972FAB2DBC2D8093FE28909343
:10958000FF28A0930029B093012940927C1B5092A0
:109590007D1B60927E1B70927F1B0FB6F894DEBF1E
:1095A0000FBECDBF9CC9232809F4ABC9F8948091A4
:1095B000531B9091541BA091551BB091561B78944E
:1095C0009F938F9380915D028F9380915C028F9324
:1095D00080E097E09F938F931F9287E78F93C70157
:1095E0000296A1E0B0E0AC0FBD1F8A0F9B1F9F93B6
:1095F0008F930E941393E80EF91E0FB6F894DEBF06
:109600000FBECDBF7EC98091432490914424A09188
:109610004524B0914624BF93AF939F938F9380E1ED
:1096200097E09F938F931F9287E78F93C7010296CE
:1096300021E030E02C0F3D1F820F931F9F938F93EB
:109640000E941393E80EF91EC7010E9453420FB601
:10965000F894DEBF0FBECDBF892B11F00C94D6421B
:1096600062C980914E248F9380914D248F93809175
:109670004C248F9380914B248F9380914A248F9315
:10968000809149248F93809148248F93809147241F
:109690008F938BE197E09F938F931F92B7E7CB2E29
:1096A000CF92C7010296A1E0B0E0AC0FBD1F8A0FB8
:1096B0009B1F9F938F930E941393E80EF91EC7017F
:1096C0000E9453420FB6F894DEBF0FBECDBF892B68
:1096D00011F00C94D64280913D2090913E2090FF55
:1096E00034C9809152248F93809151248F9380911B
:1096F00050248F9380914F248F938FE397E09F9313
:109700008F931F92CF92C701029621E030E02C0F79
:109710003D1F820F931F9F938F930E941393E80E18
:10972000F91EC7010E9453420FB6F894DEBF0FBE68
:10973000CDBF892B11F00C94D64207C98091341CFF
:109740008F938091331C8F938091321C8F938091E3
:10975000311C8F9381E597E09F938F931F9287E74A
:109760008F93C7010296A1E0B0E0AC0FBD1F8A0F36
:109770009B1F9F938F930E941393E80EF91EC701BE
:109780000E9453420FB6F894DEBF0FBECDBF892BA7
:1097900011F00C94D642EAC88091F8288F938091FA
:1097A000F7288F938091F6288F938091F5288F93D7
:1097B0008CE597E09F938F931F9287E78F93C70164
:1097C000029621E030E02C0F3D1F820F931F9F93E4
:1097D0008F930E941393E80EF91EC7010E94534213
:1097E0000FB6F894DEBF0FBECDBF892B11F00C94DD
:1097F000D642CDC881E00E94410A20917802309182
:10980000790240917A0250917B020E94018B9F93D2
:109810008F937F936F9389E697E09F938F931F9227
:1098200087E78F93C7010296A1E0B0E0AC0FBD1FA0
:109830008A0F9B1F9F938F930E941393E80EF91E2C
:10984000C7010E9453420FB6F894DEBF0FBECDBFD2
:10985000892B11F00C94D642A8C882E00E94410ADC
:1098600020917402309175024091760250917702F6
:109870000E94018B9F938F937F936F9386E797E06E
:109880009F938F931F9287E78F93C701029621E0E2
:1098900030E02C0F3D1F820F931F9F938F930E94E8
:1098A0001393E80EF91EC7010E9453420FB6F894B5
:1098B000DEBF0FBECDBF892B11F00C94D64283C8FA
:1098C00083E00E94410A9F938F937F936F9383E875
:1098D00097E09F938F931F9287E78F93C70102961C
:1098E000A1E0B0E0AC0FBD1F8A0F9B1F9F938F9329
:1098F0000E941393E80EF91E8C98C7010E945342F0
:109900000FB6F894DEBF0FBECDBF892B11F00C94BB
:10991000D6426AC880913D2087FF74C821E042E1A9
:1099200061E080ED0E9482619F938F937F936F939C
:1099300080E997E09F938F931F9287E78F93C701EA
:10994000029621E030E02C0F3D1F820F931F9F9362
:109950008F930E941393E80EF91EC7010E94534291
:109960000FB6F894DEBF0FBECDBF892B11F00C945B
:10997000D64248C880913D2087FF52C821E042E18D
:1099800062E080ED0E9482619F938F937F936F933B
:109990008EE997E09F938F931F9287E78F93C7017C
:1099A0000296A1E0B0E0AC0FBD1F8A0F9B1F9F93F2
:1099B0008F930E941393E80EF91EC7010E94534231
:1099C0000FB6F894DEBF0FBECDBF892B11F00C94FB
:1099D000D64226C880913D2087FF30C821E042E171
:1099E00063E080ED0E9482619F938F937F936F93DA
:1099F0008CEA97E09F938F931F9287E78F93C7011D
:109A0000029621E030E02C0F3D1F820F931F9F93A1
:109A10008F930E941393E80EF91EC7010E945342D0
:109A20000FB6F894DEBF0FBECDBF892B11F00C949A
:109A3000D6420C941E4580913D2087FF0DC821E041
:109A400042E164E080ED0E9482619F938F937F9357
:109A50006F938AEB97E09F938F931F9287E78F9383
:109A6000C7010296A1E0B0E0AC0FBD1F8A0F9B1F9B
:109A70009F938F930E941393E80EF91EC7010E94D3
:109A800053420FB6F894DEBF0FBECDBF892B11F045
:109A90000C94D6420C942C4580913D2082FD02C04E
:109AA0000C943D4546E061E083E00E944B130C942A
:109AB0003D4580913D2082FD02C00C944E4521E041
:109AC00046E061E083E00E944B130C944E45809188
:109AD0003D2082FD02C00C945C4580912B1C8F932D
:109AE00080912A1C8F938091291C8F938091281C30
:109AF0008F9388EC97E09F938F931F9287E78F93C4
:109B0000C701029641E050E04C0F5D1F840F951F86
:109B10009F938F930E941393E80EF91EC7010E9432
:109B200053420FB6F894DEBF0FBECDBF892B11F0A4
:109B30000C94D6420C945C4580913D2082FD02C07D
:109B40000C946A4580912F1C8F9380912E1C8F93CB
:109B500080912D1C8F9380912C1C8F9380ED97E02A
:109B60009F938F931F9287E78F93C7010296E1E03F
:109B7000F0E0EC0FFD1F8E0F9F1F9F938F930E94AD
:109B80001393E80EF91EC7010E9453420FB6F894D2
:109B9000DEBF0FBECDBF892B11F00C94D6420C94C2
:109BA0006A4580913D2090913E2090FD02C00C942A
:109BB000794580E090E00E94471E9F938F937F93AA
:109BC0006F938BED97E09F938F931F9287E78F930F
:109BD000C701029641E050E04C0F5D1F840F951FB6
:109BE0009F938F930E941393E80EF91EC7010E9462
:109BF00053420FB6F894DEBF0FBECDBF892B11F0D4
:109C00000C94D6420C94794580913D2090913E2051
:109C100090FD02C00C94884581E090E00E94471EB0
:109C20009F938F937F936F938BEE97E09F938F9388
:109C30001F9287E78F93C7010296E1E0F0E0EC0FF7
:109C4000FD1F8E0F9F1F9F938F930E941393E80E0B
:109C5000F91EC7010E9453420FB6F894DEBF0FBE33
:109C6000CDBF892B11F00C94D6420C94884580917D
:109C70003D2090913E2090FD02C00C94974581E0DC
:109C800090E00E94471E4B015C0180E090E00E9442
:109C9000471E9B01AC01C501B4010E94481C9F9363
:109CA0008F937F936F938CEF97E09F938F931F9287
:109CB00087E78F93C701029641E050E04C0F5D1F8C
:109CC000840F951F9F938F930E941393E80EF91EA4
:109CD000C7010E9453420FB6F894DEBF0FBECDBF3E
:109CE000892B11F00C94D6420C94974580913D201D
:109CF00090913E2090FD02C00C94A64581E090E03A
:109D00000E94471E4B015C0180E090E00E94471ECC
:109D10009B01AC01C501B4010E94A91C9F938F93C4
:109D20007F936F9387E098E09F938F931F9287E7CD
:109D30008F93C7010296E1E0F0E0EC0FFD1F8E0F5C
:109D40009F1F9F938F930E941393E80EF91EC701E4
:109D50000E9453420FB6F894DEBF0FBECDBF892BD1
:109D600011F00C94D6420C94A64580913D20909120
:109D70003E2090FD02C00C94B54581E090E00E9429
:109D8000471E4B015C0180E090E00E94471E9B0152
:109D9000AC01C501B4010E940A1D9F938F937F936C
:109DA0006F9385E198E09F938F931F9287E78F933E
:109DB000C701029641E050E04C0F5D1F840F951FD4
:109DC0009F938F930E941393E80EF91EC7010E9480
:109DD00053420FB6F894DEBF0FBECDBF892B11F0F2
:109DE0000C94D6420C94B54580913D2090913E2034
:109DF00091FD02C00C94C4450E9495179F938F93C8
:109E00007F936F9388E298E09F938F931F9287E7E9
:109E10008F93C7010296E1E0F0E0EC0FFD1F8E0F7B
:109E20009F1F9F938F930E941393E80EF91EC70103
:109E30000E9453420FB6F894DEBF0FBECDBF892BF0
:109E400011F00C94D6420C94C445C257DF4FA88140
:109E5000B981CE58D04016968C9116971F928F9349
:109E600015968C9115971F928F9313968C9113973B
:109E70001F928F9312968C911F928F9389E398E093
:109E80009F938F931F9287E78F93C7010296E1E01C
:109E9000F0E0EC0FFD1F8E0F9F1F9F938F930E948A
:109EA0001393E80EF91EC7010E9453420FB6F894AF
:109EB000DEBF0FBECDBF892B11F00C94D6420C949F
:109EC000D2458091C5099091C60982FD0CC0809150
:109ED000580280FD08C081FD02C00C9401461D9906
:109EE00002C00C9401461F930F9380E598E09F9366
:109EF0008F930E94B092809173020F900F900F90F9
:109F00000F90882311F40C9401461F928F938DEDCE
:109F10009EE09F938F930E94C2920F900F900F909C
:109F20000F900C9401468DED99E00E94EE56892B1E
:109F300011F40C94BB460E949C678091580287FDE7
:109F400002C00C94D6422B9A0C94D642C856DF4FCE
:109F50000FB6F894DEBF0FBECDBFDF91CF911F913A
:109F60000F91FF90EF90DF90CF90BF90AF909F90B8
:109F70008F907F906F905F904F903F902F900895BB
:109F80000C94B4524F925F926F927F928F929F92F5
:109F9000AF92BF92CF92DF92EF92FF920F931F93F7
:109FA000CF93DF93CDB7DEB760970FB6F894DEBFDF
:109FB0000FBECDBF6B010E94E268E82FF0E0EE0F0C
:109FC000FF1FEF5BF44E8081918101969183808326
:109FD0008091C5099091C60981FD749880905802BE
:109FE00090905902A0905A02B0905B020E940E5BC2
:109FF0007C01FC018081982F92959F70913099F49B
:10A000008F7051F48091251B9091261B019690939F
:10A01000261B8093251B07C1B60182E199E20E94AD
:10A020002A52892B51F08091231B9091241B019679
:10A030009093241B8093231BF6C0D501C4011EE01E
:10A04000B695A795979587951A95D1F7F82FF17042
:10A050008F2E8CEF99E00E9435558C01009709F402
:10A0600048C0B601C80102960E942A52892BE9F124
:10A07000980143E859E060E074E6C8010F960E9439
:10A08000B557F7019181F8018481981321C0828529
:10A090008F5F82878091211B9091221B0196909364
:10A0A000221B8093211B84E00E942B5CF8012085F9
:10A0B00030E02817390708F0A9C184E00E942B5C22
:10A0C000F8018087F70180818F70F8018187ABC02C
:10A0D000F801128684E00E942B5CF8018087F7016A
:10A0E00080818F70F801818792C1C8010E94DD557F
:10A0F000B4CF84E092E00E94CA548C01009709F426
:10A1000092C0B601C80102960E942152F7018181D6
:10A110008150F801848380E091E0A0E0B0E0838783
:10A120009487A587B687128684E00E942B5CF8018D
:10A130008087F70180818F70F8018187B8018CEFEB
:10A1400099E00E949555980143E859E060E074E673
:10A15000C8010F960E94B55799249394F701818105
:10A16000F8018483F70180818F70F801878384E090
:10A170000E942B5CF801858383E00E942B5C5C01CC
:10A18000F801868387818F3009F0912CF701418097
:10A19000F8018481481A512C612C712C76E0440C12
:10A1A000551C661C771C7A95D1F723853485458527
:10A1B0005685A0ECB0E00E94DF8BBB27A92F982F1B
:10A1C000872F480E591E6A1E7B1E4386548665865D
:10A1D00076868091C5099091C60981FD2EC0809137
:10A1E000580280FD2AC081FD26C0809158029091BE
:10A1F0005902A0915A02B0915B0297FDD2C09920FA
:10A2000091F082E0809354241092562410925524A9
:10A21000109358240093572444E554E262E184E308
:10A2200092E00E9448548091C5099091C60981FF2F
:10A23000F0C0749AEEC01D9BD8CFA4E6B0E0A30195
:10A2400092010E94DF8B672F782F892F992724E6B0
:10A2500030E040E050E00E942A8C7F936F93452CC1
:10A26000562C672C77245F924F92BB24BF92AF92FB
:10A27000F80185811F928F93F70180818F701F9263
:10A280008F9381811F928F93F60181811F928F930B
:10A2900080811F928F93C70102969F938F9388E6C8
:10A2A00098E09F938F930E94B092809173020FB6B3
:10A2B000F894DEBF0FBECDBF882361F01F928F934D
:10A2C0008AED9EE09F938F930E94C2920F900F9011
:10A2D0000F900F908091580290915902A0915A02CC
:10A2E000B0915B0296FF2DC0882059F1F7012081C3
:10A2F000322F3F70832F90E00297D4F08FEF830FBF
:10A30000207F822B808381EF99E00E94C04F809153
:10A310001F1B9091201B01969093201B80931F1B65
:10A320008091C5099091C60996FF0BC0739809C02A
:10A330008091251B9091261B01969093261B80935C
:10A34000251B80913D2086FF50CF0E94D160C70120
:10A3500005960E949D60F70181811F928F93F801FD
:10A3600086811F928F9385811F928F938CEA98E04C
:10A370009F938F931F9280E18F939E012F5F3F4F9A
:10A380006901DF922F930E94139382E00E94B760CD
:10A39000C6010E949D600FB6F894DEBF0FBECDBF10
:10A3A00024CF8EE09BE120910E1B222309F427CFBE
:10A3B0009F938F938FEB98E09F938F93FE0131963D
:10A3C0006F01DF92EF930E9450935C01B601C701C9
:10A3D00002960E9435920F900F900F900F900F9061
:10A3E0000F90009709F40BCF95012F5F3F4F280F77
:10A3F000391FA9012F5F3F4FFA0180818032C9F3D5
:10A4000062E18CE092E00E944854F9CE812C912CBC
:10A41000A5CE60960FB6F894DEBF0FBECDBFDF911C
:10A42000CF911F910F91FF90EF90DF90CF90BF9051
:10A43000AF909F908F907F906F905F904F90089516
:10A440000895FB012081FC012083FB012181FC0197
:10A4500021830895FC019081DB018C91981309C040
:10A4600081E090E0318111962C91321721F080E04B
:10A47000089580E090E00895BC0182E199E20C9497
:10A480002152DC011996ED91FC911A970280F3811B
:10A49000E02D309709F0099408950F931F93CF93FF
:10A4A000DF9300D0CDB7DEB78C0188E10E943E5C1F
:10A4B000BC01CE0101960E942152D8011996ED915E
:10A4C000FC911A970190F081E02DBE016F5F7F4FE4
:10A4D000C80109950F900F90DF91CF911F910F91B7
:10A4E0000895EF92FF920F931F93CF93DF93EC01A8
:10A4F0008B017A0142E053E00E949A52FA86E98683
:10A5000066E073E0C801DF91CF911F910F91FF903A
:10A51000EF900C94F3520C94B252CF93DF93EC0172
:10A5200062E179E288E10E94345CCE01DF91CF9153
:10A530000C94B452EF92FF920F931F93CF93DF933B
:10A54000EC018B017A010E94CF52F886EF826AE01B
:10A5500073E0C801DF91CF911F910F91FF90EF90B1
:10A560000C94F3520C94D7520C945E6DDC01179648
:10A57000ED91FC9118970190F081E02D0994DC0198
:10A580001796ED91FC9118970280F381E02D30979A
:10A5900009F00994089580E092E10C943155FC0192
:10A5A00073836283BC0180E092E10C949555BC01F9
:10A5B00080E092E10C947A55CF93DF93EC0180E038
:10A5C00092E10E943555009749F0FC0122813381C8
:10A5D0002C173D0729F00E94DD55F5CF80E090E073
:10A5E000DF91CF9108950F931F93CF93DF938B014A
:10A5F0000E94DC52EC01009731F01D830C83C801EE
:10A600000E948F6F8E83DF91CF911F910F910895DC
:10A610001F93CF93DF93EC01162FEC81FD813097D0
:10A62000D1F0909303128093021282E08887CE01CA
:10A6300006960995992787FD90950297029710F045
:10A64000133839F4BE01CE01DF91CF911F910C94E4
:10A65000355381E08887DF91CF911F910895FC01E8
:10A66000208520FD0C9408530895CF92DF92EF923D
:10A67000FF920F931F93CF93DF93EC016B01E09058
:10A680000212F09003120091041210910512F801C9
:10A69000EC17FD0739F0309709F44AC00190F081BA
:10A6A000E02DF6CF209709F443C08885882309F16F
:10A6B00018860115110561F0C017D10729F0AE0108
:10A6C00067E8C8010E942F53F80100811181F1CF82
:10A6D000EC81FD81309769F0CC15DD0551F0D09308
:10A6E0000312C093021240E050E063E8CE010696E8
:10A6F0000995E0910412F0910512CE17DF0769F475
:10A700008881998190930512809304120DC08081F5
:10A7100091818C179D0721F0FC013097C1F704C08F
:10A720008881998191838083F0920312E0920212D2
:10A73000DF91CF911F910F91FF90EF90DF90CF901D
:10A7400008951F93CF93DF9310920E12C0910412BD
:10A75000D091051211E0209779F08985882341F086
:10A760001887198640E050E062E8CE010E94085345
:10A770000990D881C02DEFCFDF91CF911F9108951F
:10A780008091B11291E0980F9093B1120895609169
:10A790000212709103120C9435538AE88093B1121F
:10A7A0001092AF121092B012109205121092041271
:10A7B0001092031210920212089580910E128111CC
:10A7C0000E94A1537091B012772309F451C0E09117
:10A7D000AF122E2F30E085E0E89FF0011124E15FF9
:10A7E000FD4E608160930D124181528150930C1295
:10A7F00040930B128381948190930A1280930912E3
:10A800002F5F3F4F2F7133272093AF1271507093FA
:10A81000B012009731F58091041290910512909337
:10A820000812809307128091071290910812892BC9
:10A83000F9F080910E1281110E94A15340910B12E8
:10A8400050910C1260910D12809107129091081294
:10A850000E942F53E0910712F0910812808191819C
:10A86000DECF613819F421E0FC0120870E942F53CC
:10A8700080910E122091B01290E0820F911D0895E8
:10A8800080910E122091B01290E0820F911D0895D8
:10A890002091B0122032B9F0E091AF12E20FEF71C7
:10A8A000E093061235E0E39FF0011124E15FFD4ED5
:10A8B000608352834183948383832F5F2093B012FC
:10A8C00080E090E0089581E090E00895CF93DF93D9
:10A8D000C0910212D09103120E942F53D093031201
:10A8E000C0930212DF91CF910895AB013091041211
:10A8F00020910512E32FF22FE817F907B1F03097F6
:10A9000021F00190F081E02DF7CF009771F0FC016C
:10A9100030832183909305128093041221E02087D5
:10A920001782168261E80C9466540895009749F0E6
:10A93000FC0120852150223020F421E02187209342
:10A940000E12089521E030E0FC018085811102C0E3
:10A9500020E030E0C9010895CF93DF93EC014A81F4
:10A960005B8160E070E08C819D810E9404922A816D
:10A970003B8188819981289FA001299F500D389F94
:10A98000500D112460E070E08E819F81DF91CF91A6
:10A990000C940492FC018281938120E030E028171E
:10A9A0003907D1F0A481B581A20FB31F4C91411199
:10A9B00010C081E08C9380819181289FA001299F04
:10A9C000500D389F500D112486819781840F951F5B
:10A9D00008952F5F3F4FE3CF80E090E00895FC01A2
:10A9E000268137814281538180E090E0841795076A
:10A9F000C9F02617370781F4A481B581A80FB91FC4
:10AA00002C91121614F421502C930480F581E02D22
:10AA1000E80FF91F80810895A081B1812A0F3B1FA3
:10AA20000196E4CF8FEF0895FC0186819781681726
:10AA30007907A0F0A081B18142815381A49F900148
:10AA4000A59F300DB49F300D1124280F391F81E0D0
:10AA500090E06217730720F080E0089580E090E0B6
:10AA60000895FC01118210820895FC01808191817A
:10AA70000895FB0120813181FC01318320830895F9
:10AA8000DC01ED91FC91309731F08081918100974C
:10AA900029F0FC01FACF80E090E00895CF010895FD
:10AAA000DC01ED91FC9111973097A9F02081318163
:10AAB000232B21F41D921C92CF010895A081B18116
:10AAC0008D919C911197892B11F0FD01F7CF118287
:10AAD0001082CD01089580E090E00895DC01ED91B1
:10AAE000FC911197309721F0208131812D933C9377
:10AAF000CF010895DC01ED91FC913097A9F0A0E021
:10AB0000B0E020813181E617F70741F4109709F48E
:10AB1000DC012D933C93118210820895211531059B
:10AB200019F0DF01F901EDCF08950F931F93CF9333
:10AB3000DF938C01EB010E947A5519821882C801BB
:10AB40000E944055009711F4F80101C0FC01D18327
:10AB5000C083DF91CF911F910F9108950F931F93A1
:10AB6000CF93DF93EC018B010E947A558881998104
:10AB7000F8019183808319830883DF91CF911F911E
:10AB80000F910895DC01ED91FC9180E090E0309709
:10AB900029F001960190F081E02DF9CF0895FB0195
:10ABA000309719F4BA010C94AE5580819181DA0185
:10ABB0008D939C93518340830895009721F0FC016D
:10ABC00080819181089580E090E008958091B41291
:10ABD0009091B512892B29F41092B3121092B212EF
:10ABE00008950E94E964E091B412F091B5122281B7
:10ABF000338140815181240F351F281B390B04807C
:10AC0000F581E02D309769F0428153816081718137
:10AC1000460F571F481B590B4217530780F79A01DD
:10AC2000EECF280F391F3093B3122093B21208953C
:10AC300086E892E00C949654EF92FF920F931F9344
:10AC4000CF93DF938C01FC0180819181009799F073
:10AC50008A359105D9F0F8011182108283E068C02D
:10AC6000868197818417950709F049C00480F58192
:10AC7000E02D3097A9F71092B5121092B4128AE520
:10AC800090E0F8019183808381E052C0673891F1B0
:10AC90006238A9F7C091B412D091B512E12CF12C11
:10ACA000209769F3CE010E946073892BF1F0AE0109
:10ACB00068E88E819F810E944854892BA1F41F82ED
:10ACC0001E828C819D81E114F10421F0F7019583AE
:10ACD000848304C09093B5128093B4121D821C82A9
:10ACE0000E94E655D7CF0E9418567E010C80DD8168
:10ACF000C02DD6CFE091B412F091B512BACFF09337
:10AD0000B512E093B412A481B581109709F4B7CFBE
:10AD100016968D919C9117978417950711F0FD0158
:10AD2000F2CF14968D919C91159795838483EBCFE8
:10AD3000DF91CF911F910F91FF90EF900895CF93E6
:10AD4000DF93EC010E9418568E819F813091B412DE
:10AD50002091B512892B59F0E32FF22F309739F05B
:10AD6000EC17FD0781F00480F581E02DF7CF80918D
:10AD70000212909103129F838E833C832D83D09384
:10AD8000B512C093B412DF91CF910C94E655CF93D6
:10AD9000DF93EC010E944073CE01DF91CF910C94C0
:10ADA0009F56CF93DF93EC010E944C73CE01DF914D
:10ADB000CF910C949F56CF93DF93EC010E94567372
:10ADC000CE01DF91CF910C949F56FC0120813181FF
:10ADD000260F371F318320830C94E65521E030E0A5
:10ADE000FC0186819781892B11F020E030E0C901B8
:10ADF0000895FC012281338180819181820F931F0C
:10AE00000895FC0180819181089581E090E0209176
:10AE1000B4123091B512232B11F480E090E0089524
:10AE20008091B4129091B512892B29F08091B212C1
:10AE30009091B312089580E090E00895CF93DF934E
:10AE4000EC01E091B412F091B5128E179F0769F4EE
:10AE50008C819D819093B5128093B4120DC0848132
:10AE600095818C179D0721F0FC013097C1F706C032
:10AE70008C819D81958384830E94E6551D821C826E
:10AE80001F821E82DF91CF910895EF92FF920F9360
:10AE90001F93CF93DF938C017A01FC018081918114
:10AEA000009741F08B34910501F1F8011182108275
:10AEB00083E048C087EB92E10E943555EC01209772
:10AEC00051F06C817D81CE0102960E94C756099097
:10AED000D881C02DF4CF81E08093B6128BE490E04E
:10AEE000F8019183808381E02DC06838E1F787EB1A
:10AEF00092E10E943555EC01209781F3CE01029634
:10AF0000E816F906D9F4BE0187EB92E10E947A5562
:10AF1000E0900212F09003128A859B8590930312B1
:10AF200080930212EC85FD85309719F08E859F8500
:10AF30000995F0920312E0920212D0CF0990D881C5
:10AF4000C02DDACFDF91CF911F910F91FF90EF903D
:10AF500008951092B61287EB92E10E94315560E09D
:10AF600070E080E992E00C9475540F931F93CF9397
:10AF7000DF93EC0100910212109103121B870A87E4
:10AF80005D874C873F872E878091B612882379F0A2
:10AF900080E992E09093031280930212CE01029610
:10AFA0000E94C756109303120093021202C07D83C1
:10AFB0006C83BE0187EB92E10E947A55BE0187EB5C
:10AFC00092E1DF91CF911F910F910C9495550F93C2
:10AFD0001F93CF93DF93EC018091B612882391F0F9
:10AFE000009102121091031280E992E090930312F3
:10AFF00080930212CE0102960E94D1561093031242
:10B0000000930212BE0187EB92E10E947A55BE01C5
:10B0100087EB92E1DF91CF911F910F910C949555A1
:10B020000F931F93CF93DF93EC018091B612882387
:10B0300091F0009102121091031280E992E0909336
:10B04000031280930212CE0102960E94DB561093E7
:10B05000031200930212BE0187EB92E10E947A551F
:10B06000BE0187EB92E1DF91CF911F910F910C947C
:10B070009555CF93DF93EC018091B612882329F088
:10B08000CE0102960E941E5704C01F821E8219869E
:10B090001886BE0187EB92E1DF91CF910C947A552F
:10B0A000CF93DF93EC018091B612882331F0CE016B
:10B0B0000296DF91CF910C94EE5687EB92E10E94BD
:10B0C0003555009739F08C179D0739F0FC018081C8
:10B0D0009181F7CF81E090E002C080E090E0DF91C5
:10B0E000CF9108952F923F924F925F926F927F92ED
:10B0F0008F929F92AF92BF92CF92DF92EF92FF9288
:10B100000F931F93CF93DF93CDB7DEB7E8970FB6BA
:10B11000F894DEBF0FBECDBFE9E4FBE220813181B0
:10B1200042815381E5E4FBE25080418032802380FC
:10B13000E1E4FBE28081898391819A83A281AB83E0
:10B140006380EDE3FBE2B081BC8381818D839281DA
:10B150009E83A381AF83E9E3FBE2B081B88781815D
:10B16000898792819A87A381AB87E5E3FBE2B0816F
:10B17000BC8781818D8792819E87A381AF87E1E320
:10B18000FBE2B081B88B8181898B92819A8BA381FC
:10B19000AB8BEDE2FBE2B081BC8B81818D8B928128
:10B1A0009E8BA381AF8BE9E2FBE2B081B88F8181F6
:10B1B000898F92819A8FA381AB8FE5E2FBE2B08108
:10B1C000BC8F81818D8F92819E8FA381AF8FE1E2B1
:10B1D000FBE2B081B8A3818189A392819AA3A38164
:10B1E000ABA3EDE1FBE2B081BCA381818DA3928191
:10B1F0009EA3A381AFA3E9E1FBE2B081B8A781815F
:10B2000089A792819AA7A381ABA7E5E1FBE2B08170
:10B21000BCA781818DA792819EA7A381AFA7E1E101
:10B22000FBE2B081B8AB818189AB92819AAB73802C
:10B23000EDE0FBE2B080A18092808380E9E0FBE258
:10B24000F080E180D280C380E5E0FBE2A081AFAB7B
:10B25000B181B8AF128103812BAB3CAB4DAB5EAB80
:10B260000E9417655EA95F934DA94F933CA93F9338
:10B270002BA92F932F923F924F925F926F922B8127
:10B280002F932A812F9329812F932F812F932E8102
:10B290002F932D812F932C812F932B852F932A85EC
:10B2A0002F9329852F9328852F932F852F932E85D4
:10B2B0002F932D852F932C852F932B892F932A89BC
:10B2C0002F9329892F9328892F932F892F932E89A4
:10B2D0002F932D892F932C892F932B8D2F932A8D8C
:10B2E0002F93298D2F93288D2F932F8D2F932E8D74
:10B2F0002F932D8D2F932C8D2F932BA12F932AA13C
:10B300002F9329A12F9328A12F932FA12F932EA103
:10B310002F932DA12F932CA12F932BA52F932AA5EB
:10B320002F9329A52F9328A52F932FA52F932EA5D3
:10B330002F932DA52F932CA52F937F922AA92F937E
:10B3400029A92F9328A92F938F929F92AF92BF92F2
:10B35000CF92DF92EF92FF920F931F9328AD2F931E
:10B360002FA92F939F938F937F936F93A3E1B9E2BC
:10B370008C911F928F93E2E1F9E280811F928F936B
:10B3800085E59FE09F938F930E94C292E9E7FBE2DD
:10B390002081318142815381E5E7FBE25080418089
:10B3A00032802380E9E6FBE29080818072806380B6
:10B3B000E5E6FBE28081898391819A83A281AB8358
:10B3C000B381BC83E1E6FBE280818D8391819E8322
:10B3D000A281AF83B381B887EDE5FBE280818987E5
:10B3E00091819A87A281AB87B381BC87E9E5FBE2B3
:10B3F00080818D8791819E87A281AF87B381B88B31
:10B40000E5E5FBE28081898B91819A8BB280A380F4
:10B41000E1E5FBE2F080E180D280C380EDE4FBE275
:10B42000A081AB8BB181BC8B128103810FB6F894E4
:10B43000DEBF0FBECDBF2BAB3CAB4DAB5EAB0E94B6
:10B4400017655EA95F934DA94F933CA93F932BA924
:10B450002F932F923F924F925F926F927F928F9293
:10B460009F922C812F932B812F932A812F932981B7
:10B470002F9328852F932F812F932E812F932D810A
:10B480002F932C852F932B852F932A852F932985F6
:10B490002F9328892F932F852F932E852F932D85DA
:10B4A0002F93AF92BF922A892F9329892F93CF92FE
:10B4B000DF92EF92FF920F931F932C892F932B898A
:10B4C0002F939F938F937F936F93A3E1B9E28C9116
:10B4D0001F928F93E2E1F9E280811F928F9386EEB3
:10B4E0009EE09F938F930E94C2920FB6F894DEBFA6
:10B4F0000FBECDBFE8960FB6F894DEBF0FBECDBF2E
:10B50000DF91CF911F910F91FF90EF90DF90CF903F
:10B51000BF90AF909F908F907F906F905F904F9073
:10B520003F902F90089580E380936D130895CF93FB
:10B53000DF9360916D1370E0C0E3D0E0C61BD70BC2
:10B5400065547D4EAE010E94FB91CE01DF91CF91FB
:10B550000895CF92DF92EF92FF920F931F93CF93B4
:10B56000DF937C01C0907013D090711360916D13C4
:10B5700070E0E601E096C61BD70BC138D105D8F4C0
:10B5800000E310E0061B170B65547D4EA8010E94D6
:10B59000FB916091B9127091BA1280916E139091E3
:10B5A0006F13680F791FA601C701800F911F0E94BA
:10B5B000FB91CE0102C080E090E0DF91CF911F911E
:10B5C0000F91FF90EF90DF90CF90089590916D13C1
:10B5D000980F90936D1308954091701350917113CB
:10B5E0004817590798F020916E1330916F13280F68
:10B5F000391F30936F1320936E13481B590B5093D0
:10B6000071134093701381E090E0089580E090E022
:10B6100008959093711380937013089580916E1321
:10B6200090916F1385519D4E089580916D1390E018
:10B6300085549D4E089581E090E02091B91230919B
:10B64000BA122B5E324111F480E090E008950E941E
:10B650001B5B892B61F06091B9127091BA12409115
:10B660007013509171138BEE92E10C94FB91209129
:10B670006E1330916F1321153105B9F0809170135D
:10B6800090917113C096EBEEF2E1AF014B5B52412A
:10B690004817590734F4DF01A20FB31F4C914193AF
:10B6A000F4CF10926F1310926E1308958091B91217
:10B6B0009091BA120895809170139091711308952A
:10B6C00090916D1380E3891B089520E380916D13A1
:10B6D000281B8091701390917113820F911D089512
:10B6E0001F93CF93DF93EC0110916D13812F90E0A6
:10B6F0008C179D076CF00E94655B8C0F9D1F813835
:10B70000910530F41C1B10936D1381E090E002C092
:10B7100080E090E0DF91CF911F910895CF93DF9368
:10B72000ECE1F9E21192119289E2EC34F807D1F7D9
:10B73000C4E1D9E260E073E0CE010E94215222967A
:10B7400089E2CC31D807B1F7DF91CF9108951092FB
:10B750006F1310926E13109271131092701380E396
:10B7600080936D138BEE92E19093BA128093B9128D
:10B770000C948E5BEF92FF920F931F93CF93DF9306
:10B7800000D0CDB7DEB78C0169837A830E94A75BB6
:10B790006981E62E7A81F72E81E8E816F10418F027
:10B7A00080E8E82EF12CA701B8018091B9129091A0
:10B7B000BA120E94FB91F0927113E0927013C701CC
:10B7C0000F900F90DF91CF911F910F91FF90EF900D
:10B7D00008950F931F93CF93DF938C01EB010E9489
:10B7E000A75B1093BA120093B912D0937113C09350
:10B7F0007013DF91CF911F910F91089520E3ECE139
:10B80000F9E2DC0101900D922A95E1F788E0E4E18C
:10B81000F9E2DB0101900D928A95E1F7089520E3AA
:10B82000FC01ACE1B9E201900D922A95E1F788E0C4
:10B83000FB01A4E1B9E201900D928A95E1F7089528
:10B84000E82FF0E0EE0FFF1FE45EF64D718360839A
:10B8500081E090E00895E82FF0E0EE0FFF1FE45E36
:10B86000F64D80819181089590E0880F991F8C5149
:10B87000974D0E94215281E090E0089590E0880F5A
:10B88000991F8C51974D08958115910511F00197DD
:10B89000F1F70895E0914F29F0915029908180911E
:10B8A0004E2989230895E0914C29F0914D298081FA
:10B8B00090914E29892B8083E0915129F091522952
:10B8C000808190914E29892B80830895E0914C29A5
:10B8D000F0914D29908180914E2980958923808314
:10B8E000E0915129F0915229908180914E298095C3
:10B8F0008923808308951F93CF93DF93E0914C2990
:10B90000F0914D29908180914E29809589238083E3
:10B91000E0915129F0915229808190914E29892BF3
:10B9200080838FEB93E00E94445C1FB7F894E09112
:10B930005129F0915229908180914E298095892337
:10B94000808383E890E00E94445CE0914F29F0916D
:10B950005029D081C0914E291FBF78948BE393E08A
:10B960000E94445CE0914F29F09150299081809190
:10B970004E29982319F08D2F8C2301C081E0DF918F
:10B98000CF911F910895509352294093512970935C
:10B990004D2960934C299093502980934F2981E041
:10B9A00001C0880F2A95EAF780934E290C947B5C9E
:10B9B000CF93DF93C82FDFB7F894E0915129F0912E
:10B9C0005229808190914E29892B808383E090E0D9
:10B9D0000E94445CCC2351F0E0915129F09152290E
:10B9E000808190914E2990959823908387E190E0F3
:10B9F0000E94445CE0914F29F09150298081909100
:10BA00004E29892309F4C0E089E590E00E94445C56
:10BA1000E0915129F0915229808190914E29909581
:10BA200098239083DFBF8BE390E00E94445C8C2FCF
:10BA3000DF91CF910895CF93DF93C82FD8E08C2F5B
:10BA400081700E94D85CC6958111C068D150B9F749
:10BA50008C2FDF91CF9108958FEF0C941B5DDF92B7
:10BA6000EF92FF920F931F93CF93DF93E82EEB019A
:10BA70000E947B5C81112FC080EF0E941B5DF12C26
:10BA800010E488EFD82ED10E81E00E94D85C082FF8
:10BA900081E00E94D85C882319F0002361F01DC06A
:10BAA000011109C01E1528F0888180FF04C0E1162D
:10BAB00011F0F12E01E0802F0E94D85C98819695BC
:10BAC00001119068988311501D11DECF219611113C
:10BAD000D8CF8F2D03C08FEF01C08EEFDF91CF91B4
:10BAE0001F910F91FF90EF90DF900895FF920F93B9
:10BAF0001F93CF93DF93F82EEB010E947B5C20977E
:10BB000069F085E50E941B5D8E01085F1F4F8991DA
:10BB10000E941B5DC017D107D1F703C08CEC0E94B7
:10BB20001B5D8F2DDF91CF911F910F91FF900C9492
:10BB30001B5D0F931F93CF93DF93DB01EC91119665
:10BB40009C911197F0E0F92B803181F4BF016E7F59
:10BB5000E3E0660F771FEA95E1F716969C9116973A
:10BB6000ECE0F0E0E91BF109E60FF71FF7FF07C073
:10BB700091E0EA019883F195E195F10902C0EA01AB
:10BB80001882883279F414968C91982F907690369A
:10BB900049F086FF02C0EE7F05C085FF02C0EC7F42
:10BBA00001C0E87FCF0144E0969587954A95E1F77B
:10BBB000D9018C93EF70E801E88380E0DF91CF91A9
:10BBC0001F910F9108950F931F93CF93DF93EC0173
:10BBD0008B01B80188810E942F5D888381508D3F41
:10BBE00030F4F8018081883211F0803191F7DF91D3
:10BBF000CF911F910F910895CF93DF93EC010E9495
:10BC00007B5CBE0184EB0E94765D81E00E94D85C83
:10BC1000C82F0E947B5C81E0C11101C080E0DF91F0
:10BC2000CF9108951F93CF93DF9300D0CDB7DEB7A8
:10BC3000182F69837A830E947B5C0E944A5C698129
:10BC40007A81882341F084E40E94765D113029F0E6
:10BC50000E94535C02C082E001C080E00F900F9010
:10BC6000DF91CF911F9108954F925F926F927F92D3
:10BC70008F929F92AF92BF92CF92DF92EF92FF92FC
:10BC80000F931F93CF93DF93CDB7DEB729970FB6EE
:10BC9000F894DEBF0FBECDBF6C015B014A01890184
:10BCA0000E947B5CB6018EEB0E94765DCE01019610
:10BCB0007C013E019AE0690E711C27010E942C5DF7
:10BCC000F70181937F01E615F705C1F769E070E0A0
:10BCD000C2010E94D177811109C09401A501B2016E
:10BCE000F60180810E94995D80E001C083E0299681
:10BCF0000FB6F894DEBF0FBECDBFDF91CF911F917D
:10BD00000F91FF90EF90DF90CF90BF90AF909F90FA
:10BD10008F907F906F905F904F9008955F926F9299
:10BD20007F928F929F92AF92BF92CF92DF92EF92CB
:10BD3000FF920F931F93CF93DF93CDB7DEB7299771
:10BD40000FB6F894DEBF0FBECDBF582E6B015A015F
:10BD5000890160E070E08EEB0E94765DCE01019675
:10BD60007C014E019AE0890E911C37010E942C5DE6
:10BD7000F70181937F01E815F905C1F769E070E0EB
:10BD8000C3010E94D177811108C09501A601B301BA
:10BD9000852D0E94995D80E001C083E029960FB651
:10BDA000F894DEBF0FBECDBFDF91CF911F910F91F1
:10BDB000FF90EF90DF90CF90BF90AF909F908F90CB
:10BDC0007F906F905F9008950F931F93CF93DF93B1
:10BDD000CDB7DEB728970FB6F894DEBF0FBECDBF44
:10BDE000182F062F98E0ECE0F3E0DE0111960190A9
:10BDF0000D929A95E1F7242F332727FD309541E7DF
:10BE000052E0249FC001259F900D349F900D112476
:10BE100064E670E00E94168CCB0144E6049F800D1E
:10BE2000911D1124FE013196AE01475F5F4F619174
:10BE300070E02617370711F4019603C0E417F507E1
:10BE4000B1F7112319F091958195910928960FB6B4
:10BE5000F894DEBF0FBECDBFDF91CF911F910F9140
:10BE60000895EF92FF920F931F93CF93DF93CDB777
:10BE7000DEB72B970FB6F894DEBF0FBECDBFF82EFE
:10BE8000E92E682F792F88E08F0D0E94125E88239B
:10BE900019F084E391E243C066E471E48FE090E03E
:10BEA0000E949C5F8E01075F1F4F9801AE01465FA5
:10BEB0005F4FBE01655F7F4F8F2D9E2D0E94345EC8
:10BEC0008111E7CF88E0ECE0F3E0DE01119601900C
:10BED0000D928A95E1F7498521E732E0429FC00142
:10BEE000439F900D112464E670E00E94168C8A85B1
:10BEF00094E6899F600D711D1124FE013196819198
:10BF0000481303C06F5F7F4F03C0E017F107B9F715
:10BF10008B85882319F0719561957109CB012B965A
:10BF20000FB6F894DEBF0FBECDBFDF91CF911F914A
:10BF30000F91FF90EF900895DC01CB0181159105E1
:10BF4000A105B10529F081509040A040B040D9F73B
:10BF500008959B01AC011092B90060E072E18AE79C
:10BF600090E00E942A8C20513109410951095695CF
:10BF70004795379527952093B800089594EA9093B4
:10BF8000BC0040EA56E861E070E09091BC0097FD8B
:10BF90000BC04150510961097109411551056105F5
:10BFA000710599F781E008959091B900987F9830D4
:10BFB00011F09031B9F78093BB0084E88093BC0006
:10BFC00080EA96E8A1E0B0E02091BC0027FD08C01F
:10BFD0000197A109B1090097A105B105A9F7E2CF21
:10BFE0008091B900887F883111F08034D9F680E0E3
:10BFF000089524EA34E844E92093BC009091BC0001
:10C0000097FFFCCF9091B900987F983011F0903154
:10C0100099F78093BB003093BC009091BC0097FFD0
:10C02000FCCF9091B900987F903211F0983539F497
:10C030004093BC009091BC0094FDFCCFDDCF0895EF
:10C040000C94BE5F84E98093BC008091BC0084FDA9
:10C05000FCCF08958093BB0084E88093BC0080915E
:10C06000BC0087FFFCCF9091B900987F81E09832A7
:10C0700009F480E0089584EC8093BC008091BC00BA
:10C0800087FFFCCF8091BB00089584E88093BC00BB
:10C090008091BC0087FFFCCF8091BB000895E0E158
:10C0A000DC01FD91CD01F0933F01E150C9F7809192
:10C0B0003C018F7D80933C0180913C01877F809380
:10C0C0003C01FB0180E1919190933E018150D9F7B1
:10C0D00080913C01806880933C0180913D0180FF0C
:10C0E000FCCF4051510980913C01806280933C011A
:10C0F00080913C01877F80933C01141615069CF4C7
:10C10000FB0180E1919190933E018150D9F780919C
:10C110003C01806880933C0180913D0180FFFCCF11
:10C1200040515109EACFF90180E190913E0191938C
:10C130008150D9F781E090E008950F931F93CF933A
:10C14000DF93EC018CE70E94F95F8CE70E942A6084
:10C150008E01005F1F4F89910E942A60C017D1078E
:10C16000D1F7DF91CF911F910F910C942260813014
:10C1700019F440E050E002C040EC50E060E070E0B4
:10C180008CE790E00C947811813019F44EE050E087
:10C1900002C048E050E060E070E08CE790E00C9472
:10C1A000781141E050E060E070E08CE790E00E94A0
:10C1B00078116AE67AE080E090E00C949C5F48E3B6
:10C1C00050E060E070E08CE790E00E94781149E375
:10C1D00050E060E070E08CE790E00E94781144E16C
:10C1E00050E060E070E08CE790E00E94781148E752
:10C1F00050E060E070E08CE790E00E9478114EE53E
:10C2000050E060E070E08CE790E00E9478114DE62D
:10C2100050E060E070E08CE790E00E9478116CE103
:10C220007AE186E090E00E949C5F4CE050E060E0A4
:10C2300070E08CE790E00E94781141E050E060E00F
:10C2400070E08CE790E00E94781146E050E060E0FA
:10C2500070E08CE790E00E9478116AE67AE080E076
:10C2600090E00C949C5FCF93DF93CDB7DEB7A2979D
:10C270000FB6F894DEBF0FBECDBF81E1E0E4F9E078
:10C28000DE01529601900D928A95E1F781E1E1E598
:10C29000F9E0DE01119601900D928A95E1F70E9476
:10C2A000DF60CE0142960E949D6082E00E94B760EE
:10C2B0006AE67AE080E090E00E949C5FCE01019601
:10C2C0000E949D6060E17EEA88E290E00E949C5FAF
:10C2D00080E00E94C46060E17EEA88E290E00E9413
:10C2E0009C5F4EE050E060E070E08CE790E00E94E0
:10C2F0007811A2960FB6F894DEBF0FBECDBFDF91C6
:10C30000CF910895CF92DF92EF92FF920F931F93F8
:10C31000CF93DF9300D01F92CDB7DEB7F82E042F56
:10C32000122F213031F0223031F0243031F028301A
:10C3300031F090E005C091E003C092E001C093E0CD
:10C340000C3059F00E3011F4946007C0003111F434
:10C35000986003C0023109F49C60613059F062308A
:10C3600011F4906207C0633011F4906403C064302C
:10C3700009F490669068692F70E023E030E0AE0128
:10C380004F5F5F4F8F2D90E00E948F1169E07AE13F
:10C3900080E090E00E949C5F8F2D8160F82E0E94CB
:10C3A000BE5F0E943B6089830E943B608A830231AA
:10C3B00019F40E943B608B830E943B6087FDF1CFA4
:10C3C0000E9445600E94226069E07AE180E090E08E
:10C3D0000E949C5F8F2D0E94BE5F0E943B608983FC
:10C3E0000E943B608A83023119F40E9445608B836E
:10C3F0000E9445600E94226039812A81023149F5FC
:10C40000832F90E0A0E0B0E04B817727662731FFD3
:10C410000EC030E0322F2227620F731F811D911D45
:10C42000640F711D811D911D8C6F9F6F0BC030E0DB
:10C43000322F2227620F731F811D911D640F711D02
:10C44000811D911D0E941F8920E83FEF4FEF57E4A7
:10C4500020C0632F70E0762F6627620F711D88273A
:10C4600077FD8095982F0E941F890C3029F420E0D9
:10C4700030EE4FEF54E40DC00E3029F420E038EFD9
:10C480004FEF55E406C0003131F420E03EEF4FEFAE
:10C4900056E40E9480882FE632E143E050E40E9497
:10C4A000018B6B017C01612F70E080E090E00E94C5
:10C4B0001F899B01AC01C701B6010E9480880F90C3
:10C4C0000F900F90DF91CF911F910F91FF90EF9000
:10C4D000DF90CF900895E6E4F1E0808120819081A3
:10C4E0003081829586958695837022952F70822B58
:10C4F000832B92959F70892B08950F931F93CF9351
:10C50000DF9300D0CDB7DEB746E06CE080E00E945C
:10C51000AD6589E18093C4001092C50082E08093EC
:10C52000C00080E00E9438660E94D96484B784B756
:10C5300084B784B784B7E3EDF1E322E432E43183D6
:10C5400020833A968DB79EB70A97E817F907B8F394
:10C5500082E699E09F938F9382EA90E19F938F9375
:10C560000E94C2920E9414740E94CD5360E070E059
:10C5700086E892E00E9475540E94A957E091140346
:10C58000F091150309950E946B6290E00E9450742F
:10C59000CE0101960E940E640F900F900F900F90A5
:10C5A000882341F082E890E19F938F930E94C2928A
:10C5B0000F900F90CE0101960E943C520E941C6485
:10C5C0008C010E941864AE014F5F5F4FB8010E945A
:10C5D00004690E9488630E94E5680E9420640E94AA
:10C5E0003E6A85E790E19F938F930E94C2928A8171
:10C5F0001F928F9301E710E11F930F930E94C29245
:10C6000089811F928F931F930F930E94C2928FE68E
:10C6100090E19F938F930E94C2920E945474E09184
:10C620005103F09152030995E0914303F0914403C3
:10C630000995E0912A03F0912B0309950E94456A20
:10C64000182F0E94E2681F921F931F928F93809170
:10C6500050038F9380914F038F93809142038F9368
:10C66000809141038F9384E590E19F938F930E9483
:10C67000C292E0915B03F0915C030FB6F894DEBFC9
:10C680000FBECDBF309791F00995BC0180E890E0D6
:10C690000E94028C7F936F9381E490E19F938F932C
:10C6A0000E94C2920F900F900F900F908FE390E135
:10C6B0009F938F930E94C29260E070E08CED92E0B5
:10C6C0000E94755480EF92E00E94247387E390E10A
:10C6D0009F938F930E94C2920F900F900F900F9094
:10C6E0000F900F90DF91CF911F910F9108957F933D
:10C6F0006F939F938F9381E390E19F938F930E9419
:10C70000C2920F900F900F900F900F900F9008957E
:10C710001F93CF93DF93CDB7DEB7A0970FB6F894F2
:10C72000DEBF0FBECDBF8DE590E00E942E94182F86
:10C73000282F35EF380F303108F0982F90952917B2
:10C7400009F461C08DEB90E19F938F930E94C29298
:10C75000E2E0F1E10F900F90DE01119684918D934C
:10C76000319681E1EA30F807C9F7F89448E050E0E3
:10C7700069E770E0CE0101960E943494E4EFF0E1A5
:10C78000DE01119684918D93319681E1E230F807B4
:10C79000C9F74EE050E06BE670E0CE0101960E94D2
:10C7A0003494EAEEF0E1DE01119684918D93319696
:10C7B00080E1E43FF807C9F74AE050E061E670E045
:10C7C000CE0101960E9434946DEC7BEA8BE590E0FB
:10C7D0000E944C9460E070E089E590E00E944C94E7
:10C7E00060E088E590E00E943E9460E070E08FE5B4
:10C7F00090E00E944C941AE16AE175EE8DE590E0BC
:10C800000E944C947894812FA0960FB6F894DEBFC6
:10C810000FBECDBFDF91CF911F910895F89442E0F4
:10C8200050E069E770E00E941694789480E00895E3
:10C830008BE590E00C942E9489E590E00C942E9476
:10C8400088E590E00C9426944091612950916229EA
:10C85000609163297091642990E0A0E0B0E0480FF6
:10C86000591F6A1F7B1F409361295093622960936F
:10C8700063297093642940915D2950915E296091EC
:10C880005F2970916029480F591F6A1F7B1F4093D1
:10C890005D2950935E2960935F29709360292091F0
:10C8A000012B2223A1F04091592950915A296091DE
:10C8B0005B2970915C29480F591F6A1F7B1F4093A9
:10C8C000592950935A2960935B2970935C290895E4
:10C8D0001F920F920FB60F9211240BB60F922F9347
:10C8E0003F934F935F936F937F938F939F93AF93F8
:10C8F000BF93EF93FF9380917413909175130196FA
:10C900009093751380937413809173138F5F80934A
:10C9100073138038A9F41092731380916129909158
:10C920006229A0916329B09164290196A11DB11DCE
:10C930008093612990936229A0936329B09364291D
:10C940008091012B8823E1F0809172138F5F809397
:10C9500072138038A9F41092721380915929909122
:10C960005A29A0915B29B0915C290196A11DB11DA6
:10C970008093592990935A29A0935B29B0935C29FD
:10C980000E940557892B11F00E941856FF91EF91D4
:10C99000BF91AF919F918F917F916F915F914F91D7
:10C9A0003F912F910F900BBE0F900FBE0F901F90D5
:10C9B0001895F8941092B60016BC83EF87BD82E0FC
:10C9C00084BD94E095BD95B395BB80936E0078943B
:10C9D0000895809174139091751320917413309180
:10C9E000751382179307A9F70895009751F022E372
:10C9F00030E000002150310921153105D1F70197B0
:10CA0000F4CF08950F931F93CF93DF93EC010E940F
:10CA1000E9648C010E94E964801B910B8C179D07CF
:10CA2000C8F3DF91CF911F910F91089508950F934F
:10CA30001F9360916129709162298091632990917F
:10CA40006429009161291091622920916329309114
:10CA50006429601771078207930759F71F910F9197
:10CA600008951F920F920FB60F9211241092B202E6
:10CA70000F900FBE0F901F9018951F920F920FB638
:10CA80000F9211240BB60F922F933F934F935F9306
:10CA90006F937F938F939F93AF93BF93EF93FF9386
:10CAA000E091A802F091A9028081E091B302F09197
:10CAB000B402309709F00995FF91EF91BF91AF91C2
:10CAC0009F918F917F916F915F914F913F912F91A6
:10CAD0000F900BBE0F900FBE0F901F9018951F92D6
:10CAE0000F920FB60F9211241092BF020F900FBE3B
:10CAF0000F901F9018951F920F920FB60F9211244E
:10CB00000BB60F922F933F934F935F936F937F9347
:10CB10008F939F93AF93BF93EF93FF93E091B502F1
:10CB2000F091B6028081E091C002F091C10230978D
:10CB300009F00995FF91EF91BF91AF919F918F916E
:10CB40007F916F915F914F913F912F910F900BBE0D
:10CB50000F900FBE0F901F9018959DE0899FF001D8
:10CB60001124E855FD4FA281B3811C92A481B581A7
:10CB70006C93A681B78188ED8C93A085B1854C9389
:10CB800012861486138608959DE0899FF001112472
:10CB9000E855FD4F81E08287A081B1816C933A9680
:10CBA00080818111FDCF08951F93CF93DF93182FBC
:10CBB000EB01FE016491662329F0812F0E94C46578
:10CBC0002196F7CFDF91CF911F9108951F93CF93B7
:10CBD000DF93182FEB018881882369F08A3021F4D4
:10CBE0006DE0812F0E94C46569916D30A1F3812FA2
:10CBF0000E94C465F0CFDF91CF911F910895CF932C
:10CC0000DF93CDB7DEB79E01285F3F4F4E815F8136
:10CC100060E470E086E793E10E947F9366E773E14A
:10CC20008D810E94E665DF91CF910895CF93C82F43
:10CC30008A3031F46DE08091B6130E94C46502C061
:10CC40008D3029F06C2F8091B6130E94C46580E06E
:10CC500090E0CF9108959DE0899FF0011124E8555F
:10CC6000FD4F748763870895682F80E00C94C46536
:10CC70008093B6138AE992E09093CE318093CD31C0
:10CC8000089584B7877F84BF88E10FB6F8948093B6
:10CC90006000109260000FBE08952FE088E190E0E0
:10CCA0000FB6F894A895809360000FBE20936000A3
:10CCB0000895A895089588E10FB6F89480936000D0
:10CCC000109260000FBE0895F89428E088E190E08B
:10CCD0000FB6F894A895809360000FBE2093600073
:10CCE000FFCF80916C2980916C2990E0089540E0FD
:10CCF0006FE181E491E00C94DA6BE9E3F1E080818B
:10CD000080818D7F80838DE090E00197F1F723E0B3
:10CD100040E06FE182E491E00E94E46B83E090E008
:10CD20000197F1F708959091390191FD0AC0282FDC
:10CD3000803108F02FE040E06FE085E491E00C9452
:10CD4000E46B08958091390181FD0EC040E06FE1F0
:10CD500081E491E00E94DA6B282F2F7E81E090E041
:10CD6000213021F080E0089580E090E008958091E6
:10CD7000390181FD10C040E06FE181E491E00E9443
:10CD8000DA6B8F3131F0982F9F7E915081E0923095
:10CD900018F480E0089581E008950E94B766882322
:10CDA000E1F30895CF93DF93C82F0E94CD660E94D0
:10CDB0007766D82FC81789F1C83019F40E947D66AC
:10CDC00025C0C93121F4863189F429E005C0C63176
:10CDD00069F4893159F426E040E06FE182E491E0A2
:10CDE0000E94E46BE3E0F0E03197F1F72C2F40E094
:10CDF0006FE182E491E00E94E46BD83019F4E9E637
:10CE0000F1E002C0E3E0F0E03197F1F70E947766CD
:10CE10008C1719F083E490E002C080E490E0DF9189
:10CE2000CF9108950E94CD661092012B0E947D66DD
:10CE3000809139018260809339018091842B88230D
:10CE4000D9F180919400909195004091952B50914B
:10CE5000962B84179507A0F48091612B9091622BFB
:10CE6000A091632BB091642B8C57914EAF4FBF4F65
:10CE70008093612B9093622BA093632BB093642BD0
:10CE80002091940030919500241B350B8091612BEB
:10CE90009091622BA091632BB091642B820F931F12
:10CEA000A11DB11D8093612B9093622BA093632BE6
:10CEB000B093642B1092842B8091862B8823D9F118
:10CEC00080919400909195004091992B50919A2BCC
:10CED00084179507A0F48091692B90916A2BA091FB
:10CEE0006B2BB0916C2B8C57914EAF4FBF4F8093F3
:10CEF000692B90936A2BA0936B2BB0936C2B209192
:10CF0000940030919500241B350B8091692B9091F2
:10CF10006A2BA0916B2BB0916C2B820F931FA11DDC
:10CF2000B11D8093692B90936A2BA0936B2BB093C8
:10CF30006C2B1092862B08958091012B882381F011
:10CF400080913A14811104C00E94B766811106C015
:10CF500081E08093381481E090E008950E94126788
:10CF600080E090E0089580919400909195009093D6
:10CF70009A2B8093992B21E02093862B8091390165
:10CF800081FD08C08091390181FD1AC086E10E94AF
:10CF9000D26616C02093002B80919400909195004A
:10CFA0009093962B8093952B2093842B809139011D
:10CFB0008D7F809339018091002B8111FCCFE2CFCE
:10CFC00081E08093012B08958091012B81110AC08B
:10CFD00080913A14882321F081E08093391402C0B3
:10CFE0000E94B36781E090E008951F93CF93DF9391
:10CFF0001F92CDB7DEB78FB7898380913A14811124
:10D0000026C0F8948091012B882351F0809139013A
:10D0100081FD1BC00E94B7668823B9F080E003C081
:10D020000E94E46781E02091470191E02E3008F0F2
:10D0300090E0192F119581110E949C67107429F0BE
:10D0400089818FBF81E090E004C089818FBF80E03B
:10D0500090E00F90DF91CF911F9108958091391446
:10D06000882321F00E94B3671092391480913814FC
:10D07000882321F00E9412671092381410923A14FB
:10D0800008950F931F93AB0121E020933A14009170
:10D09000452B1091462B2091472B3091482B0F5F49
:10D0A0001F4F2F4F3F4F0093452B1093462B20933C
:10D0B000472B3093482B22E0260F27FF0CC080918E
:10D0C000FE2A9091FF2A01969093FF2A8093FE2AD0
:10D0D0000FEF1FEF07C0BC0187EB93E10E94FB91AC
:10D0E00000E010E00E942E68C8011F910F91089582
:10D0F00080933C1408950E947766823011F082314B
:10D1000011F480E0089581E0089508958FEF8093F1
:10D110004E0122E044E060EF8CE691E00E94E46B77
:10D1200025E041E06EE08CE290E00E94E46B80E854
:10D1300080936F018091460180936D0121E045E06D
:10D1400060E284E491E00C94E46B8DEF93E001974E
:10D15000F1F70E94D06B109275291092F729109266
:10D16000792A1092742910927329E9E3F1E0808101
:10D170008E7F808380818D7F80838DE090E001971A
:10D18000F1F7E9E3F1E080818160808323E040E012
:10D190006FE182E491E00E94E46B8DEF93E00197F0
:10D1A000F1F780915D0180915E010E94866860E0E8
:10D1B00070E082EC92E00E9475540E94B36781E0B7
:10D1C00090E0089580913B140895CF93DF931F92D0
:10D1D000CDB7DEB789830E94CD66898180933B14E9
:10D1E000282F40E06FE188E491E00F90DF91CF912C
:10D1F0000C94E46B0E94E5688091390181FD03C0C5
:10D2000086E00C94D2660895FA01809362019093AF
:10D21000630160936001709361013097C1F0808178
:10D2200080936B01818180936A018281809369017F
:10D2300083818093680184818093670185818093D5
:10D2400066018681809365018781809364010895DA
:10D2500082EC92E00E94965481E080936C29809148
:10D260006D2990916E29019690936E2980936D2976
:10D2700081E090E008958091742992E8899FF001FF
:10D280001124EB58F64D10828F5F833018F4809391
:10D29000742902C010927429E091742982E8E89FF1
:10D2A000F0011124EB58F64D808181110C9428690E
:10D2B00010926C2908951F93CF93DF9320917429C6
:10D2C00012E8129F90011124D901AB58B64D4C9130
:10D2D000411103C00E943B6993C05091390151FD37
:10D2E0008FC05091012B552309F48AC047FF16C007
:10D2F0000E943B698091352B9091362BA091372B62
:10D30000B091382B0196A11DB11D8093352B9093C0
:10D31000362BA093372BB093382B72C04330B0F428
:10D320000E943B698091312B9091322BA091332B3D
:10D33000B091342B0196A11DB11D8093312B909398
:10D34000322BA093332BB093342B5AC050E0EA0118
:10D3500022976C177D07B0F40E943B6980912D2BBA
:10D3600090912E2BA0912F2BB091302B0196A11DC7
:10D37000B11D80932D2B90932E2BA0932F2BB09328
:10D38000302B3EC0B9016A58764D0E94FB91E09166
:10D3900074291E9FF0011124EB50F64D808180937B
:10D3A00065290E943B69809147018093662990918D
:10D3B0006B29992311F0891710F480936B296091E0
:10D3C000662970E084E00E94205C6091652970E02D
:10D3D00083E00E94205C4091492B50914A2B609140
:10D3E0004B2B70914C2B4F5F5F4F6F4F7F4F409394
:10D3F000492B50934A2B60934B2B70934C2B02C0BC
:10D40000C0E0D0E0CE01DF91CF911F910895CF937E
:10D41000DF93EC01888199810097E9F0873095408E
:10D4200021F01982188283E026C06238C1F410927C
:10D430006C290E94A75B0E940E5B60E870E00E946E
:10D440005B69181619066CF40E94095BE09155039C
:10D45000F0915603099587E095E09983888381E0F0
:10D460000AC08091692990916A29019690936A294E
:10D4700080936929F0CFDF91CF91089591E0909347
:10D480003A140E9493660C942E688091390181FDB4
:10D4900006C040E06FE085E491E00C94DA6B80E137
:10D4A00008950F931F93CF93DF93182F21E02093BC
:10D4B0003A140091012B8091390181FF16C08091AF
:10D4C0009400909195009093962B8093952B2093A8
:10D4D000842B2093002B809139018D7F809339011B
:10D4E0008091002B8111FCCF00E00E94CD668091DD
:10D4F000012B882309F43FC08091862B8823D9F122
:10D500008091940090919500E091992BF0919A2B45
:10D510008E179F07A0F44091692B50916A2B609160
:10D520006B2B70916C2B4C57514E6F4F7F4F40932C
:10D53000692B50936A2B60936B2B70936C2B20910B
:10D540009400309195002E1B3F0B4091692B509118
:10D550006A2B60916B2B70916C2B420F531F611DD6
:10D56000711D4093692B50936A2B60936B2B7093C2
:10D570006C2B1092862B8091390181FD03C089E1CB
:10D580000E94D26686E00E942B5C892B51F00E949B
:10D59000456AC82F86E00E942B5C81500E949366EA
:10D5A00002C0C0E0D0E0209194003091950030930B
:10D5B000982B2093972B81E08093852BF894809172
:10D5C0003901826080933901809139018D7F809388
:10D5D000390162E0610F87EB93E10E94156C78944A
:10D5E0002091FB2A3091FC2A2F5F3F4F3093FC2A79
:10D5F0002093FB2A0E94CD6645E060EE82E491E034
:10D600000E94DA6B182F86E00E942B5C892B19F0A0
:10D610008C2F0E949366002319F00E94B36702C00A
:10D620000E9412678091852B8823D9F18091940004
:10D6300090919500E091972BF091982B8E179F0772
:10D64000A0F44091652B5091662B6091672B7091EF
:10D65000682B4C57514E6F4F7F4F4093652B509323
:10D66000662B6093672B7093682B20919400309108
:10D6700095002E1B3F0B4091652B5091662B6091BE
:10D68000672B7091682B420F531F611D711D4093D2
:10D69000652B5093662B6093672B7093682B1092C9
:10D6A000852B8091012B882361F02091940030918B
:10D6B000950030939A2B2093992B81E08093862BB1
:10D6C00007C023E040E06FE182E491E00E94E46B58
:10D6D0000E942E681130E9F01330A9F480913D2B9F
:10D6E00090913E2BA0913F2BB091402B0196A11D14
:10D6F000B11D80933D2B90933E2BA0933F2BB09375
:10D70000402B12E009C0153031F0173029F411E038
:10D7100003C010E001C013E0812F90E0DF91CF91B2
:10D720001F910F910895CF93DF93EB010E94416801
:10D73000009729F4CE010E94516A009751F0209180
:10D74000FE2A3091FF2A2F5F3F4F3093FF2A20930C
:10D75000FE2ADF91CF910895CF93DF938091012B23
:10D76000811104C00E94E467D1E001C0D0E00E94B2
:10D770007766863111F0813119F4C091470109C0F3
:10D7800040E06FE186E491E00E94DA6BC82FCC0F95
:10D79000C80FD1110E949C678C2FDF91CF91089503
:10D7A00010923E1410923D14EFE6F0E0808180620A
:10D7B00080830895FC018081862390E002C09595C6
:10D7C00087954A95E2F70895F894FC015081362F29
:10D7D00030955323042E01C0220F0A94EAF7262322
:10D7E000522B50837894089540917B01FC01419322
:10D7F000A0E8B1E050E8540F9D012F5F3F4F6C91BE
:10D800006193521711F0D901F7CF4150E42FF0E0A6
:10D81000E058FE4F2181FC01E058FF4F2083FC01BE
:10D82000EF57FF4F21E02083089560938001E1E8E6
:10D83000F1E061589F012F5F3F4FDC014D91CD0119
:10D840004083621711F0F901F5CF08951F920F92EE
:10D850000FB60F9211240BB60F922F933F934F9355
:10D860005F936F937F938F939F93AF93BF93EF9348
:10D87000FF9380914701809366298091732922E864
:10D88000829FC00111248B58964D0E94F46B8091A9
:10D8900073298F5F833018F48093732902C010922C
:10D8A00073290E942869FF91EF91BF91AF919F91D9
:10D8B0008F917F916F915F914F913F912F910F9039
:10D8C0000BBE0F900FBE0F901F9018951F920F92D6
:10D8D0000FB60F9211240F900FBE0F901F90189546
:10D8E0001F920F920FB60F9211240F900FBE0F9040
:10D8F0001F9018951F920F920FB60F9211240F9040
:10D900000FBE0F901F9018951F920F920FB60F9297
:10D9100011241092002B0F900FBE0F901F9018959E
:10D920001F920F920FB60F9211241092002B0F909E
:10D930000FBE0F901F9018951F920F920FB60F9267
:10D9400011248F9381E080936C298F910F900FBEEB
:10D950000F901F9018951F920F920FB60F921124DF
:10D960001092002B0F900FBE0F901F9018951F92D2
:10D970000F920FB60F9211248F939F9380913D14B5
:10D9800090913E14019690933E1480933D149F9184
:10D990008F910F900FBE0F901F901895CF92DF922E
:10D9A000EF92FF920F931F93CF93DF937C018B0134
:10D9B0006A018FE394E10E943555EC01009751F024
:10D9C000EC81FD81309711F0C8010995CE010E94CC
:10D9D000DD55F3CFA601B801C701DF91CF911F91AB
:10D9E0000F91FF90EF90DF90CF900C94BF520F9368
:10D9F0001F93CF93DF9300D0CDB7DEB78091092B73
:10DA000090910A2BA0910B2BB0910C2B0196A11D8C
:10DA1000B11D8093092B90930A2BA0930B2BB093ED
:10DA20000C2B0E94616F8C018FE394E10E943555AD
:10DA3000009779F0DC011296ED91FC9113973097E5
:10DA400029F089839A8309959A8189810E94DD55FD
:10DA5000EFCF0115110549F0C8010F900F90DF912C
:10DA6000CF911F910F910C94B6520F900F90DF91B0
:10DA7000CF911F910F9108950E9454740E94A75B4B
:10DA80000E94886D81E493E09093042B8093032B94
:10DA90000E945F6F2FEF31E040E05EE160E074E0F4
:10DAA00082E090E00C94286FBC018FE394E10C9429
:10DAB0009555BC018FE394E10C947A55CF93DF9395
:10DAC000EC014091052B5091062B6091072B709132
:10DAD000082B4F5F5F4F6F4F7F4F4093052B509345
:10DAE000062B6093072B7093082B0E94746F00978E
:10DAF00061F00E94275BE0914503F0914603BE016F
:10DB00008EEC9CE6099581E090E0DF91CF9108953D
:10DB100085E494E10C9431550F93CF93DF93EC019E
:10DB20007B836A8318865F834E83BC0185E494E11E
:10DB30000E949555E0914114F0914214309749F0BC
:10DB40004C815D8101E020E030E068858A819B8125
:10DB50000995DF91CF910F910895BC0185E494E17F
:10DB60000C947A550F93DC0118961C921897E0914B
:10DB70004114F0914214309759F000E020E030E079
:10DB800040E050E060E012968D919C9113970995CA
:10DB90000F9108950F93DC01AB0114962D913C91E8
:10DBA000159781E018968C93189715967C936E9331
:10DBB0001497E0914114F0914214309739F000E04D
:10DBC00061E012968D919C91139709950F9108959C
:10DBD0000F93DC01E0914114F0914214309771F001
:10DBE00014964D915C91159701E09A0118966C91ED
:10DBF000189712968D919C91139709950F910895FE
:10DC0000E0914314F0914414309709F00994089579
:10DC100090934414809343140895909342148093F6
:10DC20004114089585E494E10C943555EF92FF92E8
:10DC30000F931F93CF93DF938C01EB017A0185E45F
:10DC400094E10E9435550097D9F0DC0112962D9190
:10DC50003C9113972C173D0781F41696ED91FC919A
:10DC60001797309769F09701AE01B801DF91CF9116
:10DC70001F910F91FF90EF9009940E94DD55E3CF23
:10DC8000DF91CF911F910F91FF90EF90089508952C
:10DC9000CF93DF93C8E7D4E16881798120E030E059
:10DCA00047E65EE682E694E10E94B5570E94527410
:10DCB000688179810E94028C20E030E04BE75EE6CB
:10DCC000BC0182E594E1DF91CF910C94B55780912E
:10DCD0007814909179142091761430917714880FEC
:10DCE000991F2817390708F4C90190937914809374
:10DCF00078140C94486ECF93DF930E94A75B0E9428
:10DD00000E5BEC01198218820E94126E2881398103
:10DD1000009719F1FC0140854423F9F0FC01428190
:10DD20005381F901EE0FFF1FEE0FFF1FEC0FFD1FD8
:10DD300053834283FC01448155812F5F3F4FF9019A
:10DD4000EE0FFF1FEE0FFF1FEC0FFD1F51834083EF
:10DD5000398328830E94DD55D9CFC901880F991FC7
:10DD6000880F991F02960E94095B88819981892BEF
:10DD700031F087E494E1DF91CF910C948D52DF91E3
:10DD8000CF910895AF92BF92CF92DF92EF92FF9220
:10DD90000F931F93CF93DF9300D0CDB7DEB76B0106
:10DDA0000E940E5BFC01008111811A8309830C30F3
:10DDB000110518F4E12CF12C0DC01F930F9380E88E
:10DDC00099E09F938F930E94B0920F900F900F90C5
:10DDD0000F9021C0E016F106F1F00E940E5BF701F2
:10DDE000EE0FFF1FEE0FFF1FE80FF91FA280B38099
:10DDF0000E940E5BFFEFEF1AFF0AF701EE0FFF1F05
:10DE0000EE0FFF1FE80FF91F40815181B501C601D8
:10DE10000E94166EDFCF0F900F90DF91CF911F9170
:10DE20000F91FF90EF90DF90CF90BF90AF9008954B
:10DE30000F93013059F48091721490917314909360
:10DE40007914809378140F910C94486E0F91089573
:10DE5000EF92FF920F931F93CF93DF938B01EA0111
:10DE600079014EE253E0BC0187E494E10E947152D3
:10DE70001093731400937214D0937514C093741498
:10DE8000F0927714E092761488E19FE6DF91CF91CB
:10DE90001F910F91FF90EF900C940D6E82E694E12C
:10DEA0000E94395882E594E10E94395887E494E150
:10DEB0000C948B52809178149091791408950C945D
:10DEC000CB52CF93DF93E0913203F0913303099566
:10DED000EC01009729F06A817B8181E00E94205C3F
:10DEE000CE01DF91CF9108950F931F93CF93DF93CE
:10DEF000EC01E0913403F091350309958C016A81BE
:10DF00007B8181E00E94205C81E090E0012B11F494
:10DF100080E090E0DF91CF911F910F910895E09103
:10DF20003603F0913703099420E030E00296FC01BB
:10DF300032974081442331F0FC0131974081240F16
:10DF4000311DF4CFC9010895FC01208130E0322F4A
:10DF500022278181282B02C0220F331F6A95E2F706
:10DF6000832F9927FA01E85CFC4F208130E082235F
:10DF7000932328E030E0241B350B02C0969587954B
:10DF80002A95E2F708956F927F928F929F92AF92B7
:10DF9000BF92CF92DF92EF92FF920F931F93CF9396
:10DFA000DF938C01EB016A0179012830310524F4FB
:10DFB000A901B601CE014AC0590123E0B594A79446
:10DFC0002A95E1F74115510521F04801612C712C8A
:10DFD00003C0D801FB0120C048E050E0B601CE01EB
:10DFE000860D971D0E94A46FF40181934F01FFEFEE
:10DFF0006F1A7F0A6A147B047CF3C501B7FE02C066
:10E0000080E090E0A701477055274115510511F1B7
:10E01000080F191FB60118C0CF018C1B9D0B8A1564
:10E020009B051CF481918D93F7CFC501B7FE02C00B
:10E0300080E090E0A701477055274115510551F048
:10E04000080F191F60E070E08C0F9D1F0E94A46FE5
:10E05000F8018083DF91CF911F910F91FF90EF9096
:10E06000DF90CF90BF90AF909F908F907F906F90F8
:10E0700008958F929F92AF92BF92CF92DF92EF92CC
:10E08000FF920F931F93CF93DF9300D0CDB7DEB7EE
:10E090000E940E5B8C0182E090E00E94EC5A892B7A
:10E0A00019F480E090E05DC0F801818190E0982F44
:10E0B00088272081820F911D0E94DC527C010097ED
:10E0C00081F30E940E5B4C01F7012681822F869519
:10E0D0008695869590E0422F477021E030E011F45C
:10E0E00020E030E0820F931F0E94EC5A892BC9F286
:10E0F000F70104811581C12CD12CF801808188237E
:10E1000079F1F801A180B12CB60133E075956795DE
:10E110003A95E1F7A60147705527680D791D8831BA
:10E1200068F09501CE0101960E94C36FBE016F5F3A
:10E130007F4FF80180810E94345C0DC01A821982E1
:10E140009501CE0101960E94C36F69817A81F80121
:10E1500080810E94205CCA0CDB1C0E5F1F4FCDCF5C
:10E16000C7010F900F90DF91CF911F910F91FF90FA
:10E17000EF90DF90CF90BF90AF909F908F900895D9
:10E18000DC0150E0E0E1F0E0E61BF70BE21BF30BF3
:10E1900002C0440F551FEA95E2F78C91852B8C93B2
:10E1A00011968C911197842B11968C9308956F92F0
:10E1B0007F928F929F92AF92BF92CF92DF92EF9217
:10E1C000FF920F931F93CF93DF938C016B01EA01B2
:10E1D0007901283031051CF44881C8015CC039013F
:10E1E00053E0759467945A95E1F76115710521F034
:10E1F0004E01A12CB12C03C0D801FE0127C0F401AF
:10E2000041914F0128E030E0B601C8018A0D9B1D05
:10E210000E94C070FFEFAF1ABF0AA614B7047CF3C8
:10E22000C30177FE02C080E090E09701277033279A
:10E230002115310509F43FC0C80FD91F488150E0AE
:10E24000B601621B730B685F7F4F1CC0CF018C1B34
:10E250009D0B861597051CF481918D93F7CFC30113
:10E2600077FE02C080E090E09701277033272115E8
:10E27000310509F1C80FD91F488150E068E070E00E
:10E28000621B730B02C0559547956A95E2F760E0F3
:10E2900070E0800F911FDF91CF911F910F91FF9040
:10E2A000EF90DF90CF90BF90AF909F908F907F9036
:10E2B0006F900C94C070DF91CF911F910F91FF90E0
:10E2C000EF90DF90CF90BF90AF909F908F907F9016
:10E2D0006F9008956F927F928F929F92AF92BF92AC
:10E2E000CF92DF92EF92FF920F931F93CF93DF9322
:10E2F00000D0CDB7DEB78C01FC018681E82EE69414
:10E30000E694E694F12C282F277081E090E011F438
:10E3100080E090E0E80EF91EC70102960E94705B53
:10E32000009709F445C00E94155BF8012281FC01A9
:10E330002083F8012381FC0121830E94155B029652
:10E340005C01A70160E070E00E940492F801048182
:10E350001581E12CF12CF8018081882339F1F80135
:10E360008180912C670163E0D594C7946A95E1F7A9
:10E370003701F7E06F227724CA0CDB1C883128F0C4
:10E380000E943E5C9401AC0108C00E942B5C9A8301
:10E3900089839401AE014F5F5F4FB301C6010E94B4
:10E3A000D770E80CF91C0E5F1F4FD5CF81E090E0CD
:10E3B0000F900F90DF91CF911F910F91FF90EF90F1
:10E3C000DF90CF90BF90AF909F908F907F906F9095
:10E3D0000895E0915303F09154030994E0912C03C4
:10E3E000F0912D030994E0915703F091580309949B
:10E3F000E0915903F0915A03099480E090E0089568
:10E400000895E0912403F0912503099480E090E0C1
:10E4100008950F931F93CF93DF93CDB7DEB7E097A7
:10E420000FB6F894DEBF0FBECDBF0E945B5B8C01C0
:10E430000E940E5BAE014F5F5F4F602F0E94D97943
:10E44000882309F446C088A99801281B3109C9010D
:10E450000E94EC5A892BE9F12E8121110CC0BE01DA
:10E460006A5E7F4F88E10E94345CE0914703F0913F
:10E47000480309952EC08A859B858D3C3BEA93070E
:10E4800011F0019631F5223019F088E090E002C0D9
:10E4900082E090E001979C012F5F3F4F1216130618
:10E4A000F4F6E1E0F0E0EC0FFD1FE80FF91F238523
:10E4B0002F3F81F3BE01645F7F4F89E10E94345C8E
:10E4C00089E10E943E5C62E179E20E942A52892B36
:10E4D00031F6E0960FB6F894DEBF0FBECDBFDF91E8
:10E4E000CF911F910F910895AF92BF92CF92DF927B
:10E4F000EF92FF920F931F93CF93DF93CDB7DEB7C9
:10E50000E0970FB6F894DEBF0FBECDBF8C016B0154
:10E51000CE0101967C0180E3F70111928A95E9F71B
:10E5200081E089838CE00E942B5C8C831D821F829A
:10E5300080917C1491E0980F90937C14898783E0FC
:10E54000B82EB8868DEC9BEA9B878A8789E10E946A
:10E550003E5C60E073E00E942A52892B31F082E039
:10E560008E838FEF8C878D8709C089E10E943E5C86
:10E57000BC01CE010C960E942152BE828DEC9BEA1A
:10E580009D8B8C8B62E179E2CE0146960E942152EE
:10E590000E940E5B9FA78EA70E945B5B88ABC701A2
:10E5A0000E94D278B82E90E00E94705B892B31F1E6
:10E5B0000E94155BBC014B2DC7010E94F078E090D2
:10E5C0001A03F0901B030E94655B5C010E94155BBF
:10E5D000B501F70109950115110581F0009739F092
:10E5E000019761F441E050E064E070E004C041E074
:10E5F00050E060E070E0C601F8010995E0960FB6C2
:10E60000F894DEBF0FBECDBFDF91CF911F910F9168
:10E61000FF90EF90DF90CF90BF90AF9008950E9451
:10E62000527480937C14E0912403F09125030994A3
:10E63000892B29F0E0912403F091250304C0E09197
:10E640002603F09127030994CF93DF93EC0189917E
:10E650009991009729F060E070E00E947554F7CF1F
:10E66000DF91CF910895CF93DF93EC018991999138
:10E67000009719F00E94C753F9CFDF91CF91089509
:10E68000CF93DF93EC017B836A830E94E9649983D3
:10E690008883DF91CF910895FC018081918122814F
:10E6A0003381820F931F918380830895CF93DF93EB
:10E6B000EC010E94E96499838883DF91CF910895EA
:10E6C000CF93DF93EC010E94E96428813981821B9A
:10E6D000930B9C012F5F3F4F81E090E04A815B816B
:10E6E0004217530710F080E090E0DF91CF9108953A
:10E6F000CF93DF93FC01C281D38180819181C80FC8
:10E70000D91F0E94E9649E01281B390BC901DF91C2
:10E71000CF910895CF93DF93EBE8FBE2CDE4DBE20A
:10E72000AFE7BBE2119211921992199219921992C4
:10E730001D928BE2E33AF807A9F7DF91CF91089594
:10E74000CF93DF93FC01E158F44D40819C01220FEF
:10E75000331F220F331F442301F1A0919400B09185
:10E760009500FC01EE0FFF1FE557F44D808191816C
:10E77000AD01481B590BCA01E901C35BD44D488167
:10E7800059816A817B81480F591F611D711D488322
:10E7900059836A837B83B183A083F901E35BF44DE2
:10E7A0006081718182819381DF91CF91089560E0D2
:10E7B00070E0CB010895FC01EE0FFF1FEE0FFF1F6D
:10E7C000E35BF44D40835183628373830895CF9359
:10E7D000DF932FE73BE2CDE4DBE2EBE8FBE2D9019C
:10E7E0008D919D018823B9F040919400509195003E
:10E7F00080819181BA01681B790B88819981AA81F6
:10E80000BB81860F971FA11DB11D88839983AA83A1
:10E81000BB835183408324963296BBE22B383B075F
:10E82000F1F6DF91CF9108950C9461780F931F93C7
:10E83000FC01CB0140917D1450917E1433832283DF
:10E840001583048371836083F0937E14E0937D14B9
:10E85000452B11F40E947B7880E090E01F910F918E
:10E86000089580917D1490917E140097C1F01092CC
:10E870007E1410927D14DC0114966D917C91159795
:10E880001296ED91FC9113970995E0917D14F0910A
:10E890007E14309721F0808191810C947B780895CB
:10E8A0000C948E8E0C948A8E84ED92E00E94AC546F
:10E8B0008CEC92E00C94AC54CF93DF930E941B5BE2
:10E8C000892BA9F08CEC92E00E94CA54EC010097CD
:10E8D00021F10E945B5B998388830E94565B9B8336
:10E8E0008A83CE0104960E94975A8CAB14C084EDA3
:10E8F00092E00E94CA54EC01009779F002960E94BF
:10E90000A95A99838883BE016E547F4FCE018E57DA
:10E910009F4F0E94FE5BCE0102C080E090E0DF913D
:10E92000CF910895BC016E547F4F8E579F4F0C942A
:10E93000FE5BCF93DF93EC01BC0184ED92E00E947B
:10E940001455BE01892B19F084ED92E009C08CECBE
:10E9500092E00E941455892B39F0BE018CEC92E0B4
:10E96000DF91CF910C94EF54DF91CF9108950F93E5
:10E970001F93CF93DF93EC01BC0184ED92E00E94E2
:10E980001455892B91F0FE0161917191CF010E9484
:10E99000BA5BBE016E547F4FCE018E579F4FDF9101
:10E9A000CF911F910F910C940F5CBE018CEC92E003
:10E9B0000E941455892BD1F00E94A75B6881798150
:10E9C0008A819B810E94BA5B8CA990E00E94705B57
:10E9D0000CA910E00E94155BBE016C5F7F4FA8017F
:10E9E000DF91CF911F910F910C94FB91DF91CF910B
:10E9F0001F910F910895CF93DF93EC01BC0184ED3B
:10EA000092E00E941455892B19F0CE0102960CC099
:10EA1000BE018CEC92E00E941455892B19F08A817A
:10EA20009B8102C080E090E0DF91CF910895FC01CE
:10EA3000808191810895860F911D860F911D8E57BB
:10EA40009F4F0895860F911D860F911D8E579F4FE2
:10EA5000FC0180819181089508958CED9AE10E94D6
:10EA6000EE56892B21F08CED9AE10C94DB5608953B
:10EA7000E091C81AF091C91A309709F0099480E022
:10EA80000895EF92FF920F931F93CF93DF937C0132
:10EA9000EA01FC0180819181009741F08C30934024
:10EAA00071F1F7011182108283E0F2C080E024E06E
:10EAB000829FF0011124E653F54E118210828F5F80
:10EAC0008430A8F38093C71A8091021290910312A8
:10EAD0009093DB1A8093DA1A0E94C0538093A32B81
:10EAE00060E470E08CED9AE10E94C7560E944F7B73
:10EAF0008CE093E0F7019183808381E0C9C06230AC
:10EB0000D9F48091A42B9091A52B892B89F3809126
:10EB1000B52B863029F48091CD2B81FD0E942D7577
:10EB200081E00E948D7C8091A42B9091A52B892B54
:10EB3000F9F20E945177DCCF633060F5611114C0A7
:10EB40002097B1F2D093B230C093B13083E00E94ED
:10EB50008D7C8091A42B9091A52B892B11F00E9484
:10EB600038750E942D75C4CF613011F6209709F4D5
:10EB7000BFCFD093AE30C093AD3085E00E948D7C86
:10EB80008091A42B9091A52B892B09F4B1CF0E94E1
:10EB90003875AECF6738E9F51092C61A0AEC1AE15B
:10EBA0008091C61A8430B8F4F801828193818C1761
:10EBB0009D0749F4808191810E945A7CF80111825D
:10EBC0001082138212820C5F1F4F8091C61A8F5FD2
:10EBD0008093C61AE5CFECECF0E3838194818C1727
:10EBE0009D0719F4148213821082B09621E3EC344D
:10EBF000F20799F7E9E4F1E3818592858C179D0787
:10EC000011F4158214823D9681E3EB3CF807A1F7DD
:10EC10006FCF683809F06CCFCC5DDA4109F068CF6E
:10EC20008CED9AE10E94EE56892B09F461CF109287
:10EC3000C61AE091C61AE43008F05ACF20E2E29FEB
:10EC4000F0011124ED54FF4C818D8823D9F08CED17
:10EC50009AE10E94DB568091C61AE0E28E9FC001C5
:10EC600011248D549F4C9093B2308093B13082E048
:10EC70000E948D7C8091A42B9091A52B892B11F063
:10EC80000E9438758091C61A8F5F8093C61AD1CFC3
:10EC9000DF91CF911F910F91FF90EF900895909386
:10ECA000C91A8093C81A0895209102123091031254
:10ECB00060E0EAECFAE1643098F440815181481751
:10ECC000590759F4428153814217530731F4609335
:10ECD000C51A118210820C945A7C34966F5FEBCF68
:10ECE0006093C51A089540E0EAECFAE14430A8F4D4
:10ECF00051E0540F20813181232B61F44093C41AD9
:10ED000091838083209102123091031233832283F6
:10ED10000C94747C3496452FE9CF4093C41A08951F
:10ED20002091021230910312FC01358F248F778FCE
:10ED3000668F08952091021230910312FC013287F0
:10ED40002187748763870895CF93DF93EA010E9438
:10ED5000FD7B009749F02091021230910312FC01D3
:10ED600032872187D487C387DF91CF9108950F938E
:10ED70001F93CF93DF9300D000D0CDB7DEB78C01C7
:10ED8000AB018FEF89838A838B838C83B801CE019B
:10ED900001960E94A476009719F0FC011583048364
:10EDA0000F900F900F900F90DF91CF911F910F91C7
:10EDB000089540E050E062E08CED92E00E946654DD
:10EDC0001092A52B1092A42B0895AC0161E08CED5C
:10EDD00092E00C944854AC0160E08CED92E00C940D
:10EDE00048540F931F93CF93DF938A010E947B7B3C
:10EDF000EC01009759F080910212909103129D8FBF
:10EE00008C8F1F8F0E8FCE010E94EB76CE01DF918B
:10EE1000CF911F910F910895CF93DF93A091B130BF
:10EE2000B091B230109719F0ED016C9605C0C09109
:10EE3000AD30D091AE3029968091AC3086FF22C0A3
:10EE40001092C31A40E0EAECFAE14430B8F42081B1
:10EE5000318114968D919C9115972817390759F493
:10EE600082819381009739F04093C31A99838883F4
:10EE70001B821A8205C034964F5FE7CF4093C31AB6
:10EE80000E942D7588819981009741F04A815B81AC
:10EE90006091A32BDF91CF910C946654DF91CF91B9
:10EEA00008950F931F93CF93DF938091B52B8630F6
:10EEB00009F071C08091A42B9091A52B81159540EC
:10EEC00009F069C0C4E9D2E0D093A52BC093A42B6C
:10EED00002E00093AE2B14E91093AF2B1092D12BCC
:10EEE0001092D02B0E94497B809590959093D12BC6
:10EEF0008093D02B1092B72B1092B62B0E94387BA8
:10EF0000809590959093B72B8093B62B0E9438757F
:10EF1000D093A52BC093A42B0093AE2B1093AF2BB3
:10EF2000A091AF30B091B030FD01E459FD4F8CE6B7
:10EF300092E001900D920197E1F76CE672E084ECAB
:10EF40009BE20E94F77A8091A82B8093C42B80913A
:10EF5000A92B8093C52B8091AA2B8093C62B8091DF
:10EF6000AB2B8093C72B1092D12B1092D02B0E94E9
:10EF7000497B809590959093D12B8093D02B1092C4
:10EF8000B72B1092B62B0E94387B8095909590936A
:10EF9000B72B8093B62BDF91CF911F910F910C94DB
:10EFA0003875FC01680F791F80E048E1E617F70724
:10EFB00081F0219198E0322F3827532F517030FD86
:10EFC00084278695513009F480682695915099F7E9
:10EFD000EDCF08951F920F920FB60F9211240BB62A
:10EFE0000F922F933F934F935F936F937F938F93E2
:10EFF0009F93AF93BF93EF93FF9380919400909171
:10F0000095009093902B80938F2B81E08093812BA0
:10F0100080917100807D809371000E943174809195
:10F02000812B8823D9F18091940090919500409193
:10F030008F2B5091902B84179507A0F48091552B1E
:10F040009091562BA091572BB091582B8C57914EE5
:10F05000AF4FBF4F8093552B9093562BA093572BB8
:10F06000B093582B2091940030919500241B350BC0
:10F070008091552B9091562BA091572BB091582BE6
:10F08000820F931FA11DB11D8093552B9093562B7A
:10F09000A093572BB093582B1092812BFF91EF9197
:10F0A000BF91AF919F918F917F916F915F914F91A0
:10F0B0003F912F910F900BBE0F900FBE0F901F909E
:10F0C00018959FB7F894E1E7F0E08081807D808318
:10F0D00088B38F6288BB10929000E1E9F0E0108263
:10F0E0001092920010929500109294008081856099
:10F0F00080839FBF08952FB7F894909399008093D1
:10F10000980088B38F6288BBE1E7F0E0808182607D
:10F1100080832FBF0895CF93DF93FC01DB0185E04F
:10F12000EB0119928A95E9F78581837011F082E0ED
:10F130008C938781837021F082E012968C931297D2
:10F140008581837081F08781837069F02389348998
:10F15000818592852817390731F481E084831296DE
:10F160001C92129701C0148285818370823021F035
:10F17000833021F080E003C082E001C088E0119676
:10F180008C93119787818370823021F0833021F036
:10F1900080E003C082E001C088E013968C93DF9189
:10F1A000CF910895CF93DF9300D000D01F92CDB7B9
:10F1B000DEB7BE016F5F7F4F0E948B7889819A8195
:10F1C000890F8D5F9B81890F9C81890F9D81890F9C
:10F1D0000F900F900F900F900F90DF91CF910895A7
:10F1E0004F925F926F927F928F929F92AF92BF9257
:10F1F000CF92DF92EF92FF920F931F93CF93DF9303
:10F2000000D000D000D0CDB7DEB78C017B01BE01AD
:10F210006F5F7F4F4E830E948B78B981AA815B809C
:10F220004C808B2F90E003962A2F30E0820F931FA3
:10F23000850D911D642D70E0860F971F5D81850FF0
:10F24000911D4E8150E0481759070CF49AC0F801FF
:10F25000818180FB662460F8712C43E0660C771C8A
:10F260004A95E1F7828180FB882480F8912C54E054
:10F27000880C991C5A95E1F7862880818770882A26
:10F28000838180FBAA24A0F8B12C85E0AA0CBB1CCA
:10F290008A95E1F78A28848180FBCC24C0F8D12CA0
:10F2A00096E0CC0CDD1C9A95E1F78C28F701808262
:10F2B000F80145814370F4E04F9FA0011124F8014B
:10F2C00086818370F0E18F9FC0011124482BF801E3
:10F2D0008781F0E48F9FC0011124482BF7014183FF
:10F2E000F8018085F7018283B23059F4F8018185F5
:10F2F000F7018383F8018285F701848395E0C92EA5
:10F3000002C083E0C82EB0E080E090E0200F311F03
:10F31000DB2EDC0C0197BA1761F0A901480F591FC9
:10F32000FA01B384A7014D0D511DFA01B082BF5FF0
:10F33000EFCF9D2DF2E05F120EC0D701AD0DB11DD4
:10F34000F80183898C9381E08D0DD701A80FB11D41
:10F350009E5F84898C9340E020E030E0060F171F09
:10F36000842F890F21503109441561F0D801A20F73
:10F37000B31F55965C91D701A80FB11D5C934F5FE9
:10F38000EFCF80E026960FB6F894DEBF0FBECDBF5C
:10F39000DF91CF911F910F91FF90EF90DF90CF9071
:10F3A000BF90AF909F908F907F906F905F904F90A5
:10F3B0000895BF92CF92DF92EF92FF920F931F9327
:10F3C000CF93DF937C01D62EEA0182E0861708F006
:10F3D000B2C0F701808186FBBB24B0F89181292F50
:10F3E000269526952370C92EC294C694C69453E0E0
:10F3F000C522382F3770388383FB332730F93983A0
:10F4000084FB332730F93A8385FB882780F98B8387
:10F41000BC822D83892F829583708E83CF828281D7
:10F420008887222391F13381848190E0982F882767
:10F43000830F911D9A87898787010B5F1F4F2230A9
:10F4400079F460E073E0CE010B960E942152F7013F
:10F4500086818B8785818C878701095F1F4F20C03C
:10F460002330F1F4F7013D9680E090E03E2F2F2FFE
:10F470004291DE01A80FB91F1B964C93019688306C
:10F480009105B1F7032F122F0BC087010D5F1F4F9E
:10F4900060E073E0CE010B960E9421521A86198615
:10F4A000CC20B9F1B1100DC0F8012081818190E02C
:10F4B000982F8827820F911D9C8B8B8B0E5F1F4F7F
:10F4C00004C089859A859C8B8B8BF2E0CF120EC08D
:10F4D00060E073E0CE0145960E942152F8018181DF
:10F4E0008D8B80818E8B0E5F1F4F1BC0F3E0CF1280
:10F4F00018C0085F1F4FF80180E090E02291DE0104
:10F50000A80FB91F55962C93019688309105B1F735
:10F5100008C060E073E0CE0145960E9421521C8A2B
:10F520001B8AC8018E199F092D2D281B2FA71EA7E6
:10F530000DA7D81608F480E0DF91CF911F910F91AD
:10F54000FF90EF90DF90CF90BF900895FB01415066
:10F550005109460F571FE417F50778F4208130E072
:10F56000322F22276181260F311D820F931F8217B0
:10F57000930708F401963296EECFE417F50751F49D
:10F58000208130E0322F2227820F931F82179307AA
:10F5900008F401960895CF93DF93C091AF2BD0E08C
:10F5A00064972091AE2B30E0322F2227C20FD31F59
:10F5B00048E050E068EB7BE29E01280F311DC90155
:10F5C0000E94A67AAE0160EC7BE20E94A67A0097C8
:10F5D00021F098278927982702C08FEF9FEFDF91AE
:10F5E000CF9108959093F51A8093F41A0895FC0131
:10F5F0005381560F5093AB2B872F99274281480F89
:10F600004093AA2BA181A093A92BE081E093A82B82
:10F61000242F30E02817390748F481E08A0F8093BF
:10F62000A92B811103C0EF5FE093A82B852F90E0F9
:10F6300077278617970788F44F5F4093AA2B4111CD
:10F640000CC08091A92B8F5F8093A92B811105C0DD
:10F650008091A82B8F5F8093A82B0895AB01BC01EC
:10F6600080E090E00E94A67A98278927982708953D
:10F6700044E150E06CEA7BE280E090E00E94A67AF0
:10F68000009721F098278927982708958FEF9FEFFB
:10F69000089586E00C94CB7A81E10C94CB7A80E0DB
:10F6A000E82FF0E0EE0FFF1FED5CFE4C11821082A0
:10F6B0008F5F8430A8F380E090E2899FF0011124ED
:10F6C000ED54FF4C118E8F5F8430B0F380E094E0F6
:10F6D0009093EF1A8093EE1A80E09DE0989FF001DE
:10F6E0001124E75BFE4C158214828F5F8A30B0F3E1
:10F6F0008093ED1A0895CF932091EE1A3091EF1A6E
:10F700002F5F3F4F21154DE7340710F020E030E127
:10F71000522F432FE3EBF0E3C0E0C43059F0A18D4A
:10F72000AA2329F0A481B581A417B50749F3CF5FB7
:10F73000B096F3CF3093EF1A2093EE1A1092ED1A91
:10F7400020E0E0E0F0E02430E8F430E2239FD00154
:10F750001124AD54BF4C59963C915997311104C0B6
:10F760002093ED1AFD0110C0373041F4309739F085
:10F770005A964C915A97328D341708F0DF012F5F5B
:10F78000FD01E1CF2093ED1A3097A1F122E0218F06
:10F790002091F01A24872091F11A25872091F21ADE
:10F7A00026872091F31A278728ED34E0338B228BAC
:10F7B000358B248B21E030E0318B208B138E21E0C0
:10F7C000228F23E0208F168A20E1278B2091EE1ACA
:10F7D0003091EF1A3227232732273583248377830A
:10F7E0006683DC014D915D916D917C9140835183E5
:10F7F00062837383CF01CF910895CF93DF932091DC
:10F80000EE1A3091EF1A2F5F3F4F21154DE7340765
:10F8100010F020E030E1522F432FEDE4F1E3C0E09F
:10F82000CA3041F0A081B181CF5F3D96A417B507E2
:10F83000B9F7E9CF3093EF1A2093EE1A40E05DE07C
:10F840004A30A0F4A1E0A40F549FF0011124E75B1B
:10F85000FE4C24813581232B39F44093ED1A3097E7
:10F8600041F480E090E023C04A2FEACF4093ED1AA4
:10F87000F8CF2091EE1A3091EF1A32272327322742
:10F880003583248377836683009729F4108211825D
:10F890001282138209C0EC0188819981AA81BB81FF
:10F8A00080839183A283B38380E48087CF01DF913B
:10F8B000CF91089540E04430A0F4E42FF0E051E00F
:10F8C000540FEE0FFF1FED5CFE4C20813181281795
:10F8D000390729F44093ED1A118210820895452FBB
:10F8E000EACF4093ED1A089540E0443098F4E42FB5
:10F8F000F0E051E0540FEE0FFF1FED5CFE4C208155
:10F900003181232B29F44093ED1A9183808308954C
:10F91000452FEBCF4093ED1A0895AF92BF92CF924F
:10F92000DF92EF92FF920F931F93CF93DF93C091DB
:10F93000B130D091B230843009F4DCC124ED3BE227
:10F940003093B0302093AF303093A72B2093A62B69
:10F95000833059F4898D8F70833009F06BC08889AA
:10F960009989892B09F0DFC67FC0823009F080C0F9
:10F970008091F31A8F5F8093F31A811113C08091E5
:10F98000F21A8F5F8093F21A81110CC08091F11AE4
:10F990008F5F8093F11A811105C08091F01A8F5FFB
:10F9A0008093F01A1092A52B1092A42B109248313C
:10F9B00010924731298D822F8D7F853041F48A8DB9
:10F9C0008F5F8A8F843109F0AEC6198EACC62223B0
:10F9D00009F4A9C688899989892B09F441C08A8DBF
:10F9E0009FEF980F9A8F81119EC68B8D883031F0D2
:10F9F0009FEF920F923048F4853039F4198E80E8E9
:10FA00008093AC300E940C7747C5853038F493E082
:10FA1000082E01C0990F0A94EAF701C090E39A8F6B
:10FA20008F5F8B8F822F8F708330A1F048F48130ED
:10FA300009F44FC3823009F076C61092CD2B4CC327
:10FA4000863009F4C8C4883009F4C5C4843009F08C
:10FA50006AC6C1C484E08093AC300E940C774EC566
:10FA60002F70233009F05FC688E08093AC3009C561
:10FA7000853019F5E091AD30F091AE3084819581FB
:10FA8000892B09F450C61092B2301092B13088EC34
:10FA90009BE29093B0308093AF309093A72B8093EC
:10FAA000A62B10924831109247311092A52B10923C
:10FAB000A42B88E08093AC301BC18091AC2B8534A3
:10FAC00009F031C60091AE2B10E0102F0027809175
:10FAD000AF2B080F111D8091A42B9091A52B80179F
:10FAE000910708F420C61093A52B0093A42B8091B6
:10FAF000B22B8F7309F017C68091B32B811113C6F7
:10FB00008091433190914431C0915D03D0915E0367
:10FB10008C179D0759F44091453150914631209101
:10FB20005F033091600342175307A1F02091BC2B73
:10FB30003091BD2B2817390709F0F5C52091BE2B50
:10FB40003091BF2B8091453190914631281739076C
:10FB500009F0E9C50E94387B019609F0E4C580915F
:10FB6000B52B863009F429C18131E9F1813009F0E2
:10FB7000DAC58091C02B883009F0D5C51092C02B12
:10FB80008091C22B9091C32B873F3FEF930710F0DA
:10FB9000099601C008969093C32B8093C22B809145
:10FBA000B82B9091B92BA091BA2BB091BB2B80931D
:10FBB000BC2B9093BD2BA093BE2BB093BF2B8091F9
:10FBC000433190914431A0914531B09146318093B9
:10FBD000B82B9093B92BA093BA2BB093BB2B80E496
:10FBE0008093B42B7DC50C5111091093A52B009364
:10FBF000A42B88EC9BE29093B0308093AF3080913F
:10FC0000C62B9091C72B892B29F00E944C7B019623
:10FC100009F089C52091C22B3091C32B21153105E4
:10FC200009F481C589E491E39093AE308093AD30BF
:10FC3000A090C02BB090C12B40915F035091600306
:10FC40006091610370916203A0916303B0916403BA
:10FC50000091B82B1091B92BE090BA2BF090BB2BF0
:10FC6000E091AD30F091AE3081E3EB3CF80708F065
:10FC70005AC584819581009721F12817390709F524
:10FC800086819781009719F0A816B906D1F4808172
:10FC900091818C179D0729F4C280D380C416D506A4
:10FCA000B1F08617970729F4C280D380CA16DB0605
:10FCB00071F00817190729F482819381E816F90673
:10FCC00031F03D96F093AE30E093AD30C9CF109255
:10FCD000B2301092B13082E08093AC3088EC9BE27D
:10FCE0009093A72B8093A62B109248311092473106
:10FCF0000E940C778091473190914831009709F428
:10FD000012C59C01245E3F4F3093A52B2093A42B5A
:10FD10003093AE2B2093AF2BE091AD30F091AE300D
:10FD200020852093B42B21E12093B52B08969827AA
:10FD3000892798279093C52B8093C42B1092C72BAB
:10FD40001092C62B848195819093C12B8093C02BF8
:10FD5000868197819093C32B8093C22B80914331EE
:10FD600090914431A0914531B09146318093B82BA8
:10FD70009093B92BA093BA2BB093BB2B8081918128
:10FD8000A281B3818093BC2B9093BD2BA093BE2BFB
:10FD9000B093BF2B84ED9BE29093B0308093AF3053
:10FDA0000E944C7B80959095009711F48FEF9FEF08
:10FDB0009093C72B8093C62B93C40E94497B0196D6
:10FDC00009F0B1C48091C22B9091C32B009709F424
:10FDD000AAC42091C02B3091C12B2115310509F403
:10FDE000A2C44091B82B5091B92B6091BA2B70915D
:10FDF000BB2BECECF0E3C3EBD0E3F080FF20A9F0E9
:10FE0000AC81BD818A179B0781F4AE81BF812A171F
:10FE10003B0759F4A881B9814A175B0731F4AA81DD
:10FE2000BB816A177B0709F46FC1A096B096A1E366
:10FE3000C333DA0711F72091CD2B2F732230D9F479
:10FE40009093EB1A8093EA1A40E0443090F4E42F48
:10FE5000F0E0EE0FFF1FED5CFE4C208131814F5F23
:10FE60008217930791F71092ED1A20E0C0E0D0E0DE
:10FE70007EC04093ED1A8091CD2B82FD54C484E165
:10FE80008093CD2B88E290E09093A52B8093A42BB8
:10FE900080E58093CC2B8091C72B9091CB2B9093B6
:10FEA000C72B3091C62B9091CA2B9093C62B3093C1
:10FEB000CA2B2091C52B9091C92B9093C52B2093D1
:10FEC000C92B9091C42B9093ED1A4091C82B40936D
:10FED000C42B9093C82B8F5F8093CB2B81110FC0C5
:10FEE00081E0830F8093CA2B811109C081E0820FCA
:10FEF0008093C92B811103C09F5F9093C82B809181
:10FF0000C02B9091C12B9093EB1A8093EA1A209109
:10FF1000C22B3091C32B3093C12B2093C02B9093D5
:10FF2000C32B8093C22B8091B82B9091B92BA091B9
:10FF3000BA2BB091BB2B8093BC2B9093BD2BA0937D
:10FF4000BE2BB093BF2B8091433190914431A0914F
:10FF50004531B09146318093B82B9093B92BA09343
:10FF6000BA2BB093BB2BA1C3373089F02F5F24305D
:10FF7000C0F430E2239FC0011124FC01ED54FF4C7A
:10FF8000318D3111F1CF2093ED1AEF010CC0209784
:10FF900021F0428D3A8D341748F7EC01CD54DF4CF7
:10FFA000E5CF2093ED1A209709F4BDC3D093B2306A
:10FFB000C093B13083E08A8F888F1E8A84E08F8B54
:10FFC0001B8E8091C22B9091C32B9D838C8380913B
:10FFD000C02B9091C12B9F838E838091B82B9091E1
:10FFE000B92BA091BA2BB091BB2B88839983AA839C
:10FFF000BB8381E0898F8091F01A8C878091F11A00
:020000021000EC
:100000008D878091F21A8E878091F31A8F8781E015
:1000100090E0998B888B8091C72B8B878091C62B22
:100020008A878091C52B89878091C42B888781E03E
:1000300090E00E94F7838091CC2B282F207F30E026
:10004000213531050CF445C082958F7090E00597FD
:10005000880F991F880F991F3091EC1A20E0E22F2A
:10006000F0E0E817F9078CF5E455F44D30A53111AF
:1000700005C02093ED1A1092EC1A2BC0313011F408
:100080002F5FEDCF3230E1F441A54430C9F4209325
:10009000ED1A3093EC1A82A590E0982F882723A5BB
:1000A000822B9093EB1A8093EA1A893DA4E09A0779
:1000B00010F088ED94E09B8B8A8B9D8B8C8B09C014
:1000C00041A5442311F0240FCACF2093ED1A309399
:1000D000EC1A80E18093CD2B8091CD2B82608093B0
:1000E000CD2B82E08093D42B84E08093D52B80931A
:1000F000D62B88ED8093D72B8CE290E09093A52BA4
:100100008093A42B80E67EC2D093B230C093B130EE
:100110001092AC309091CD2B92FF03C0198E80E2EB
:100120001AC28091CC2B82958F70880F880F809394
:10013000ED1A081B1109045111091093A52B009306
:10014000A42B8F2D8F70823029F4892F8F738231E9
:1001500039F41FC0813021F4892F8F738230C9F0A8
:10016000012B19F4892F8370A1F02091C42B88856D
:1001700028133EC22091C52B8985281339C22091AE
:10018000C62B8A85281334C22091C72B8B85281350
:100190002FC294FF4AC0688979896115710509F4F5
:1001A00044C0CE010C960E94F77A3091C82B809102
:1001B000A82B38133AC02091C92B8091A92B281362
:1001C00034C09091CA2B8091AA2B98132EC0809195
:1001D000CB2B4091AB2B841328C03C872D879E8767
:1001E0008F878B8D81111AC02E89888D9A8D891BDE
:1001F000922F969596959695891B280F2E8B87FDA5
:1002000081959F89392F36953695931B980F9F8B33
:10021000822F869586958695890F888F81E08093B9
:10022000AC30888D8A8F198A188A498D842F8F70F7
:1002300090E0FC013197E830F10508F074C2E05716
:10024000FF4F0C94C68D8091AC3080FF14C083E0CA
:10025000898F80E48093AC30198A188A8091A42B0E
:100260009091A52B009709F408C122E42093AC30AB
:100270000E94F78302C18091CD2B8F73823009F0E9
:1002800052C227CF8091AC3080FF70C08091CD2BBF
:100290008F73823109F06AC08091CC2B282F207F88
:1002A00030E0213531050CF445C082958F7090E027
:1002B0000597880F991F880F991F3091EC1A20E03D
:1002C000E22FF0E0E817F9078CF5E455F44D30A57E
:1002D000311105C02093ED1A1092EC1A2BC0313069
:1002E00011F42F5FEDCF3230E1F441A54430C9F471
:1002F0002093ED1A3093EC1A82A590E0982F88276E
:1003000023A5822B9093EB1A8093EA1A893D24E06F
:10031000920710F088ED94E09B8B8A8B9D8B8C8BE1
:1003200009C041A5442311F0240FCACF2093ED1A30
:100330003093EC1A83E0898F8091C42B8887809159
:10034000C52B89878091C62B8A878091C72B8B8785
:1003500081E090E00E94F78382E48093AC30198AB8
:10036000188A1092A52B1092A42B87C080E280934C
:10037000AC300E940C77E091B130F091B230118E28
:100380007ACD8091CD2B80FF28C044FD26C088897E
:100390009989892B09F0C7C18091A42B9091A52B35
:1003A00001960E94F7832091AC30822F8061809368
:1003B000AC308091A42B9091A52B892B19F0226150
:1003C0002093AC300E940C7781E090E0998B888B71
:1003D00088E0898F1B8E81E10CC185FF1CC0809154
:1003E000D22B90E0982F88272091D32B822B20911D
:1003F000AF303091B030280F391F3093B030209398
:10040000AF302091A42B3091A52B281B390B3093B2
:10041000A52B2093A42B8091A42B9091A52B009722
:1004200049F044FD07C02091AC3022602093AC30ED
:100430000E94F7838091CE2B90E0982F88272091FF
:10044000CF2B820F911D9093EB1A8093EA1A2C897F
:100450003D892817390710F0892B21F43093EB1AC6
:100460002093EA1A8091EA1A9091EB1A9B8B8A8B5F
:100470008091AC30837009F456C1109248311092CB
:1004800047310E940C778091AC3085FF07C01092F5
:10049000483110924731198E84E1ABC084FF0AC005
:1004A000109248311092473181E090E0998B888B0F
:1004B00084E08FCF209147313091483121153105AB
:1004C000E1F080FF02C0198A188A8889998900970B
:1004D00081F48A899B898217930720F4909348318D
:1004E000809347318091473190914831998B888B27
:1004F00004C090934831809347311B8E8091A62B86
:100500009091A72B9093B0308093AF30809147317A
:1005100090914831892B59F088899989009739F051
:1005200088969093A52B8093A42B88E10BC0809193
:10053000AC3081FFF8C088E290E09093A52B8093C7
:10054000A42B80E18093CD2B5CC08091AC3080FFE8
:10055000EAC0198E80E18093AC300E940C77E3C032
:100560008091A42B9091A52B009711F00E94F78306
:100570009091CD2B8091AC3090FF0BC080FF06C0D6
:1005800087E0898F1A8E198A188A19C086E0898FA8
:1005900016C080FF1EC085E0898F198A188AC3C0E3
:1005A0008091A42B9091A52B009711F00E94F783C6
:1005B0008091CD2B80FF0DC087E0898F1A8E81E05E
:1005C00090E00E94F78380E18093AC300E940C772A
:1005D0000FC08091A42B9091A52B892B49F4A3C027
:1005E0008091AC3080FF9FC087E0898F1A8E9BC0BE
:1005F00080E18093CD2B88E290E09093A52B8093AF
:10060000A42B80E58093CC2B88858093C82B89858B
:100610008093C92B8A858093CA2B8B858093CB2BA3
:100620008C858093C42B8D858093C52B8E8580937C
:10063000C62B8F858093C72B86E08093B52B8C814A
:100640009D819093C12B8093C02B8E819F8190932D
:10065000C32B8093C22B8091433190914431A09160
:100660004531B09146318093B82B9093B92BA0932C
:10067000BA2BB093BB2B88819981AA81BB818093CF
:10068000BC2B9093BD2BA093BE2BB093BF2B898D19
:1006900084FF05C01092CF2B1092CE2B06C084E0B1
:1006A0008093CE2B88ED8093CF2B80E48093B42B66
:1006B0008091A42B9091A52B9093AE2B8093AF2B80
:1006C0001092D32B1092D22B1092D12B1092D02BB0
:1006D0000E94497B809590959093D12B8093D02B4D
:1006E00085E48093AC2B1092AD2B1092B32B10921B
:1006F000B22B8091F41A9091F51A01969093F51A05
:100700008093F41A9093B02B8093B12B1092B72B57
:100710001092B62B0E94387B809590959093B72BC2
:100720008093B62B04C01092A52B1092A42B10928C
:10073000AC30DF91CF911F910F91FF90EF90DF9040
:10074000CF90BF90AF900895982789279827089554
:100750000E94CC8D0895FC018091A62B9091A72B2F
:100760002CEA30E3281B390BAB01261737070CF4B2
:10077000A9011416150654F450934831409347319B
:10078000E817F90719F0BF010C94FB91089580E870
:1007900080936100109261000E947D620E94DD538F
:1007A0000E9459668091532990915429009729F00D
:1007B00001979093542980935329C0905529D09044
:1007C0005629E0905729F09058290E941765C616BF
:1007D000D706E806F90611F30E94176560935529BC
:1007E000709356298093572990935829D7CF2091F9
:1007F000B1303091B230BC01C90108960E94F77A3D
:10080000E091B130F091B2308091A82B8087809137
:10081000A92B81878091AA2B82878091AB2B83871C
:1008200008952F923F924F925F926F927F928F9294
:100830009F92AF92BF92CF92DF92EF92FF920F936F
:100840001F93CF93DF93CDB7DEB763970FB6F894BE
:10085000DEBF0FBECDBF7C011B016A01FC01178208
:100860001682838181FF66C3BE016F5F7F4F4B019C
:10087000F7019381F10193FD859193FF81911F0110
:10088000882309F453C3853239F493FD859193FF8E
:1008900081911F01853239F4B70190E00E947E9268
:1008A00056016501E5CF10E0512C20E02032A0F484
:1008B0008B3269F030F4803259F0833269F4206170
:1008C0002CC08D3239F0803339F4216026C022608B
:1008D000246023C0286021C027FD27C030ED380FD9
:1008E0003A3078F426FF06C0FAE01F9F300D11243D
:1008F000132F13C06AE0569E300D1124532E206230
:100900000CC08E3221F426FD11C3206406C08C3643
:1009100011F4206802C0883641F4F10193FD8591FD
:1009200093FF81911F018111C1CF9BEB980F9330F1
:1009300018F42061805E06C09BE9980F933008F0A0
:10094000AAC12F7E26FF16E02F73722E853621F462
:10095000F22FF0647F2E08C0863621F4622F606883
:10096000762E02C01111115077FE07C01C3348F4D7
:1009700044244394410E27E00BC0183030F4212F5B
:1009800006C027E04CE3442E03C027E017E0412CCB
:10099000560174E0A70EB11CF6016081718182815D
:1009A0009381042DA4010E9403916C01098100FF31
:1009B00002C003FF06C071FC07C072FC08C0612CB6
:1009C00008C03DE2632E05C02BE2622E02C090E219
:1009D000692E802F8C7099F1662011F084E001C09F
:1009E00083E0851510F0512C0BC0581A73FC08C019
:1009F000B70180E290E00E947E925A94C9F7F3CF4B
:100A0000662029F0B701862D90E00E947E9203FDBA
:100A100003C00EE011E102C00AE011E1F72DF07110
:100A20007F2EF8018491882309F476C271108052D8
:100A3000B70190E00E947E920F5F1F4FF2CF77FECA
:100A40000FC04C0C04FF04C08A81813309F44A941E
:100A5000141474F5F8E0F41578F588E0482E2CC0ED
:100A600076FC2AC0812F90E08C159D059CF06CEFE0
:100A7000C6166FEFD60674F0772D7068772E0AC011
:100A8000E2E0F0E0EC0FFD1FE10FF11D808180330B
:100A900019F411501111F4CF77FE0EC04424439481
:100AA000410E812F90E0C816D9062CF41C1904C001
:100AB0004424439401C010E077FE07C01C141D04B9
:100AC0003CF496012F5F3F4F05C025E030E002C0A7
:100AD00021E030E0662011F02F5F3F4F112331F00D
:100AE000412F50E04F5F5F4F240F351F452D50E0E1
:100AF0002417350714F4521A01C0512C872D897020
:100B000049F4552039F0B70180E290E00E947E92CE
:100B10005A94F7CF662029F0B701862D90E00E9405
:100B20007E9273FC09C0552039F0B70180E390E054
:100B30000E947E925A94F7CF77FE5FC09C2D8D2D38
:100B4000D7FE02C090E080E0692E782E40E050E0B1
:100B5000C601841991099D878C879601261937094A
:100B6000280D391D812F90E0EE27FF27E81BF90B98
:100B7000FF87EE87FFEF6F167F0669F4B7018EE2FD
:100B800090E02B8B3A8B488B598B0E947E9259892F
:100B900048893A892B89C614D70454F06C857D8521
:100BA000661577052CF4F901E40FF51F818101C06A
:100BB00080E371E0671A71084F5F5F4FEE85FF8534
:100BC0006E167F066CF0B70190E02B8B3A8B488B4A
:100BD000598B0E947E922B893A8948895989CACFBC
:100BE0006C147D0439F49A81963318F4953311F41A
:100BF00004FF81E3B70190E04BC08A81813309F0A3
:100C00000F7EB70190E00E947E92111105C074FE24
:100C100018C085E490E017C0B7018EE290E00E9412
:100C20007E9282E066246394680EF401E80FF11D61
:100C30008081B70190E00E947E92115041F3862D91
:100C4000F1CF85E690E0B7010E947E92D7FC05C007
:100C5000C114D10439F404FF05C0D194C194D10862
:100C60008DE201C08BE2B70190E00E947E9280E3AA
:100C70006AE0C616D1042CF08F5FFAE0CF1AD108D3
:100C8000F7CFB70190E00E947E92B701C601C096EF
:100C90000E947E9241C1833631F0833779F08335EB
:100CA00009F058C021C0560172E0A70EB11CF60130
:100CB0008081898301E010E0640114C05601F2E0F4
:100CC000AF0EB11CF601C080D18026FF03C0612F9A
:100CD00070E002C06FEF7FEFC6012B8B0E942A925B
:100CE0008C012B892F7715C05601F2E0AF0EB11C95
:100CF000F601C080D18026FF03C0612F70E002C0E2
:100D00006FEF7FEFC6012B8B0E94EC918C012B893A
:100D10002068722E23FD1AC0852D90E00817190750
:100D2000A8F4B70180E290E00E947E925A94F4CF3A
:100D3000F60177FC859177FE81916F01B70190E014
:100D40000E947E9251105A9401501109011511050B
:100D500079F7E2C0843611F0893651F5560127FF44
:100D600009C0F4E0AF0EB11CF6016081718182818F
:100D700093810AC0F2E0AF0EB11CF601608171816F
:100D8000882777FD8095982F022F0F7697FF08C050
:100D900090958095709561957F4F8F4F9F4F00681C
:100DA0002AE030E0A4010E94B893C82EC8183EC0C3
:100DB000022F853721F40F7E2AE030E01DC0097F25
:100DC0008F3691F018F4883559F0B0C0803719F09B
:100DD000883711F0ABC0006104FF09C0046007C090
:100DE00024FF08C0066006C028E030E005C020E10E
:100DF00030E002C020E132E0560107FF09C0F4E014
:100E0000AF0EB11CF601608171818281938108C0AF
:100E1000F2E0AF0EB11CF6016081718180E090E0DC
:100E2000A4010E94B893C82EC8180F7706FF0BC004
:100E3000202F2E7FC11650F404FF0AC002FD08C007
:100E4000202F2E7E05C0DC2C202F03C0DC2C01C0FF
:100E5000D12E24FF0DC0FE01EC0DF11D80818033E9
:100E600011F4297E09C022FF06C0D394D39404C094
:100E7000822F867809F0D39423FD13C020FF06C08B
:100E80001C2DD51418F4150D1D19D52CD51468F486
:100E9000B70180E290E02B8B0E947E92D3942B8945
:100EA000F5CFD51410F45D1801C0512C24FF12C0E9
:100EB000B70180E390E02B8B0E947E922B8922FF6A
:100EC00017C021FF03C088E590E002C088E790E0EA
:100ED000B7010CC0822F867859F021FD02C080E254
:100EE00001C08BE227FD8DE2B70190E00E947E9267
:100EF000C11638F4B70180E390E00E947E92115051
:100F0000F7CFCA94F401EC0DF11D8081B70190E098
:100F10000E947E92C110F5CF552009F4C2CCB701D2
:100F200080E290E00E947E925A94F6CFF70186818B
:100F3000978102C08FEF9FEF63960FB6F894DEBFE4
:100F40000FBECDBFDF91CF911F910F91FF90EF901A
:100F5000DF90CF90BF90AF909F908F907F906F90D9
:100F60005F904F903F902F9008955058BB27AA272D
:100F70000ED04EC23FD230F044D220F031F49F3F29
:100F800011F41EF4FFC10EF4E095E7FBF5C1E92F63
:100F900050D280F3BA17620773078407950718F0D9
:100FA00071F49EF568C20EF4E0950B2EBA2FA02DB9
:100FB0000B01B90190010C01CA01A0011124FF2706
:100FC000591B99F0593F50F4503E68F11A16F04001
:100FD000A22F232F342F4427585FF3CF4695379500
:100FE0002795A795F0405395C9F77EF41F16BA0BC5
:100FF000620B730B840BBAF09150A1F0FF0FBB1F73
:10100000661F771F881FC2F70EC0BA0F621F731FBB
:10101000841F48F4879577956795B795F7959E3F18
:1010200008F0B3CF9395880F08F09927EE0F9795A6
:1010300087950895DFD158F080E891E009F49EEF9C
:10104000E0D128F040E851E059F45EEF09C09AC1C0
:1010500012C2E92FE078EDD168F3092E052AC1F319
:10106000261737074807590738F00E2E07F8E025EE
:1010700069F0E025E0640AC0EF6307F8009407FA1E
:10108000DB01B9019D01DC01CA01AD01EF9347D03D
:10109000BFD10AD05F91552331F02BED3FE049E4F9
:1010A00050FD49EC63CF0895DF93DD27B92FBF775B
:1010B00040E85FE31616170648075B0710F4D92FC0
:1010C000E5D19F938F937F936F934AD3E0E3F1E051
:1010D0006CD19ED12F913F914F915F919ED2DD2394
:1010E00049F09058A2EA2AED3FE049EC5FE3D0785E
:1010F0005D274DDFDF918CC11BD108F481E008959D
:101100000CD086C17ED140F075D130F021F45F3F24
:1011100019F032C15111B0C135C18BD198F3992367
:10112000C9F35523B1F3951B550BBB27AA276217AB
:101130007307840738F09F5F5F4F220F331F441FF0
:10114000AA1FA9F333D00E2E3AF0E0E830D0915028
:101150005040E695001CCAF729D0FE2F27D0660F15
:10116000771F881FBB1F261737074807AB07B0E854
:1011700009F0BB0B802DBF01FF2793585F4F2AF06A
:101180009E3F510568F0F8C077C15F3FECF3983E91
:10119000DCF3869577956795B795F7959F5FC9F7C7
:1011A000880F911D9695879597F90895E1E0660F50
:1011B000771F881FBB1F621773078407BA0720F0C9
:1011C000621B730B840BBA0BEE1F88F7E095089532
:1011D00019F40EF0D1C04FC1D5C033D1C8F3963841
:1011E000C0F707F80F92E8942BE33AEA48EB5FE781
:1011F00016D20F920F920F924DB75EB70F92CED1CB
:10120000EDE5F1E0D2D04F915F91EF91FF91E5953F
:10121000EE1FFF1F49F0FE57E0684427EE0F441F02
:10122000FA95E1F74195550B3AD10F9007FE2EC183
:10123000089597FB0EF4A9D03EC0E89409C097FB2F
:101240003EF490958095709561957F4F8F4F9F4F9D
:101250009923A9F0F92F96E9BB279395F6958795E1
:1012600077956795B795F111F8CFFAF4BB0F11F4A4
:1012700060FF1BC06F5F7F4F8F4F9F4F16C088234B
:1012800011F096E911C0772321F09EE8872F762F81
:1012900005C0662371F096E8862F70E060E02AF0C2
:1012A0009A95660F771F881FDAF7880F96958795AE
:1012B00097F90895E894F92F96EBFF2381F0121621
:1012C00013061406440B9395F695879577956795C5
:1012D00057954040FF23B9F71BC0992708958823ED
:1012E00051F49850D2F7872B762F652F542F432F28
:1012F000322F20E0B1F3121613061406440B882394
:101300003AF09A95440F551F661F771F881FCAF73A
:1013100055234AF4440F551F11F460FF04C06F5F5A
:101320007F4F8F4F9F4F880F9695879597F9089518
:10133000990F0008550FAA0BE0E8FEEF16161706E6
:10134000E807F907C0F012161306E407F50798F04E
:10135000621B730B840B950B39F40A2661F0232B67
:10136000242B252B21F408950A2609F4A140A695E3
:101370008FEF811D811D089597F99F6780E870E0C8
:1013800060E008959FEF80EC0895909580957095AA
:10139000609550954095309521953F4F4F4F5F4F49
:1013A0006F4F7F4F8F4F9F4F0895DF93CF931F93C2
:1013B0000F93FF92EF92DF927B018C01689405C03E
:1013C000DA2EEF012AD1FE01E894A59125913591FD
:1013D00045915591AEF3EF01DADDFE019701A801C9
:1013E000DA9479F7DF90EF90FF900F911F91CF91F2
:1013F000DF91089500240A941616170618060906A8
:10140000089500240A94121613061406050608957A
:10141000092E0394000C11F4882352F0BB0F40F402
:10142000BF2B11F460FF04C06F5F7F4F8F4F9F4F42
:10143000089557FD9058440F551F59F05F3F71F0C4
:101440004795880F97FB991F61F09F3F79F087952B
:101450000895121613061406551FF2CF4695F1DFB4
:1014600008C0161617061806991FF1CF8695710544
:10147000610508940895E894BB2766277727CB0178
:1014800097F9089555DF08F48FEF08959B01AC019B
:1014900060E070E080E89FE333CE6ECF64C1D1DFBF
:1014A000E8F39923D9F3940F511DBBF391505040A9
:1014B00094F059F0882332F0660F771F881F9150FF
:1014C0005040C1F79E3F510544F7880F911D9695F6
:1014D000879597F908955F3FACF0983E9CF0BB2745
:1014E000869577956795B79508F4B1609395C1F7A0
:1014F000BB0F58F711F460FFE8CF6F5F7F4F8F4F3E
:101500009F4FE3CFB9CF0AD029ED3BE54EED5EE327
:1015100078C00EF028C136CF68942ECF92DFC8F382
:101520009923D1F3C6F3DF93CF931F930F93FF92C9
:10153000C92FDD2788232AF02197660F771F881F80
:10154000DAF720E030E040E85FEB9FE3883920F0F5
:10155000803E30F021968F7709DDE5E8F1E003C0A9
:1015600005DDE2EBF1E021DF8B01BE01EC01FB2E9A
:101570006F5771097595771F880B990B60DE28E10D
:1015800032E741E35FE349D0AF2D9801AE01FF9010
:101590000F911F91CF91DF91FADC3ACFFA01DC0174
:1015A000AA0FBB1F9B01AC01BF5728F4222733278A
:1015B000442750781FC0B75188F4AB2F00244695BC
:1015C00037952795011CA395D2F3002069F0220FCF
:1015D000331F441FB395DAF30DD0C7CC61307105CA
:1015E000A0E88A07B94630F49B01AC01662777274B
:1015F00088279078309621F020833183428353836B
:1016000008950BD005CFF6DE28F0FBDE18F0952309
:1016100009F0B2CEB7CE11242FCF0BDFA0F3959FE8
:10162000D1F3950F50E0551F629FF001729FBB27C9
:10163000F00DB11D639FAA27F00DB11DAA1F649F75
:101640006627B00DA11D661F829F2227B00DA11D28
:10165000621F739FB00DA11D621F839FA00D611DAE
:10166000221F749F3327A00D611D231F849F600DCF
:10167000211D822F762F6A2F11249F5750408AF008
:10168000E1F088234AF0EE0FFF1FBB1F661F771F94
:10169000881F91505040A9F79E3F510570F06CCEC5
:1016A000EBCE5F3FECF3983EDCF38695779567953C
:1016B000B795F795E7959F5FC1F7FE2B880F911DB2
:1016C0009695879597F90895FA01EE0FFF1F3096CA
:1016D0002105310599F16115710561F48038BFE389
:1016E0009B0749F168949038810561F08038BFEF1D
:1016F0009B0741F0992342F5FF3FE10531052105A4
:1017000011F1E8940894E795D901AA2329F4AB2FA5
:10171000BE2FF85FD0F310C0FF5F70F4A695E0F71E
:10172000F73950F019F0FF3A38F49F779F930CD0B7
:101730000F9007FC905808953EF024CE60E070E0D2
:1017400080E89FE308954FE79F775F934F933F9320
:101750002F93E4DE2F913F914F915F9152DF3DCD6A
:101760009B01AC014ECF9F3F31F0915020F4879503
:1017700077956795B795880F911D9695879597F9F9
:1017800008950E94C98B332312F48A1B9B0B0C947F
:10179000DA8BA29FB001B39FC001A39F700D811D82
:1017A0001124911DB29F700D811D1124911D08956A
:1017B0000E94C98BB7FF0895821B930B08950E9466
:1017C000C98BA59F900DB49F900DA49F800D911D76
:1017D00011240895B7FF0C94DF8B0E94DF8B821BCE
:1017E000930B0895DB018F939F930E94DF8BBF9132
:1017F000AF91A29F800D911DA39F900DB29F900D60
:1018000011240895AA1BBB1B51E107C0AA1FBB1FCF
:10181000A617B70710F0A61BB70B881F991F5A957C
:10182000A9F780959095BC01CD01089597FB072EEF
:1018300016F4009407D077FD09D00E94028C07FCB3
:1018400005D03EF4909581959F4F089570956195D0
:101850007F4F0895A1E21A2EAA1BBB1BFD010DC0EC
:10186000AA1FBB1FEE1FFF1FA217B307E407F50750
:1018700020F0A21BB30BE40BF50B661F771F881F2C
:10188000991F1A9469F760957095809590959B01C2
:10189000AC01BD01CF010895052E97FB1EF4009405
:1018A0000E94778D57FD07D00E942A8C07FC03D039
:1018B0004EF40C94778D50954095309521953F4F7F
:1018C0004F4F5F4F0895689401C0E894F92FF12BB2
:1018D00012F00C94978CA0E0B0E0E1E7FCE80C94E7
:1018E000958D092E059422F40E947F8D112392F488
:1018F000F0E80F26FFEFE094F09400951095B09477
:10190000C094D094A194BF0ACF0ADF0AEF0AFF0A5D
:101910000F0B1F0B0E94268D07FC0E947F8DCDB7F9
:10192000DEB7ECE00C94B18D689401C0E8948F921E
:101930009F92CF93DF930E94268DDF91CF919F904E
:101940008F900895DF93CF931F930F939A9DF02D5F
:10195000219FF00D8B9DF00D8A9DE02DF10D039FD1
:10196000F00D029FE00DF11D4E9DE00DF11D5E9DFD
:10197000F00D4F9DF00D7F936F93BF92AF925F93E9
:101980004F93D5010E94C98B8B01AC01D7010E94F6
:10199000C98BEB01E80FF91FD6010E94F28C2F9141
:1019A0003F91D6010E94C98BC60FD71FE81FF91FB0
:1019B000AF91BF910E94F28C2F913F910E94C98BF1
:1019C000C60FD71FE81FF91FD6010E94C98BE60F6B
:1019D000F71F9801BE01CF0111240F911F91CF91E4
:1019E000DF9108950E94C98B460F571FC81FD91F4A
:1019F00008F431960895E894DF93CF93FC01DB015E
:101A00000E94C98B7F936F93E9019A01AC01BF9348
:101A1000AF933F932F93DF010E94C98B26F46C1B79
:101A20007D0B820B930B9E01EB01FC010E94F28C5B
:101A3000AF91BF912F913F910E94F28CBE01CF01D7
:101A4000F9012F913F91CF91DF9108958824992436
:101A5000F401E401B0E49F93AA279A158B049C0437
:101A6000ED05FE05CF05D007A10798F4AD2FDC2FBB
:101A7000CF2FFE2FE92D982C892E982F872F762F88
:101A8000652F542F432F322F2227B85031F7BF91A3
:101A900027C01B2EBF91BB27220F331F441F551F8A
:101AA000661F771F881F991F881C991CEE1FFF1F38
:101AB000CC1FDD1FAA1FBB1F8A149B04EC05FD056C
:101AC000CE05DF05A007B10748F08A189B08EC098E
:101AD000FD09CE09DF09A00BB10B21601A94E1F6D4
:101AE0002EF49401AF01BE01CD01000C0895909534
:101AF0008095709561957F4F8F4F9F4F08956095AA
:101B000070958095909530954095509521953F4FD3
:101B10004F4F5F4F6F4F7F4F8F4F9F4F08952F92C3
:101B20003F924F925F926F927F928F929F92AF926D
:101B3000BF92CF92DF92EF92FF920F931F93CF93BA
:101B4000DF93CDB7DEB7CA1BDB0B0FB6F894DEBF51
:101B50000FBECDBF09942A88398848885F846E8477
:101B60007D848C849B84AA84B984C884DF80EE80C1
:101B7000FD800C811B81AA81B981CE0FD11D0FB6CA
:101B8000F894DEBF0FBECDBFED010895EE0FFF1F2D
:101B90000590F491E02D0994692796276927782705
:101BA0008727782708950F93083090F0982F872F74
:101BB000762F652F542F432F322F22270850F4CF32
:101BC000220F331F441F551F661F771F881F991F41
:101BD0000A95B2F70F91089597FB10F81694000834
:101BE0000F93083098F00850232F342F452F562F8D
:101BF000672F782F892F902DF4CF0594979587958F
:101C00007795679557954795379527950A95AAF73C
